:100000000C94B8500C94E9500C94E9500C94E950BD
:100010000C94E9500C94E9500C94E9500C94E9507C
:100020000C94E9500C94E9500C94E9500C94E9506C
:100030000C94C0740C94E9500D9459150D949D12B4
:100040000C94E9500D94F6220C94E9500C94E9506C
:100050000C94E9500C94E9500C94E9500C94396DCF
:100060000C94E9500D94049A0C94E9500C94E950C6
:100070000C94E9500C946F7D0C94E9500C94E95069
:100080000D94A7170C94E9500C94E9500C94E95086
:100090000D94C0990C94E9500C94E9500C94E950DB
:1000A0000C94E9500C94E9500D94E50D0C94E95032
:1000B0000C94E9500D94C70D0C94E9500C94E95040
:1000C0000C94E9500C94E9500C94E9500D94870D70
:1000D0000C94E9500C94E9500C94E9500C94E950BC
:1000E0000C94E95000000000000000000000000037
:1000F0000000000000000000000000000000000000
:10010000A55AB44B2B30810134B7736520AA51A690
:10011000130341036A03A603CB031B0442048004B8
:10012000B7040C0543056D0580059505A805BC05BC
:10013000CC05DC05ED051F064306580673069C0634
:10014000AD06BC06D10619073D077607850790075F
:100150009907A1071203A807B107C307D607E70746
:10016000F707060811081D0828083A084B085B081D
:100170006C087F088A0812039708A108B408C5080C
:100180001203E608F00802090E091E0926093909BA
:100190004C0959096509780988099609A809B70918
:1001A000C909D909EA09FB09010A130A1F0A270A22
:1001B000380A4A0A560A5D0A650A6C0A710A7D0AFB
:1001C0008F0A950A9F0AAC0AB00ABD0AC30AD10A6F
:1001D0001203D40AE60AF50A230B2F0B3E0B6C0B15
:1001E00012037F0B900B9E0BB20BB60BC70BD40BFD
:1001F000E50B1203F40B070C190C290C390C4E0CEF
:10020000580C680C770C830C930CA80CB70CC10C21
:10021000D60CE40CF60C070D180D290D3A0D4B0DFC
:10022000510D5B0D630D680D730D7C0D820D8A0DF4
:10023000C00DF50D080E110E240E380E540E820E50
:10024000D20EF30E4A0FA80F0B106210AB10D41091
:10025000F9100011131126113711461158119E1172
:10026000F0112B126E12AD12EA12241351139B13CC
:10027000BF133814CE14F1141A1550155D157215EC
:10028000831592159F15AE15BE15D2151203E015F4
:10029000F115FC150C161A162D16411650165D1682
:1002A0006A16761689169B16AE16BA16C816CF169B
:1002B000E316F716051717172B17401752175A177B
:1002C00088179117DC17EC17FE170E181D1812036C
:1002D000321847185118591866187318801893184F
:1002E0009D18AA18B718C418D318E5180D19751950
:1002F000DB19FC19661A6F1A771A7F1A871ABA1A4D
:10030000D61ADF1A371B5E1BA81BFF1BA61CD81CA6
:100310003A1D901DBC1DE01DFE1D601E801EC31EEB
:100320002A1F651FB11F0520202049206A20982020
:10033000BE20F22041219D2147224D221203572247
:1003400065226E22772286228B2298229F22A82263
:10035000BD221203CF22E122F62209231C232D23E2
:10036000412355236A237B2389239D23A923BC236F
:10037000CE23DB23EE23032418242D2442245224ED
:100380001203652477248B249F24AF24C224D6240F
:10039000E124F024002513251203232536254725C3
:1003A0005C256D257E259125A625B925CC25E02542
:1003B000F125062619262C263E2652266726792662
:1003C0008C269C26AC26C126EB26FE264E275527DA
:1003D00059275D277A27C52702288028C528302974
:1003E0006129EA29322A712AA52ABA2A122B372B27
:1003F000912B142CAC2C462DAA2D342EB32E452F28
:10040000AE2FB62FBC2FC32F1203C92FD02F1E30F3
:10041000FB090050726F626C656D6120656E636FE1
:100420006E747261646F2C206E6976656C616369AD
:10043000AD6E205A20666F727A6F7361202E2E2E59
:10044000004E6976656C616369AD6E2066616C6CA7
:100450006964612E20496D7072657369AD6E2063A9
:10046000616E63656C6164612E0043616C656E74DE
:1004700061646F726573206465736163746976612A
:10048000646F7320706F7220656C2074656D706F7F
:1004900072697A61646F7220646520736567757232
:1004A000696461642E0043AD6469676F2047206C06
:1004B000616D696E61646F207061726120756E207C
:1004C0006E6976656C206469662E0043AD64696769
:1004D0006F2047206C616D696E61646F207061727E
:1004E0006120756E206E6976656C20646966657240
:1004F000656E74652E205675656C76652061206C7E
:10050000616D696E617220656C206D6F64656C6FE2
:10051000206465206E7565766F2E0043AD64696753
:100520006F2047206C616D696E61646F207061722D
:1005300061206E7565766F206669726D7761726590
:100540002E0043AD6469676F2047206C616D696E52
:1005500061646F2070617261206E7565766F2066D0
:1005600069726D776172652E2041637475616C6983
:100570007A6120656C206669726D776172652E0004
:1005800043AD6469676F2047206C616D696E61647B
:100590006F207061726120756E207469706F2064C5
:1005A0006520696D707265736F7261206469662E73
:1005B000436F6E742E3F0043AD6469676F20472020
:1005C0006C616D696E61646F207061726120756E1F
:1005D0006120696D707265736F7261206469666510
:1005E00072656E74652E205675656C766520612087
:1005F0006C616D696E617220656C206D6F64656CF5
:100600006F206465206E7565766F2E0050756C7373
:100610006120656C206469616C207061726120707A
:10062000726563616C656E746172206C6120626FCB
:100630007175696C6C61207920636F6E74696E7579
:10064000652E0050756C736120656C206469616C67
:1006500020706172612064657363617267617220EA
:10066000656C2066696C616D656E746F00792070D1
:10067000726573696F6E6120656C206469616C00DE
:10068000496E74726F64756369722066696C616D1E
:10069000656E746F00436F6C6F72206E6F20686FB1
:1006A0006D6F679A6E656F0046696C2E206E6F20C5
:1006B000696E74726F64756369646F0043616D6223
:1006C000696F20636F72726563746F0043616D625E
:1006D00069616E646F20636F6C6F720043616D625D
:1006E000696F20636F72726563746F21004162727B
:1006F0006520656C2074656E736F72207920726559
:100700007469726120656C2066696C616D656E74D8
:100710006F206D616E75616C6D656E74652E005332
:10072000652064657363617267AD20636F6E209AA4
:100730007869746F20656C2066696C616D656E7494
:100740006F3F0041637475616C697A6120706F72EC
:10075000206661766F722E004E7565766F20666931
:10076000726D7761726520646973706F6E69626C17
:10077000653A004573706572616E646F2061207127
:10078000756520736520656E6672A265206C6120B8
:10079000736F6E64612050494E444100506F722067
:1007A0006661766F72206573706572610053696E61
:1007B000206D6F76696D69656E746F004573706545
:1007C00072616E646F206F7264656E65732E2E2E7B
:1007D000005365206E6563657369746120756E6191
:1007E0002074656D706572617475726120616D62EF
:1007F00069656E746520656E7465203231207920DC
:10080000323643207920756E20736F706F72746575
:100810002072A26769646F2E005265616C697A610B
:10082000206C612063616C696272616369AD6E20E6
:1008300058595A207072696D65726F2E0050726936
:100840006D65726F20646573636172676120656CAA
:100850002066696C616D656E746F2C206C756567C0
:100860006F207265706974652065737461206163BF
:100870006369AD6E2E00436F6D70726F6261636964
:100880006F6E6573004420626F7175696C6C6100F6
:10089000416C66616265746F004F7264656E61726F
:1008A000005469656D706F005461726A2E20534464
:1008B0000043616D6269617220656C206964696FD3
:1008C0006D610043616D62696F20646520626F71C4
:1008D00075696C6C6100436F6E6669677572616300
:1008E00069AD6E204857005072756562612064657D
:1008F00020636172676100417061676172206D6F92
:10090000746F726573004D6F76657220656A6573EA
:100910000054656D70657261747572610043616C3D
:100920002E2050494E444100526573657420636126
:100930006C6962722E2058595A004D6F737472613F
:100940007220656E6473746F70730043616C6962CA
:1009500072616369AD6E2050494400436F72722E1C
:10096000206465206C612063616D61004E6976656D
:100970006C612E204D616C6C612042617365004397
:10098000616C6962726172205A0043616C696272C3
:1009900061722058595A004173697374656E7465A9
:1009A0000050726F62616E646F2066696C616D6584
:1009B0006E746F00496E74722E20746F646F7320B2
:1009C00066696C2E0052657469726120656C2066E0
:1009D000696C616D656E746F20646520696E6D650C
:1009E000646961746F0052656E6F6D62726172004E
:1009F00043616C2E207072696D6572612063617055
:100A00002E0053656C656363696F6E6172004C8A7A
:100A10006D696E6120646520616365726F00536F5C
:100A2000706F7274650046616C6C6F7320746F74C4
:100A3000616C6573204D4D55005265676973747222
:100A40006F2064652066616C6C6F73004573746120
:100A500064A27374696361730043616C696272615B
:100A60006369AD6E004361726761206175746F2EBA
:100A70002066696C616D2E00496E74726F647563D7
:100A800069722066696C2E004465736361726761E8
:100A90002066696C2E00436172676172206120627A
:100AA0006F7175696C6C610050726563617267612A
:100AB0002061204D4D55004E6F2068617920746192
:100AC000726A657461205344004D656E75207461CF
:100AD000726A657461205344005265616E75646189
:100AE0007220696D707265732E005061757361724A
:100AF00020696D7072657369AD6E004C6973746FB7
:100B000000436F6E6A756E746F206E6F206C697330
:100B1000746F0050726563616C656E746172004140
:100B20006A757374617200416A7573746520656ECD
:100B3000207669766F205A00566F6C766572206158
:100B400020696D7072696D6972004D6F6E69746FA6
:100B500072697A61720041736973742E00556E6117
:100B60002076657A00536F6E69646F00416C746F14
:100B70000053656E736F722046696C2E0043616D81
:100B8000626961722066696C616D656E746F0046A2
:100B90006C756A6F0056656C6F63696461640043CD
:100BA0006F6D702E20696D616E6573004E2F44006D
:100BB0005A2D73656E736F72206E722E004D616CCC
:100BC0006C6100436F6E6669677572616369AD6ED3
:100BD00000536900446574656E657220696D7072BA
:100BE000657369AD6E0056657269662E2061726329
:100BF0006869766F004172636869766F20696E6319
:100C00006F6D706C65746F2E20436F6E74696E75B6
:100C1000617220646520746F646F73206D6F646F00
:100C2000733F008441637475616C697A6172004D31
:100C3000656E75207072696E636970616C004573D2
:100C4000706572616E646F20656E667269616D6950
:100C5000656E746F206465206C612062617365202D
:100C60007920626F7175696C6C612E0053656C65DB
:100C70006363696F6E612066696C616D2E3A00492D
:100C80006E69636961722053656C66746573740084
:100C9000496E74657263616D626961646F00566567
:100CA0006E74732E2066726F6E742F697A71756917
:100CB0002E00456A65004C6F6E6769747564206428
:100CC000656C20656A6500506F6C656120737565A1
:100CD0006C74610046696E206E6F20616C63616E9A
:100CE0007A61646F0046696E206465206361727288
:100CF0006572610046696E616C657320646520638E
:100D0000617272657261004572726F722064652053
:100D1000636F6E657869AD6E00426173652F4361E4
:100D20006C656E7461646F72004E6F20686179202B
:100D3000636F6E657869AD6E0043616C656E74615A
:100D4000646F722F5465726D6973746F7200436FB4
:100D50006E74726F6C613A004572726F72205365E7
:100D60006C6674657374210053656E736F722064D2
:100D7000652066696C2E0056656E742E6675736FFD
:100D8000723A0056656E742E20642E206675736F5D
:100D9000723A0043616C696272617220706F732EE7
:100DA000696E696369616C0046616C6C6F205365A4
:100DB0006C667465737400546F646F206269656E4D
:100DC00000436F6D70726F62616E646F2073656E49
:100DD000736F72657300436F6E74726F6C2066750B
:100DE000736F7200436F6E74726F6C206261736513
:100DF0002063616C2E00436F6E74726F6C2073659C
:100E00006E736F72205A00436F6E74726F6C207332
:100E1000656E736F72205900436F6E74726F6C2031
:100E200073656E736F72205800436F6E74726F6CCF
:100E300020656E6473746F7073005461726A6574B8
:100E400061207265746972616461004174728A73B1
:100E500000456E63656E6469646F004163616C6C2C
:100E60006172004D6F646F0052656E642E706C6528
:100E70006E6F00457374726963746F0041766973B5
:100E80006F004E696E67756E6F004675736F7220E6
:100E90006120323830432120426F7175696C6C617A
:100EA0002063616D626961646F207920616A757386
:100EB000742E2061206C61206D65646964613F005F
:100EC0005061726120756E2063616D62696F20648C
:100ED0006520626F7175696C6C612C206C65650AA8
:100EE00070727573612E696F2F6E6F7A7A6C652DD3
:100EF0006D6B33730043616C2E2050494420746540
:100F0000726D696E6164610043616C2E20504944CA
:100F100000496D7072657369AD6E20656E207061F9
:100F200075736100496D7072657369AD6E206361A0
:100F30006E63656C61646100436F70696172206902
:100F400064696F6D612073656C656363696F6E6161
:100F5000646F3F0044698A6D6574726F20626F71BF
:100F600075696C6C6120696D707265736F72612058
:100F70006469666965726520646520636F642E47E5
:100F80002E0044698A6D6574726F20626F71756995
:100F90006C6C6120496D707265736F726120646959
:100FA000666965726520646520636F642E472E2034
:100FB000436F6D707275656261206C6F732076612E
:100FC0006C6F72657320656E20616A7573746573EA
:100FD0002E004E6F20686179206E696E67C06E20AA
:100FE00066696C616D656E746F20636172676164C0
:100FF0006F2E00546F646176A261206573206E6568
:101000006365736172696F20686163657220756ED4
:10101000612063616C696272616369AD6E205A2EF2
:10102000205369676120656C206D616E75616C2C61
:10103000206361706974756C6F205072696D6572A0
:101040006F73207061736F732E00496D70726573DA
:101050006F7261206E6F206573748A2063616C69A2
:10106000627261646120746F646176A2612E2055A2
:10107000736120656C206D616E75616C20636170B9
:101080006974756C6F205072696D65726F73207032
:1010900061736F732043616C696272616369AD6EE5
:1010A00020666C756A6F2E005365207265616C69ED
:1010B0007A61728A20656C2073656C6674657374DE
:1010C00020706172612063616C6962726172206379
:1010D0006F6E20707265636973696F6E206C61203A
:1010E0007675656C74612061206C6120706F736926
:1010F0006369AD6E20696E696369616C2073696EA6
:101100002073656E736F7265732E0053652068617E
:101110006E20656E636F6E747261646F20616A75B4
:101120007374657320616E746572696F7265732E76
:1011300020536520616A75737461726120656C204B
:101140005049442C206C6F73207061736F7320645E
:10115000656C206578747275736F722C206574638A
:101160002E00417669736F3A2074616E746F20654A
:101170006C207469706F20646520696D707265738E
:101180006F726120636F6D6F20656C207469706F82
:10119000206465206C6120706C6163612068616E01
:1011A0002063616D626961646F2E00417669736FBF
:1011B0003A2068612063616D626961646F20656CCB
:1011C000207469706F20646520696D707265736F3B
:1011D00072612E00417669736F3A20656C207469E4
:1011E000706F20646520706C6163612068612063AA
:1011F000616D626961646F2E004C8A6D696E610079
:1012000056656E74696C61646F72206E6F206769D9
:1012100072610056656E74696C61646F72206769F3
:1012200072616E646F0056656E742E20697A7175F6
:10123000696572646F3F0056656E742E2066726F2A
:101240006E74616C3F00546573742076656E7469CA
:101250006C61646F7265730043616C696272616393
:1012600069AD6E2058595A20636F7272656374615C
:101270002E204C61206465737669616369AD6E20D0
:10128000736520636F7272656769728A2061757415
:101290006F6D8A746963616D656E74652E0043615C
:1012A0006C696272616369AD6E2058595A20636F30
:1012B0007272656374612E204C6F7320656A65736A
:1012C00020582F59206573748A6E206C6967657287
:1012D000616D656E746520646573766961646F73B2
:1012E0002E204275656E2074726162616A6F210002
:1012F00043616C696272616369AD6E2058595A200E
:101300006F6B2E20456A657320582F5920706572C7
:1013100070656E646963756C617265732E20456ECD
:10132000686F72616275656E61210043616C69620C
:1013300072616369AD6E2058595A20636F6D707287
:101340006F6D65746964612E2050756E746F2066D0
:10135000726F6E74616C206465726563686F206E75
:101360006F20616C63616E7A61626C652E0043610F
:101370006C696272616369AD6E2058595A20636F5F
:101380006D70726F6D65746964612E2050756E7436
:101390006F732066726F6E74616C6573206E6F2060
:1013A000616C63616E7A61626C65732E0043616C7F
:1013B000696272616369AD6E2058595A2066616C2A
:1013C0006C61642E2050756E746F2066726F6E743F
:1013D000616C206465726563686F206E6F20616C5C
:1013E00063616E7A61626C652E0043616C69627242
:1013F000616369AD6E2058595A2066616C6C6964EE
:10140000612E2050756E746F732066726F6E7461FA
:101410006C6573206E6F20616C63616E7A61626CC3
:1014200065732E0043616C696272616369AD6E2001
:1014300058595A2066616C6C6964612E20436F6E46
:1014400073756C746120656C206D616E75616C2EB6
:101450000043616C696272616369AD6E2058595ACC
:101460002066616C6C6964612E2050756E746F73B8
:101470002064652063616C696272616369AD6E208E
:10148000656E206C612062617365206E6F20656EF1
:10149000636F6E747261646F732E00436F6C6F6361
:1014A00061206C61206C616D2E2064652061636534
:1014B000726F20656E206C6120626173652E00443E
:1014C000697374616E63696120656E747265206C06
:1014D000612070756E74612064656C20626F717537
:1014E000696C6C612079206C61207375706572661F
:1014F00069636965206465206C61206261736520A1
:1015000061756E206E6F2066696A6164612E20537A
:1015100069676120656C206D616E75616C2C20635C
:1015200061706974756C6F205072696D65726F734C
:10153000205061736F732E00436F6C6F717565205F
:10154000756E6120686F6A612064652070617065E6
:101550006C20646562616A6F206465206C61206242
:101560006F7175696C6C6120647572616E74652051
:101570006C612063616C696272616369AD6E206445
:1015800065206C6F73207072696D65726F732034A3
:101590002070756E746F732E205369206C61206209
:1015A0006F7175696C6C6120636F676520656C2075
:1015B000706170656C2C2061706167756520696E63
:1015C0006D6564696174616D656E74652E00427548
:1015D0007363616E646F2070756E746F2064652034
:1015E00063616C696272616369AD6E20626173658B
:1015F000004D696469656E646F20616C7475726119
:101600002064656C2070756E746F20646520636162
:101610006C696272616369AD6E004C696D7069617D
:1016200020626F7175696C6C6120706172612063FA
:10163000616C696272616369AD6E2E20436C69638F
:10164000206375616E646F206163616265732E0053
:10165000497220616C206F726967656E00436F6E1E
:1016600074696E75616E2E20696D7072657369ADF7
:101670006E0043616C656E74616E646F2050494EFC
:1016800044410043616C696272616369AD6E204FD1
:101690004B0043616C696272616E646F205A004254
:1016A000617365207072657061726164610043618D
:1016B0006C656E74616E646F204261736500436196
:1016C0006C656E74616E646F206163616261646FEA
:1016D0002E0043616C656E74616E646F2E2E2E0059
:1016E000556C74696D6120696D7072657369AD6E5A
:1016F0000046616C6C6F73204D4D550043617267FD
:1017000061204D4D552066616C6C610046616C6CCA
:101710006F20726564204D4D550043616D62696FA5
:1017200073206D6174657269616C657300C06C745F
:10173000696D6F7320696D702E2066616C6C6F73BC
:101740000046616C6C6F7320746F74616C6573001C
:1017500046696C2E206163616261646F0054656D3F
:1017600070657261747572617300496E666F207383
:10177000656E736F7200496E666F2E2064656C2013
:101780006578747275736F7200446574616C6C6512
:10179000732063616C2E2058595A004469722E20C0
:1017A000495020696D707265736F72613A006465AB
:1017B00073636F6E6F6369646F004D4D5520636F87
:1017C0006E65637461646F0046656368613A0070BA
:1017D000617261206465736361726761722066691A
:1017E0006C2E0070617261206361726761722065A6
:1017F0006C2066696C2E0050756C736120656C20DE
:101800006469616C0050726563616C656E742E2052
:10181000636F727461720050726563616C656E749F
:101820002E20657870756C7361720050726563610B
:101830006C656E742E2064657363617267617200FB
:1018400050726563616C656E742E206361726761AE
:101850007200456E66726961720053652065787426
:10186000727579652066696C616D656E746F20793B
:1018700020636F6E20656C20636F6C6F7220636FE6
:1018800072726563746F3F00457870756C73617236
:10189000004C61206361726761206175746F6D8AAD
:1018A00074696361206573748A2061637469766109
:1018B00064612C2070756C736520656C20646961AF
:1018C0006C206520696E736572746520656C206696
:1018D000696C616D656E746F2E2E2E0046696C61A9
:1018E0006D656E746F20746F74616C005469656D02
:1018F000706F20746F74616C20696D702E00466982
:101900006C616D656E746F20757361646F005469EE
:10191000656D706F20646520696D702E0050726572
:1019200063616C656E74617220626F7175696C6C55
:101930006100446973742E20656E205920646573BC
:101940006465206D696E00497A71756965726461BC
:10195000004465726563686100446573762E206D8E
:10196000656469646100446573762E206C696765FF
:10197000726100446573762E20736576657261002E
:101980005B303B305D2070756E746F206F666673E0
:10199000657400416A75737461722D5A00547261E6
:1019A00073657261205BE46D5D0046726F6E7461F9
:1019B0006C205BE46D5D0044657265636861205B6B
:1019C000E46D5D00497A71756965726461205BE45C
:1019D0006D5D0045737461626C656365722074654A
:1019E0006D702E3A00436172726F73205A20697ACB
:1019F000712E2F6465722E206573748A6E20617259
:101A000072696261206D8A78696D6F3F0043616C15
:101A1000696272616E646F2058595A2E204769724C
:101A20006120656C206469616C2070617261207353
:101A30007562697220656C206578747275736F7257
:101A400020686173746120746F636172206C6F73BE
:101A500020746F706573207375706572696F72653D
:101A6000732E2044657370759A732068617A2063C1
:101A70006C69632E0043616C696272616E646F20F1
:101A80005A2E204769726120656C206469616C2060
:101A90007061726120737562697220656C2065786F
:101AA000747275736F7220686173746120746F63F0
:101AB0006172206C6F7320746F7065732073757022
:101AC0006572696F7265732E2044657370759A73C1
:101AD0002068617A20636C69632E0046616C6C6FCC
:101AE000206465206C612063616C69627261636966
:101AF000AD6E2064652050494E4441004C61206326
:101B0000616C696272616369AD6E2050494E4441F7
:101B1000206573748A2066696E616C697A6164619C
:101B20002079206163746976612E20536520707579
:101B300065646520646573616374697661722065AC
:101B40006E20656C206D656E7520436F6E666967EB
:101B50007572616369AD6E202D3E2043616C2E204D
:101B600050494E4441004578747275736F72004D50
:101B70006F766572205A004D6F7665722059004D60
:101B80006F7665722058004C8A6D696E6120252E33
:101B900037730A5A206F66667365743A20252B31B5
:101BA0002E33666D6D0A2563436F6E74696E7561C1
:101BB000720A256352657365740043617267612020
:101BC0007072696D65726F20656C2066696C616DFD
:101BD000656E746F2E0043616E63656C61720045C3
:101BE0006A65637574617220656C204173697374F2
:101BF000656E746520626F7272617261206C6F73C2
:101C00002076616C6F7265732064652063616C6916
:101C10006272616369AD6E2061637475616C657336
:101C2000207920636F6D656E7A61728A2064652009
:101C30006E7565766F2E0050726563616C656E74AB
:101C40002E20626F7175696C6C612E204573706512
:101C5000726120706F72206661766F722E00436F22
:101C60006C6F636120656C2066696C616D656E7474
:101C70006F20656E20656C206578747275736F7265
:101C80002C206C7565676F2070726573696F6E616B
:101C900020656C206469616C2070617261206361F1
:101CA000726761726C6F2E00436F6C6F63612065A9
:101CB0006C2066696C616D656E746F20656E206561
:101CC0006C207072696D6572207475626F20646536
:101CD000206C61204D4D552C206C7565676F207010
:101CE000726573696F6E6120656C206469616C2038
:101CF00070617261206361726761726C6F2E004C5B
:101D00006120696D707265736F726120636F6D65BC
:101D10006E7A61728A206120696D7072696D697274
:101D200020756E61206C696E656120656E207A6930
:101D3000672D7A61672E204769726120656C206487
:101D400069616C20686173746120717565206C61D4
:101D5000206C696E656120616C63616E6365206CE7
:101D60006120616C74757261206F7074696D612E91
:101D7000204D697261206C617320666F746F7320EF
:101D800064656C206D616E75616C202843617069BB
:101D900074756C6F2064652063616C696272616345
:101DA00069AD6E292E0053656C656363696F6E6162
:101DB000206C612074656D7065726174757261204C
:101DC00061646563756164612061207475206D6173
:101DD00074657269616C2E004573636F6765207569
:101DE0006E2066696C616D656E746F2070617261E2
:101DF000206C612043616C696272616369AD6E2021
:101E00006465206C61205072696D65726120436168
:101E1000706120792073656C65636369AD6E616C78
:101E20006F20656E20656C206D656E7520656E2077
:101E300070616E74616C6C612E00566F7920612048
:101E400063616C6962726172206C61206469737491
:101E5000616E63696120656E747265206C612070CB
:101E6000756E7461206465206C6120626F717569A4
:101E70006C6C612079206C61207375706572666985
:101E8000636965206465206C6120626173652E0062
:101E90005365207265636F6D69656E64612063616F
:101EA0006C6962726172205A2E20456A656375748E
:101EB00061726C6F2061686F72613F005265746976
:101EC0007261206C61206C616D2E206465206163FD
:101ED00065726F206465206C6120626173652E00FD
:101EE0004573748A206C61206C8A6D696E61207301
:101EF0006F627265206C6120626173653F004C65A2
:101F00006520656C206D616E75616C20792072654D
:101F10007375656C766520656C2070726F626C6598
:101F20006D612E2044657370759A732C20726569FB
:101F30006E69636961206C6120696D707265736F91
:101F40007261207920636F6E74696E756120636FB2
:101F50006E20656C204173697374656E74652E0024
:101F60005465726D696E61646F2E2046656C69639D
:101F7000657320696D70726573696F6E657321009A
:101F80005369656D70726520707565646573206155
:101F900063636564657220616C2061736973746545
:101FA0006E74652064657364652043616C69627258
:101FB000616369AD6E202D3E204173697374656E57
:101FC0007465005369207469656E657320706C6177
:101FD0006E6368617320646520616365726F206160
:101FE000646963696F6E616C65732C2063616C69F1
:101FF0006272612073757320616A757374657320F2
:10200000656E20416A7573746573202D20416A7571
:1020100073746573204857202D20506C616E63687F
:10202000617320616365726F2E004C696D70696128
:10203000206C6120737570657266696369652064E0
:1020400065206C6120626173652C2079206C756558
:10205000676F2070726573696F6E6120656C2064B4
:1020600069616C2E005175696572657320726570C7
:102070006574697220656C20C06C74696D6F207026
:1020800061736F20706172612072652D20616A75C5
:1020900073746172206C612064697374616E63692A
:1020A0006120626F7175696C6C612D626173653F4F
:1020B0000053656C656363696F6E61206C612074A9
:1020C000656D7065726174757261207061726120F6
:1020D00070726563616C656E746172206C61206200
:1020E0006F7175696C6C6120717565207365206115
:1020F0006A757374652061207475206D61746572F2
:1021000069616C2E004573746120656C2066696C92
:10211000616D656E746F206361726761646F3F000B
:1021200041686F72612070726563616C656E746185
:10213000729A206C6120626F7175696C6C6120709D
:1021400061726120504C412E00566F7920612068E9
:10215000616365722043616C696272616369AD6E2F
:10216000205A2061686F72612E0041686F72612091
:10217000726574697261206C61207072756562614C
:10218000206465206C61206C8A6D696E61206465D5
:1021900020616365726F2E00526574697261206CF4
:1021A0006F7320736F706F72746573206465206540
:1021B0006E76A26F207072696D65726F2E00486135
:1021C000729A206C612063616C696272616369ADAF
:1021D0006E2058595A2E20507565646520746172BE
:1021E000646172206861737461203234206D696E9D
:1021F0002E005072696D65726F2C206861726520C7
:10220000656C2053656C66746573742070617261CF
:1022100020636F6D70726F626172206C6F732070DB
:10222000726F626C656D6173206465206D6F6E7492
:10223000616A65206D8A7320636F6D756E65732E9C
:1022400000486F6C612C20736F7920747520696D64
:10225000707265736F7261204F726967696E616C2D
:102260002050727573612069332E20517569657233
:10227000657320717565207465206775A26520619E
:1022800020747261766573206465206C6120636FD1
:102290006E6669677572616369AD6E3F00486F6C09
:1022A000612C20736F7920747520696D707265736D
:1022B0006F7261204F726967696E616C2050727530
:1022C00073612069332E2054652067756961729AA5
:1022D00020612074726176657320646520756E20BC
:1022E00062726576652070726F6365736F206465D6
:1022F00020636F6E6669677572616369AD6E2C20CD
:10230000656E20656C207175652073652063616C56
:1023100069627261728A20656C20656A65205A2E36
:102320002044657370759A732C2065737461728A8A
:1023300073206C6973746F207061726120696D70B5
:1023400072696D69722E0050617573610046532089
:1023500061636369AD6E004175746F636172672E6E
:1023600066696C2E0046696E2066696C2E004375A6
:102370006368696C6C6F0056656C6F636964616457
:102380002056656E74004261736500436F6D707214
:102390006F622E76656E74004D6F64656C6F0042DF
:1023A0006F7175696C6C6100456D70756A6120684C
:1023B00061737461204653656E736F72004D6F7662
:1023C00069656E646F2073656C6563746F7200522B
:1023D0006574726165722064656C2046494E4441A3
:1023E00000457870756C73616E646F2066696C610E
:1023F0006D656E746F004170617263616E646F2011
:1024000073656C6563746F720053656C6563746F9C
:102410007220766F6C7669656E646F005265616CD0
:10242000697A616E646F20636F72746500456D70C8
:10243000756A616E646F2066696C616D656E746F3C
:1024400000507265706172616E646F2063756368BD
:10245000696C6C6100456C696769656E646F2068C2
:102460007565636F2066696C2E00446573636172E5
:1024700067616E646F2066696C2E0045525220467B
:10248000616C6C6F20544D43004552522041797568
:1024900064612066696C616D656E746F00455252AF
:1024A00020496E7465726E6F0045525220457370FC
:1024B000657261207573756172696F005465726D24
:1024C0002E206D6F76696D69656E746F7300457649
:1024D000697461206D6F7264657200416C696D652D
:1024E0006E742E2061206C6120626F712E00416C31
:1024F000696D656E742E20616C20657874727573D9
:102500006F7200416C696D656E74612068617374EF
:10251000612046494E444100446573636172672EF1
:1025200020686173746120706F6C6561004465732D
:10253000636172672E2068617374612046494E445E
:102540004100536F6C74616E646F2074656E736FBD
:102550007200456E67616E6368616E646F207465BA
:102560006E736F72004552524F5220444553434F91
:102570004E4F4349444F0043414D42494F2044454B
:102580002046494C414D454E544F0046494C414D23
:10259000454E544F20455850554C5341444F0044EC
:1025A00045534341524741204D414E55414C004512
:1025B00052524F5220454A4543554349AE4E20465C
:1025C00057004143542E204657204D4D5520505220
:1025D000454349534100434F4C41204C4C454E41EB
:1025E00000484552522E20494E56414C4944410024
:1025F00046494C2E205941204341524741444F0007
:102600004552524F5220434F4D554E494341434945
:10261000AE4E004D4D55204E4F20524553504F4E1B
:102620004445004D4D552053454C46544553542088
:1026300046414C4C4F00434F52544F204452495650
:10264000455220544D43004552524F52205342525E
:10265000564F4C54414A4520544D43005245534532
:10266000542044524956455220544D43004552523D
:102670004F522044524956455220544D4300455232
:10268000524F5220534F42524543414C20544D43E8
:1026900000415649534F20544D432044454D2E2070
:1026A00043414C4F520054454E534F523A204552ED
:1026B000524F52204D4F562E0054454E534F523AD2
:1026C000204552524F5220484F4D450053454C45EE
:1026D00043542E2053494E204D4F564552534500EA
:1026E00053454C4543542E2053494E20484F4D45A9
:1026F0000046414C4C2E204341524741522041203C
:10270000455854522E00494E5350454343494F4E6D
:1027100041522046494E4441004653454E534F5284
:10272000204D55592050524F4E544F00504F4C455C
:10273000413A204552524F52204D4F562E0046539B
:10274000454E534F522041544153434F2046494C2C
:102750002E004653454E534F52204E4F2053452096
:1027600041435449564F0046494E4441204154414B
:1027700053434F2046494C2E0046494E4441204E7B
:102780004F2053452041435449564F00436F7274C4
:1027900061722066696C616D656E74004578707554
:1027A0006C736172206465204D4D5500496E7472E2
:1027B0006F64756369656E646F2066696C616D2E08
:1027C000004D4D55205265696E74656E746F3A20E8
:1027D00052657374617572616E646F2074656D709B
:1027E000657261747572612E2E2E004F7264656E73
:1027F000616E646F206172636869766F7300416C0B
:1028000067756E6F73206172636869766F73206E8F
:102810006F207365206F7264656E61728A6E2E2000
:102820004D8A78696D6F203130302061726368693C
:10283000766F7320706F72206361727065746120AF
:1028400070617261206F7264656E61722E0050411A
:102850005241444100496E6100416374004F637509
:10286000727269AD20756E206572726F7220696E2A
:10287000657370657261646F2E0043616D62696F8C
:102880002064652066696C616D656E746F204D36DD
:1028900030302E2043617267756520756E20666941
:1028A0006C616D656E746F206E7565766F206F203C
:1028B000657870756C736520656C20616E746572E7
:1028C000696F722E0052657469726520656C2066AE
:1028D000696C616D656E746F20657870756C73617D
:1028E000646F206465206C6120706172746520667D
:1028F000726F6E74616C206465206C61204D4D5563
:102900002E0046696C616D656E746F206465746538
:10291000637461646F20696E657370657261646170
:102920006D656E74652E2041736567C07261746554
:1029300020646520717565206E6F20686179612063
:102940006E696E67C06E2066696C616D656E746FCE
:10295000206361726761646F2E20436F6D707275C2
:10296000656261206C6F732073656E736F7265733F
:10297000207920656C206361626C6561646F2E0054
:102980004572726F7220696E7465726E6F20646535
:1029900020656A6563756369AD6E2E205265696E48
:1029A00069636961206C61204D4D55206F20616322
:1029B0007475616C697A6120656C206669726D77E7
:1029C0006172652E004C61207665727369AD6E2070
:1029D0006465206669726D77617265206465206C3C
:1029E00061204D4D5520657320696E636F6D706178
:1029F0007469626C6520636F6E20656C2046572099
:102A00006465206C6120696D707265736F72612EF0
:102A10002041637475616C697A61722061206C6118
:102A2000207665727369AD6E20332E302E332E0002
:102A30004572726F7220696E7465726E6F20646584
:102A40006C206669726D77617265204D4D552C2042
:102A50007265696E6963696120656C204D4D552E04
:102A600000456C2066696C2E20736F6C6963697415
:102A700061646F206E6F206573748A20646973705F
:102A80006F6E69626C6520656E2065737465206881
:102A9000617264776172652E205265766973612078
:102AA000656C2063AD6469676F2047207061726157
:102AB00020736920656C20A26E646963652064657B
:102AC0002068657272616D69656E746120657374EA
:102AD0008A2066756572612064652072616E676F19
:102AE000202854302D5434292E004E6F2073652039
:102AF0007075656465207265616C697A6172206CBD
:102B0000612061636369AD6E2C2066696C616D65DF
:102B10006E746F207961206361726761646F2E202B
:102B20005072696D65726F2064657363617267616D
:102B30002E004D4D55206E6F20726573706F6E6460
:102B40006520636F7272656374616D656E74652E66
:102B500020526576697361206C6F73206361626CCB
:102B60006573207920636F6E6563746F7265732E71
:102B7000004C61204D4D55206E6F20726573706F53
:102B80006E64652E20526576697361206C6F7320C8
:102B90006361626C6573207920636F6E6563746F27
:102BA0007265732E004D8A7320646574616C6C6568
:102BB00073206F6E6C696E652E00456C2074656EB7
:102BC000736F72206E6F20686163657220686F6D2D
:102BD0006520636F7272656374616D656E74652ED6
:102BE00020436F6D70727565626120736920686142
:102BF0007920616C676F2071756520626C6F7175EB
:102C00006561207375206D6F76696D69656E746F8F
:102C10002E004E6F207365207075656465206D6FA2
:102C20007665722053656C6563746F72206F2054F3
:102C3000656E736F722E00456C2073656C656374EE
:102C40006F72206E6F20686163657220686F6D65BA
:102C500020636F7272656374616D656E74652E209A
:102C6000436F6D7072756562612073692068617968
:102C700020616C676F2071756520626C6F7175657E
:102C800061207375206D6F76696D69656E746F2E46
:102C9000004572726F7220616C20636172676172AD
:102CA00020656E206C61206578747275736F722E6A
:102CB00020496E7370656363696F6E61206C61207B
:102CC000666F726D61206465206C612070756E7432
:102CD000612064656C2066696C616D656E746F2E31
:102CE00020526566696E61206C612063616C696267
:102CF00072616369AD6E2064656C2073656E736F7D
:102D0000722C207369206573206E65636573617230
:102D1000696F2E00456C2073656C6563746F72205B
:102D20006E6F207365207075656465206D6F7665C4
:102D3000722064656269646F206120717565204648
:102D4000494E4441206465746563746120756E204A
:102D500066696C616D656E746F2E2041736567C026
:102D60007261746520646520717565206E6F2068DE
:102D70006179612066696C2E20656E20656C207318
:102D8000656C6563746F72207920717565204649A2
:102D90004E44412066756E63696F6E6520636F7285
:102DA00072656374616D656E74652E00456C207389
:102DB000656E736F722064652066696C616D656E07
:102DC000746F207365206163746976AD2064656DEE
:102DD00061736961646F2070726F6E746F20616CD3
:102DE0002063617267617220656C2065787472750A
:102DF000736F722E20436F6D707275656261207102
:102E00007565206E6F2068612D7961206E61646147
:102E100020617461736361646F20656E20656C204E
:102E20007475626F206465207465666CAD6E207980
:102E30002071756520656C2073656E736F722076E6
:102E400061206F6B2E00456C206D6F746F72206473
:102E500065206C6120706F6C65612073652068610E
:102E60002070617261646F2E2041736567C072616A
:102E7000746520646520717565206C6120706F6CCD
:102E80006561207075656465206D6F766572736528
:102E9000207920636F6D70727565626120656C20AA
:102EA0006361626C6561646F2E00456C2073656EB2
:102EB000736F722064652066696C616D656E746FF6
:102EC000206E6F2073652061706167AD206D69654C
:102ED0006E747261732073652064657363617267D9
:102EE00061626120656C2066696C616D656E746FEE
:102EF0002E2041736567C07261746520646520711E
:102F0000756520656C2066696C616D656E746F20F7
:102F10007075656465206D6F7665727365207920C4
:102F2000656C2073656E736F722066756E63696F72
:102F30006E612E00456C2073656E736F7220646540
:102F40002066696C616D656E746F206E6F207365AD
:102F5000206163746976AD20616C20636172676182
:102F60007220656C2066696C616D656E746F2E20D1
:102F700041736567C0726174652064652071756511
:102F800020656C2066696C616D656E746F206C6C79
:102F90006567AD20616C2073656E736F7220792058
:102FA000717565209A7374652066756E63696F6EBE
:102FB000612E0046494E4441206E6F2073652061AA
:102FC000706167AD206D69656E74726173206465B0
:102FD000736361726761626120656C2066696C6110
:102FE0006D656E746F2E20496E74656E7461206419
:102FF0006573636172676172206D616E75616C6D7E
:10300000656E74652E20436F6D2D2070727565623C
:10301000612071756520656C2066696C2D20616D7D
:10302000656E746F207075656465206D6F7665726E
:10303000736520792046494E44412066756E636968
:103040006F6E612E0046494E4441206E6F207365BD
:10305000206163746976AD20616C20636172676181
:103060007220656C2066696C616D656E746F2E20D0
:1030700041736567C0726174652064652071756510
:1030800020656C2066696C616D656E746F2070756B
:10309000656465206D6F7665727365207920464999
:1030A0004E44412066756E63696F6E612E00446503
:1030B000736163742E0050617261720043617267C4
:1030C000617200446573632E005265696E742E0050
:1030D00046616C6CAD206C61206E6976656C6163D5
:1030E00069AD6E2E2053656E736F72206E6F206611
:1030F000756E63696F6E612E20526573746F7320F5
:10310000656E20626F7175696C6C613F20457370EC
:103110006572616E646F2072657365742E0053650D
:103120006E736962696C696461640000000000008C
:10313000000000000000000000000000000000008F
:10314000000000000000000000000000000000007F
:10315000000000000000000000000000000000006F
:10316000000000000000000000000000000000005F
:103600000000536F6D652070726F626C656D206590
:103610006E636F756E74657265642C205A2D6C65CF
:1036200076656C696E6720656E666F72636564208F
:103630002E2E2E0001004D65736820626564206C9B
:103640006576656C696E67206661696C65642E20BD
:103650005072696E742063616E63656C65642E00E0
:10366000020048656174696E672064697361626C09
:103670006564206279207361666574792074696D70
:1036800065722E000300472D636F646520736C69BB
:1036900063656420666F7220612064696666657286
:1036A000656E74206C6576656C2E000400472D6392
:1036B0006F646520736C6963656420666F72206156
:1036C00020646966666572656E74206C6576656CEB
:1036D0002E20506C656173652072652D736C696373
:1036E0006520746865206D6F64656C206167616931
:1036F0006E2E000500472D636F646520736C69634F
:10370000656420666F722061206E65776572206641
:1037100069726D776172652E000600472D636F64D4
:103720006520736C6963656420666F722061206E2A
:1037300065776572206669726D776172652E2050BB
:103740006C6561736520757064617465207468656B
:10375000206669726D776172652E000700472D63E0
:103760006F646520736C6963656420666F722061A5
:1037700020646966666572656E74207072696E7425
:10378000657220747970652E000800472D636F64A0
:103790006520736C6963656420666F7220612064C4
:1037A0006966666572656E74207072696E746572A2
:1037B00020747970652E20506C6561736520726588
:1037C0002D736C69636520746865206D6F64656C2A
:1037D00020616761696E2E00090050726573732065
:1037E000746865206B6E6F6220746F2070726568FC
:1037F000656174206E6F7A7A6C6520616E642063F7
:103800006F6E74696E75652E000A00506C65617389
:103810006520707265737320746865206B6E6F62CB
:1038200020746F20756E6C6F61642066696C616DC9
:10383000656E74000B00616E642070726573732096
:10384000746865206B6E6F62000C00496E73657260
:10385000742066696C616D656E74000D00436F6C59
:103860006F72206E6F7420636F7272656374000EE6
:103870000046696C616D656E74206E6F74206C6FAC
:1038800061646564000F004368616E67656420636E
:103890006F72726563746C790010004C6F616469BB
:1038A0006E6720636F6C6F720011004368616E6712
:1038B00065207375636365737321001200506C6536
:1038C000617365206F70656E2069646C657220613C
:1038D0006E642072656D6F76652066696C616D65DA
:1038E0006E74206D616E75616C6C792E00130057DB
:1038F00061732066696C616D656E7420756E6C6FA6
:103900006164207375636365737366756C3F00143F
:1039100000506C6561736520757067726164652E17
:103920000015004E6577206669726D7761726520BB
:1039300076657273696F6E20617661696C61626C25
:10394000653A00160057616974696E6720666F7288
:103950002050494E44412070726F626520636F6F42
:103960006C696E67001700506C6561736520776144
:1039700069740018004E6F206D6F76652E00190077
:103980005761697420666F7220757365722E2E2ED2
:10399000001A00537461626C6520616D6269656E26
:1039A000742074656D706572617475726520323152
:1039B0002D323643206973206E656564656420612D
:1039C000207269676964207374616E642069732072
:1039D00072657175697265642E001B00506C6561BB
:1039E00073652072756E2058595A2063616C696244
:1039F000726174696F6E2066697273742E001C00A8
:103A0000506C6561736520756E6C6F6164207468BD
:103A1000652066696C616D656E7420666972737489
:103A20002C207468656E20726570656174207468FE
:103A3000697320616374696F6E2E001D00436865B1
:103A4000636B73001E004E6F7A7A6C6520642E00E3
:103A50001F00416C706861626574002000536F72D2
:103A60007400210054696D650022004E6F726D6113
:103A70006C0023005344206361726400240053658A
:103A80006C656374206C616E677561676500250005
:103A90004E6F7A7A6C65206368616E6765002600F8
:103AA00048572053657475700027004C6F61646936
:103AB0006E67205465737400280044697361626CFA
:103AC000652073746570706572730029004D6F76A0
:103AD000652061786973002A0054656D70657261B4
:103AE00074757265002B0050494E44412063616C2F
:103AF0002E002C0052657365742058595A2063615A
:103B00006C6962722E002D0053686F7720656E64B9
:103B10002073746F7073002E005049442063616CF1
:103B20006962726174696F6E002F00426564206C77
:103B30006576656C20636F72726563740030004D4A
:103B400065736820426564204C6576656C696E67B4
:103B500000310043616C696272617465205A003201
:103B60000043616C6962726174652058595A003370
:103B70000053656C667465737400340057697A612C
:103B8000726400350054657374696E672066696CF1
:103B9000616D656E740036004C6F616420416C6C21
:103BA000003700506C656173652070756C6C206F18
:103BB00075742066696C616D656E7420696D6D65E4
:103BC00064696174656C79003800526573657400CE
:103BD000390052656E616D65003A00466972737412
:103BE000206C617965722063616C2E003B00536527
:103BF0006C656374003C00537465656C2073686584
:103C0000657473003D00537570706F7274003E00F0
:103C10004661696C207374617473204D4D55003F8B
:103C2000004661696C2073746174730040005374C2
:103C3000617469737469637300410043616C696204
:103C4000726174696F6E0042004175746F4C6F61F0
:103C5000642066696C616D656E740043004C6F6131
:103C6000642066696C616D656E74004400556E6C0D
:103C70006F61642066696C616D656E740045004C0F
:103C80006F616420746F206E6F7A7A6C65004600F5
:103C90005072656C6F616420746F204D4D55004704
:103CA000004E6F20534420636172640048005072DC
:103CB000696E742066726F6D20534400490052652E
:103CC00073756D65207072696E74004A005061757D
:103CD0007365207072696E74004B005365742052D6
:103CE00065616479004C00536574206E6F742052D6
:103CF00065616479004D0050726568656174004EBD
:103D00000054756E65004F004C6976652061646AE9
:103D1000757374205A00500052657072696E740099
:103D20005100496E666F2073637265656E005200C4
:103D30004173736973740053004F6E6365005400E0
:103D4000536F756E640055004C6F756400560046E5
:103D5000696C2E2073656E736F7200570043686143
:103D60006E67652066696C616D656E74005800460B
:103D70006C6F770059005370656564005A004D619F
:103D8000676E65747320636F6D702E005B004E2F3D
:103D900041005C005A2D70726F6265206E722E00B9
:103DA0005D004D657368005E0053657474696E67ED
:103DB00073005F005965730060004E6F006100532F
:103DC000746F70207072696E74006200436865637E
:103DD0006B696E672066696C6500630046696C6597
:103DE00020696E636F6D706C6574652E006400846D
:103DF000526566726573680065004D61696E0066A4
:103E00000057616974696E6720666F72206E6F7A01
:103E10007A6C6520616E642062656420636F6F6CEC
:103E2000696E6700670053656C6563742066696C32
:103E3000616D656E743A00680053656C66746573F5
:103E400074204F4B00690053656C66746573742071
:103E50007374617274006A005377617070656400F6
:103E60006B0046726F6E742F6C6566742066616EAF
:103E700073006C0041786973006D004178697320AC
:103E80006C656E677468006E004C6F6F73652070B0
:103E9000756C6C6579006F00456E6473746F70208B
:103EA0006E6F7420686974007000456E6473746F7F
:103EB000700071004D6F746F72007200456E647314
:103EC000746F7073007300576972696E6720657252
:103ED000726F720074004265642F48656174657288
:103EE0000075004E6F7420636F6E6E656374656459
:103EF0000076004865617465722F546865726D695B
:103F000073746F72007700506C656173652063682D
:103F100065636B3A00780053656C66746573742052
:103F20006572726F722100790046696C616D656E11
:103F3000742073656E736F72007A005072696E74CC
:103F40002066616E3A007B00486F74656E6420667F
:103F5000616E3A007C0043616C6962726174696EE3
:103F60006720686F6D65007D0053656C66746573CE
:103F700074206661696C6564007E00416C6C20632E
:103F80006F7272656374007F00436865636B696E6E
:103F9000672073656E736F7273008000436865639A
:103FA0006B696E6720686F74656E6400810043689A
:103FB00065636B696E6720626564008200436865B3
:103FC000636B696E67205A206178697300830043D0
:103FD0006865636B696E6720592061786973008436
:103FE00000436865636B696E672058206178697368
:103FF000008500436865636B696E6720656E647356
:10400000746F7073008600436172642072656D6F17
:104010007665640087004261636B008800417574B7
:104020006F20706F77657200890053696C656E74DC
:10403000008A004D6F6465008B00486967682070D6
:104040006F776572008C00537472696374008D0021
:104050005761726E008E004E6F6E65008F00486F64
:1040600074656E64206174203238304321204E6FB5
:104070007A7A6C65206368616E67656420616E643E
:10408000207469676874656E656420746F2073704E
:104090006563733F009000466F722061204E6F7A17
:1040A0007A6C65206368616E676520706C6561730A
:1040B0006520726561640A70727573612E696F2F75
:1040C0006E6F7A7A6C652D6D6B3373009100504979
:1040D000442063616C2E2066696E697368656400B4
:1040E00092005049442063616C2E00930050726925
:1040F0006E74207061757365640094005072696E0F
:10410000742061626F72746564009500436F70790A
:104110002073656C6563746564206C616E6775619E
:1041200067653F0096004E6F7A7A6C65206469611E
:104130006D65746572206469666665727320667267
:104140006F6D2074686520472D636F64652E00973E
:10415000004E6F7A7A6C65206469616D6574657272
:1041600020646966666572732066726F6D2074687C
:104170006520472D636F64652E20506C6561736503
:1041800020636865636B207468652076616C756573
:1041900020696E2073657474696E67732E009800D1
:1041A0005468657265206973206E6F2066696C6162
:1041B0006D656E74206C6F616465642E00990054A7
:1041C00068657265206973207374696C6C20612066
:1041D0006E65656420746F206D616B65205A206385
:1041E000616C6962726174696F6E2E20506C6561DA
:1041F000736520666F6C6C6F7720746865206D61E5
:104200006E75616C2C2063686170746572204669FC
:104210007273742073746570732C20736563746992
:104220006F6E2043616C6962726174696F6E2066A3
:104230006C6F772E009A005072696E7465722068F8
:104240006173206E6F74206265656E2063616C69B6
:10425000627261746564207965742E20506C6561AA
:10426000736520666F6C6C6F7720746865206D6174
:104270006E75616C2C20636861707465722046698C
:104280007273742073746570732C20736563746922
:104290006F6E2043616C6962726174696F6E206633
:1042A0006C6F772E009B0053656C66746573742089
:1042B00077696C6C2062652072756E20746F206364
:1042C000616C6962726174652061636375726174A7
:1042D000652073656E736F726C65737320726568A9
:1042E0006F6D696E672E009C004F6C64207365745F
:1042F00074696E677320666F756E642E2044656600
:1043000061756C74205049442C204573746570733A
:10431000206574632E2077696C6C2062652073655C
:10432000742E009D005761726E696E673A20626F4D
:104330007468207072696E7465722074797065207B
:10434000616E64206D6F74686572626F6172642063
:1043500074797065206368616E6765642E009E00E5
:104360005761726E696E673A207072696E74657219
:104370002074797065206368616E6765642E009FA4
:10438000005761726E696E673A206D6F746865726E
:10439000626F6172642074797065206368616E6712
:1043A00065642E00A000536865657400A1004E6F1F
:1043B00074207370696E6E696E6700A20053706935
:1043C0006E6E696E6700A3004C65667420686F743A
:1043D000656E642066616E3F00A40046726F6E7465
:1043E000207072696E742066616E3F00A5004661A0
:1043F0006E207465737400A60058595A2063616C6E
:104400006962726174696F6E20616C6C2072696799
:1044100068742E20536B65772077696C6C20626519
:1044200020636F72726563746564206175746F6D6B
:1044300061746963616C6C792E00A70058595A2029
:1044400063616C6962726174696F6E20616C6C206B
:1044500072696768742E20582F592061786573201F
:1044600061726520736C696768746C7920736B6521
:104470007765642E20476F6F64206A6F622100A801
:104480000058595A2063616C6962726174696F6E79
:10449000206F6B2E20582F59206178657320617230
:1044A000652070657270656E646963756C61722EEB
:1044B00020436F6E67726174756C6174696F6E739F
:1044C0002100A90058595A2063616C6962726174B5
:1044D000696F6E20636F6D70726F6D697365642EA6
:1044E0002052696768742066726F6E742063616C15
:1044F0006962726174696F6E20706F696E74206E8C
:104500006F7420726561636861626C652E00AA0039
:1045100058595A2063616C6962726174696F6E20C8
:10452000636F6D70726F6D697365642E2046726F74
:104530006E742063616C6962726174696F6E207061
:104540006F696E7473206E6F742072656163686149
:10455000626C652E00AB0058595A2063616C696229
:10456000726174696F6E206661696C65642E205299
:10457000696768742066726F6E742063616C69622B
:10458000726174696F6E20706F696E74206E6F74E3
:1045900020726561636861626C652E00AC005859D9
:1045A0005A2063616C6962726174696F6E20666122
:1045B000696C65642E2046726F6E742063616C694D
:1045C00062726174696F6E20706F696E7473206EB1
:1045D0006F7420726561636861626C652E00AD0066
:1045E00058595A2063616C6962726174696F6E20F8
:1045F0006661696C65642E20506C6561736520632B
:104600006F6E73756C7420746865206D616E756172
:104610006C2E00AE0058595A2063616C6962726159
:1046200074696F6E206661696C65642E20426564F2
:104630002063616C6962726174696F6E20706F696A
:104640006E7420776173206E6F7420666F756E6470
:104650002E00AF00506C6561736520706C616365FE
:1046600020737465656C207368656574206F6E20B7
:10467000686561746265642E00B00044697374619A
:104680006E6365206265747765656E20746970205D
:104690006F6620746865206E6F7A7A6C6520616E33
:1046A0006420746865206265642073757266616356
:1046B0006520686173206E6F74206265656E20737B
:1046C0006574207965742E20506C65617365206671
:1046D0006F6C6C6F7720746865206D616E75616CAE
:1046E0002C2063686170746572204669727374204F
:1046F00073746570732C2073656374696F6E2046E4
:1047000069727374206C617965722063616C69628F
:10471000726174696F6E2E00B100506C6163652028
:1047200061207368656574206F66207061706572C2
:1047300020756E64657220746865206E6F7A7A6C7D
:104740006520647572696E67207468652063616CAA
:104750006962726174696F6E206F66206669727338
:1047600074203420706F696E74732E204966207433
:104770006865206E6F7A7A6C652063617463686522
:1047800073207468652070617065722C20706F777B
:104790006572206F666620746865207072696E7439
:1047A000657220696D6D6564696174656C792E0050
:1047B000B200536561726368696E67206265642048
:1047C00063616C6962726174696F6E20706F696E8B
:1047D0007400B3004D6561737572696E6720726510
:1047E000666572656E636520686569676874206FC9
:1047F000662063616C6962726174696F6E20706FAC
:10480000696E7400B400506C6561736520636C65FB
:10481000616E20746865206E6F7A7A6C6520666FB1
:10482000722063616C6962726174696F6E2E2043DD
:104830006C69636B207768656E20646F6E652E000F
:10484000B5004175746F20686F6D6500B6005265E4
:1048500073756D696E67207072696E7400B7005071
:10486000494E44412048656174696E6700B8004351
:10487000616C6962726174696F6E20646F6E65004D
:10488000B90043616C6962726174696E67205A0095
:10489000BA0042656420646F6E6500BB00426564C7
:1048A0002048656174696E6700BC00486561746981
:1048B0006E6720646F6E652E00BD00486561746987
:1048C0006E6700BE00546F74616C00BF004C617372
:1048D00074207072696E7400C0004D4D5520666181
:1048E000696C7300C1004D4D55206C6F616420668A
:1048F00061696C7300C2004D4D5520706F77657211
:10490000206661696C7300C3004D617465726961F2
:104910006C206368616E67657300C4004C617374DA
:10492000207072696E74206661696C7572657300BF
:10493000C500546F74616C206661696C7572657333
:1049400000C60046696C2E2072756E6F7574730018
:10495000C70054656D70657261747572657300C8C7
:104960000053656E736F7220696E666F00C90045F3
:104970007874727564657220696E666F00CA00583B
:10498000595A2063616C2E2064657461696C7300F0
:10499000CB005072696E7465722049502041646486
:1049A000723A00CC00756E6B6E6F776E00CD004D65
:1049B0004D5520636F6E6E656374656400CE004470
:1049C0006174653A00CF00746F20756E6C6F61641E
:1049D0002066696C616D656E7400D000746F206C28
:1049E0006F61642066696C616D656E7400D1005002
:1049F0007265737320746865206B6E6F6200D200FD
:104A000050726568656174696E6720746F206375A4
:104A10007400D30050726568656174696E672074B4
:104A20006F20656A65637400D400507265686561C3
:104A300074696E6720746F20756E6C6F616400D549
:104A40000050726568656174696E6720746F206CD0
:104A50006F616400D600436F6F6C646F776E00D730
:104A60000046696C616D656E74206578747275645A
:104A7000696E672026207769746820636F7272659B
:104A8000637420636F6C6F723F00D800456A656382
:104A90007400D9004175746F6C6F6164696E672032
:104AA00066696C616D656E742069732061637469F9
:104AB00076652C206A757374207072657373207428
:104AC0006865206B6E6F6220616E6420696E73652D
:104AD00072742066696C616D656E742E2E2E00DA1C
:104AE00000546F74616C2066696C616D656E740052
:104AF000DB00546F74616C207072696E742074698D
:104B00006D6500DC0046696C616D656E74207573BF
:104B1000656400DD005072696E742074696D650013
:104B2000DE005072656865617420746865206E6F80
:104B30007A7A6C652100DF004552524F523A00E00C
:104B400000592064697374616E63652066726F6DCD
:104B5000206D696E00E1004C65667400E2005269E8
:104B600067687400E3004D65617375726564207356
:104B70006B657700E400536C6967687420736B653C
:104B80007700E50053657665726520736B65770085
:104B9000E6005B303B305D20706F696E74206F669D
:104BA0006673657400E70041646A757374696E67C3
:104BB000205A00E800526561722073696465205BC9
:104BC000E46D5D00E90046726F6E74207369646580
:104BD0005BE46D5D00EA0052696768742073696484
:104BE000655BE46D5D00EB004C6566742073696481
:104BF00065205BE46D5D00EC005365742074656DA9
:104C000070657261747572653A00ED0041726520DD
:104C10006C65667420616E64207269676874205ADE
:104C20002D63617272696167657320616C6C2075B8
:104C3000703F00EE0043616C6962726174696E6777
:104C40002058595A2E20526F74617465207468651B
:104C5000206B6E6F6220746F206D6F7665207468B4
:104C600065205A20636172726961676520757020E2
:104C7000746F2074686520656E642073746F707043
:104C80006572732E20436C69636B207768656E20B4
:104C9000646F6E652E00EF0043616C69627261742F
:104CA000696E67205A2E20526F7461746520746893
:104CB00065206B6E6F6220746F206D6F7665207457
:104CC0006865205A2063617272696167652075703A
:104CD00020746F2074686520656E642073746F7033
:104CE000706572732E20436C69636B207768656E04
:104CF00020646F6E652E00F00050494E44412063E1
:104D0000616C6962726174696F6E206661696C655D
:104D10006400F10050494E44412063616C69627245
:104D20006174696F6E2069732066696E6973686566
:104D30006420616E64206163746976652E20497415
:104D40002063616E2062652064697361626C6564D2
:104D500020696E206D656E752053657474696E6789
:104D6000732D3E50494E44412063616C2E00F20089
:104D7000457874727564657200F3004D6F76652036
:104D80005A00F4004D6F7665205900F5004D6F769E
:104D900065205800F600536865657420252E37732A
:104DA0000A5A206F66667365743A20252B312E33BC
:104DB000666D6D0A2563436F6E74696E75650A25AD
:104DC00063526573657400F700506C65617365200C
:104DD0006C6F61642066696C616D656E74206669D4
:104DE0007273742E00F80043616E63656C00F90005
:104DF00052756E6E696E672057697A6172642077AA
:104E0000696C6C2064656C6574652063757272658D
:104E10006E742063616C6962726174696F6E207276
:104E20006573756C747320616E6420737461727441
:104E30002066726F6D2074686520626567696E6EAA
:104E4000696E672E00FA0050726568656174696E5C
:104E500067206E6F7A7A6C652E20506C6561736581
:104E600020776169742E00FB00506C6561736520CA
:104E7000696E736572742066696C616D656E74200D
:104E8000696E746F207468652065787472756465E6
:104E9000722C207468656E2070726573732074685C
:104EA00065206B6E6F6220746F206C6F6164206987
:104EB000742E00FC00506C6561736520696E73652B
:104EC00072742066696C616D656E7420696E746FB2
:104ED0002074686520666972737420747562652039
:104EE0006F6620746865204D4D552C207468656E82
:104EF00020707265737320746865206B6E6F62201A
:104F0000746F206C6F61642069742E00FD0054681A
:104F100065207072696E7465722077696C6C20739D
:104F200074617274207072696E74696E672061209A
:104F30007A69672D7A6167206C696E652E20526FE1
:104F40007461746520746865206B6E6F6220756E85
:104F500074696C20796F752072656163682074686C
:104F600065206F7074696D616C206865696768742D
:104F70002E20436865636B207468652070696374D4
:104F80007572657320696E207468652068616E644F
:104F9000626F6F6B202843616C6962726174696F24
:104FA0006E2063686170746572292E00FE0053657F
:104FB0006C6563742074656D70657261747572657B
:104FC000207768696368206D617463686573207910
:104FD0006F7572206D6174657269616C2E00FF00DF
:104FE00053656C65637420612066696C616D656EE4
:104FF0007420666F7220746865204669727374202D
:105000004C617965722043616C6962726174696F89
:105010006E20616E642073656C6563742069742012
:10502000696E20746865206F6E2D73637265656E9E
:10503000206D656E752E0000014E6F772049207738
:10504000696C6C2063616C6962726174652064696B
:105050007374616E6365206265747765656E207434
:105060006970206F6620746865206E6F7A7A6C654F
:1050700020616E6420686561746265642073757276
:10508000666163652E0001015A2063616C6962727A
:105090006174696F6E207265636F6D6D656E6465B6
:1050A000642E2052756E206974206E6F773F000267
:1050B00001506C656173652072656D6F7665207354
:1050C0007465656C2073686565742066726F6D2009
:1050D000686561746265642E00030149732073740E
:1050E00065656C207368656574206F6E2068656106
:1050F000746265643F000401506C656173652063F0
:105100006865636B206F75722068616E64626F6F93
:105110006B20616E64206669782074686520707207
:105120006F626C656D2E205468656E2072657375B4
:105130006D65207468652057697A617264206279B0
:10514000207265626F6F74696E6720746865207085
:1051500072696E7465722E000501416C6C20697372
:1051600020646F6E652E20486170707920707269BE
:105170006E74696E6721000601596F752063616E58
:1051800020616C7761797320726573756D65207429
:1051900068652057697A6172642066726F6D20437A
:1051A000616C6962726174696F6E202D3E2057696F
:1051B0007A6172642E000701496620796F75206854
:1051C000617665206164646974696F6E616C2073D7
:1051D0007465656C207368656574732C2063616CFD
:1051E00069627261746520746865697220707265A5
:1051F0007365747320696E2053657474696E677388
:10520000202D204857205365747570202D2053742D
:1052100065656C207368656574732E000801506CB9
:105220006561736520636C65616E20686561746299
:10523000656420616E64207468656E2070726573A9
:105240007320746865206B6E6F622E000901446FD5
:1052500020796F752077616E7420746F207265708D
:10526000656174206C617374207374657020746F51
:1052700020726561646A7573742064697374616E09
:105280006365206265747765656E206E6F7A7A6CEF
:105290006520616E6420686561746265643F000A20
:1052A0000153656C656374206E6F7A7A6C6520704B
:1052B0007265686561742074656D7065726174757E
:1052C0007265207768696368206D617463686573CF
:1052D00020796F7572206D6174657269616C2E0042
:1052E0000B0149732066696C616D656E74206C6F8B
:1052F000616465643F000C014E6F77204920776937
:105300006C6C2070726568656174206E6F7A7A6C5F
:105310006520666F7220504C412E000D01492077A8
:10532000696C6C2072756E207A2063616C696272A0
:105330006174696F6E206E6F772E000E014E6F776D
:105340002072656D6F76652074686520746573746E
:10535000207072696E742066726F6D20737465655B
:105360006C2073686565742E000F01506C65617365
:10537000652072656D6F7665207368697070696EFF
:10538000672068656C706572732066697273742E2D
:10539000001001492077696C6C2072756E20787955
:1053A0007A2063616C6962726174696F6E206E6FDE
:1053B000772E2049742077696C6C2074616B6520AE
:1053C000757020746F203234206D696E732E001159
:1053D0000146697273742C20492077696C6C2072C5
:1053E000756E207468652073656C667465737420CF
:1053F000746F20636865636B206D6F737420636FD7
:105400006D6D6F6E20617373656D626C7920707263
:105410006F626C656D732E00120148692C20492063
:10542000616D20796F7572204F726967696E616C6A
:10543000205072757361206933207072696E7465D3
:10544000722E20576F756C6420796F75206C696BB4
:1054500065206D6520746F20677569646520796FBC
:1054600075207468726F756768207468652073654D
:105470007475702070726F636573733F0013014819
:10548000692C204920616D20796F7572204F7269F7
:1054900067696E616C20507275736120693320708A
:1054A00072696E7465722E20492077696C6C206772
:1054B0007569646520796F75207468726F756768A7
:1054C00020612073686F727420736574757020702A
:1054D000726F636573732C20696E207768696368E7
:1054E00020746865205A2D617869732077696C6C27
:1054F0002062652063616C696272617465642E204C
:105500005468656E2C20796F752077696C6C206209
:105510006520726561647920746F207072696E74A1
:105520002E0014015061757365001501465320412A
:105530006374696F6E001601436F6E742E0017015D
:10554000462E206175746F6C6F6164001801462EE1
:105550002072756E6F7574001901437574746572ED
:10556000001A0146616E207370656564001B01427C
:105570006564001C0146616E7320636865636B009F
:105580001D014D6F64656C001E014E6F7A7A6C656B
:10559000001F0146656564696E6720746F2046537D
:1055A000656E736F720020014D6F76696E672073B0
:1055B000656C6563746F72002101486F6D696E6779
:1055C000002201526574726163742066726F6D20EF
:1055D00046494E4441002301456A656374696E671C
:1055E0002066696C616D656E740024015061726B98
:1055F000696E672073656C6563746F720025015274
:10560000657475726E696E672073656C6563746F1F
:1056100072002601506572666F726D696E67206355
:10562000757400270150757368696E672066696C30
:10563000616D656E74002801507265706172696EEB
:105640006720626C61646500290153656C65637451
:10565000696E672066696C2E20736C6F74002A0176
:10566000556E6C6F6164696E672066696C616D650B
:105670006E74002B0145525220544D4320666169DF
:105680006C6564002C014552522048656C702066A0
:10569000696C616D656E74002D0145525220496E32
:1056A0007465726E616C002E01455252205761691B
:1056B0007420666F722055736572002F0146696E03
:1056C000697368696E67206D6F76656D656E74735A
:1056D00000300141766F6964696E67206772696E98
:1056E0006400310146656564696E6720746F206EE1
:1056F0006F7A7A6C6500320146656564696E672071
:10570000746F206578747275646572003301466544
:105710006564696E6720746F2046494E44410034C9
:1057200001556E6C6F6164696E6720746F207075CF
:105730006C6C6579003501556E6C6F6164696E67DC
:1057400020746F2046494E44410036014469736518
:105750006E676167696E672069646C657200370106
:10576000456E676167696E672069646C65720038B1
:10577000014F4B003901554E4B4E4F574E2045526D
:10578000524F52003A0146494C414D454E54204338
:1057900048414E4745003B0146494C414D454E541A
:1057A00020454A4543544544003C01554E4C4F4129
:1057B00044204D414E55414C4C59003D0146572027
:1057C00052554E54494D45204552524F52003E01CC
:1057D0004D4D5520465720555044415445204E4587
:1057E00045444544003F0151554555452046554CDB
:1057F0004C004001494E56414C494420544F4F4CB7
:1058000000410146494C2E20414C5245414459200B
:105810004C4F41444544004201434F4D4D554E4984
:10582000434154494F4E204552524F520043014D7F
:105830004D55204E4F5420524553504F4E44494EE3
:10584000470044014D4D55204D4355204552524F80
:10585000520045014D4D552053454C465445535437
:10586000204641494C4544004601544D4320445292
:10587000495645522053484F52544544004701541D
:105880004D4320554E444552564F4C5441474520B8
:10589000455252004801544D432044524956455206
:1058A000205245534554004901544D432044524928
:1058B000564552204552524F52004A01544D432002
:1058C0004F56455248454154204552524F52004B85
:1058D000015741524E494E4720544D4320544F4F9B
:1058E00020484F54004C0149444C45522043414EFE
:1058F0004E4F54204D4F5645004D0149444C4552A2
:105900002043414E4E4F5420484F4D45004E0153C9
:10591000454C4543544F522043414E4E4F54204D29
:105920004F5645004F0153454C4543544F52204379
:10593000414E4E4F5420484F4D450050014C4F4171
:105940004420544F20455854522E204641494C453E
:1059500044005101494E53504543542046494E445A
:10596000410052014653454E534F5220544F4F2051
:105970004541524C5900530150554C4C4559204318
:10598000414E4E4F54204D4F56450054014653450D
:105990004E534F522046494C2E20535455434B00F2
:1059A00055014653454E534F52204449444E5420CE
:1059B00054524947472E00560146494E444120461D
:1059C000494C414D2E20535455434B0057014649F5
:1059D0004E4441204449444E54205452494747457F
:1059E000520058014375742066696C616D656E7470
:1059F000005901456A6563742066726F6D204D4DD4
:105A000055005A014C6F6164696E672066696C616C
:105A10006D656E74005B014D4D5520526574727951
:105A20003A20526573746F72696E672074656D7089
:105A3000657261747572652E2E2E005C01536F7253
:105A400074696E672066696C6573005D01536F6DE4
:105A5000652066696C65732077696C6C206E6F7465
:105A600020626520736F727465642E204D61782EFC
:105A7000204E6F2E206F662066696C657320696EFC
:105A8000203120666F6C64657220666F7220736FC0
:105A90007274696E67206973203130302E005E01A8
:105AA00053544F505045442E005F014F66660060CE
:105AB000014F6E006101556E6578706563746564B1
:105AC000206572726F72206F636375727265642EE7
:105AD0000062014D3630302046696C616D656E7430
:105AE000204368616E67652E204C6F6164206120E1
:105AF0006E65772066696C616D656E74206F7220CB
:105B0000656A65637420746865206F6C64206F6ECD
:105B1000652E00630152656D6F766520746865209F
:105B2000656A65637465642066696C616D656E7431
:105B30002066726F6D207468652066726F6E7420C7
:105B40006F6620746865204D4D552E0064014669CE
:105B50006C616D656E742064657465637465642042
:105B6000756E65787065637465646C792E20456E1A
:105B700073757265206E6F2066696C616D656E74F9
:105B8000206973206C6F616465642E2043686563CF
:105B90006B207468652073656E736F727320616E1D
:105BA0006420776972696E672E006501496E7465BD
:105BB000726E616C2072756E74696D6520657272AB
:105BC0006F722E2054727920726573657474696ED9
:105BD0006720746865204D4D55206F722075706484
:105BE0006174696E6720746865206669726D77619B
:105BF00072652E0066014D4D552046572076657220
:105C000073696F6E20697320696E636F6D70617464
:105C100069626C652077697468207072696E74655A
:105C2000722046572E55706461746520746F20761B
:105C3000657273696F6E20332E302E332E0067012C
:105C40004D4D55204669726D7761726520696E749D
:105C500065726E616C206572726F722C20706C655B
:105C600061736520726573657420746865204D4D9D
:105C7000552E006801526571756573746564206600
:105C8000696C616D656E7420746F6F6C2069732030
:105C90006E6F7420617661696C61626C65206F6EF5
:105CA00020746869732068617264776172652E2060
:105CB000436865636B2074686520472D636F646576
:105CC00020666F7220746F6F6C20696E6465782037
:105CD0006F7574206F662072616E6765202854307E
:105CE0002D5434292E00690143616E6E6F7420704B
:105CF0006572666F726D2074686520616374696F88
:105D00006E2C2066696C616D656E7420697320610C
:105D10006C7265616479206C6F616465642E2055D6
:105D20006E6C6F61642069742066697273742E00F2
:105D30006A014D4D55206E6F7420726573706F6EE1
:105D400064696E6720636F72726563746C792E206C
:105D5000436865636B2074686520776972696E6754
:105D600020616E6420636F6E6E6563746F72732E54
:105D7000006B014D4D55206E6F7420726573706F0E
:105D80006E64696E672E20436865636B2074686576
:105D900020776972696E6720616E6420636F6E6E32
:105DA0006563746F72732E006C014D6F72652064B1
:105DB000657461696C73206F6E6C696E652E006D21
:105DC000015468652049646C65722063616E6E6F72
:105DD0007420686F6D652070726F7065726C792EBB
:105DE00020436865636B20666F7220616E7974680A
:105DF000696E6720626C6F636B696E67206974738C
:105E0000206D6F76656D656E742E006E0143616E58
:105E10002774206D6F76652053656C6563746F72AF
:105E2000206F722049646C65722E006F01546865A2
:105E30002053656C6563746F722063616E6E6F745E
:105E400020686F6D652070726F7065726C792E209E
:105E5000436865636B20666F7220616E7974686950
:105E60006E6720626C6F636B696E67206974732064
:105E70006D6F76656D656E742E0070014C6F616498
:105E8000696E6720746F206578747275646572201E
:105E90006661696C65642E20496E73706563742059
:105EA0007468652066696C616D656E7420746970D4
:105EB0002073686170652E20526566696E65207476
:105EC00068652073656E736F722063616C696272BE
:105ED0006174696F6E2C206966206E656564656407
:105EE0002E00710153656C6563746F722063616E7F
:105EF0002774206D6F76652064756520746F204669
:105F0000494E444120646574656374696E6720611D
:105F10002066696C616D656E742E204D616B652025
:105F200073757265206E6F2066696C616D656E7445
:105F300020697320696E2053656C6563746F7220ED
:105F4000616E642046494E444120776F726B732026
:105F500070726F7065726C792E00720146696C61A7
:105F60006D656E742073656E736F722074726967ED
:105F7000676572656420746F6F206561726C79204B
:105F80007768696C65206C6F6164696E6720746FF7
:105F90002065787472756465722E20436865636B42
:105FA0002074686572652069736E277420616E794C
:105FB0007468696E6720737475636B20696E205016
:105FC00054464520747562652E20436865636B20D6
:105FD000746861742073656E736F7220726561649A
:105FE000732070726F7065726C792E00730150753A
:105FF0006C6C6579206D6F746F72207374616C6C5A
:1060000065642E20456E7375726520746865207016
:10601000756C6C65792063616E206D6F76652061AB
:106020006E6420636865636B2074686520776972AD
:10603000696E672E00740146696C616D656E74202F
:1060400073656E736F72206469646E277420737752
:1060500069746368206F6666207768696C6520756F
:106060006E6C6F6164696E672066696C616D656EE8
:10607000742E20456E737572652066696C616D655E
:106080006E742063616E206D6F766520616E642092
:106090007468652073656E736F7220776F726B73AF
:1060A0002E00750146696C616D656E742073656EB6
:1060B000736F72206469646E2774207472696767F5
:1060C0006572207768696C65206C6F6164696E67C2
:1060D000207468652066696C616D656E742E20455C
:1060E0006E73757265207468652073656E736F7268
:1060F0002069732063616C696272617465642061F8
:106100006E64207468652066696C616D656E7420CC
:10611000726561636865642069742E007601464982
:106120004E4441206469646E2774207377697463F8
:1061300068206F6666207768696C6520756E6C6F85
:106140006164696E672066696C616D656E742E208E
:1061500054727920756E6C6F6164696E67206D6131
:106160006E75616C6C792E20456E73757265206654
:10617000696C616D656E742063616E206D6F76650C
:1061800020616E642046494E444120776F726B73E4
:106190002E00770146494E4441206469646E27749D
:1061A0002074726967676572207768696C65206C16
:1061B0006F6164696E67207468652066696C616DE3
:1061C000656E742E20456E73757265207468652047
:1061D00066696C616D656E742063616E206D6F76AB
:1061E0006520616E642046494E444120776F726B92
:1061F000732E00780144697361626C650079015304
:10620000746F70007A014C6F6164007B01556E6C95
:106210006F6164007C0152657365744D4D55007D5E
:10622000015265747279007E01426564206C657666
:10623000656C696E67206661696C65642E205365C4
:106240006E736F72206469646E277420747269675C
:106250006765722E20446562726973206F6E206ECE
:106260006F7A7A6C653F2057616974696E67206642
:106270006F722072657365742E007F0153656E73B3
:1062800069746976697479008001446F6E65006590
:106290006E717565696E67202200446F6E652070AF
:1062A00072696E74696E672066696C65004E6F2056
:1062B0004C696E65204E756D6265722077697468F1
:1062C00020636865636B73756D2C204C617374205B
:1062D0004C696E653A20004E6F20436865636B73AE
:1062E000756D2077697468206C696E65206E756DB8
:1062F0006265722C204C617374204C696E653A2083
:1063000000636865636B73756D206D69736D61748F
:1063100063682C204C617374204C696E653A2000D0
:106320004C696E65204E756D626572206973206ED2
:106330006F74204C617374204C696E65204E756DCE
:106340006265722B312C204C617374204C696E6530
:106350003A2000257520627974657320777269741C
:1063600074656E20746F202553206174206164640D
:1063700072657373203078253038780A00442564BC
:10638000202D20526561642F577269746520255352
:106390000A003F3F00526F6D616E61004872766186
:1063A00074736B69004D616779617200536C6F762D
:1063B000656E63696E61004E6F72736B0053766534
:1063C0006E736B61004E656465726C616E64730020
:1063D000506F6C736B69004974616C69616E6F001A
:1063E0004672616E6361697300457370616E6F6CB4
:1063F00000446575747363680043657374696E6106
:1064000000456E676C6973680020436F756E742079
:10641000583A200045303A25642052504D205052C1
:106420004E313A25642052504D204530403A257572
:106430002050524E31403A25750A00526573656E00
:10644000640025533A20256C640A25530A002F2F37
:10645000616374696F6E3A6E6F74696669636174C3
:10646000696F6E2025530A0046696C616D656E7414
:106470002072756E6F7574206465746563746564ED
:10648000210064697361626C656400656E61626CB1
:10649000656400454550524F4D005352414D0044F4
:1064A0002D31202D20456E646C657373206C6F6FE9
:1064B000700A00416374697665204578747275646A
:1064C00065723A203000496E76616C6964206578A7
:1064D000747275646572004D323230205325640049
:1064E0005344207072696E74696E672062797465B6
:1064F0002000257500556E6B6E6F776E20636F6D93
:106500006D616E643A2022004D32303020496E7643
:10651000616C696420657874727564657220007AB4
:106520005F6D61783A20007A5F6D696E3A2000797C
:106530005F6D696E3A2000545249474745524544C1
:10654000006F70656E00785F6D696E3A200052656D
:10655000706F7274696E6720656E6473746F7020FB
:10656000737461747573004D3131322063616C6CEA
:1065700065642E20456D657267656E63792053747E
:106580006F702E002F2F616374696F6E3A75766C91
:106590006F5F7265636F766572795F72656164794A
:1065A0000025533A256C7520636D0A25533A256CF6
:1065B00075206D696E0A0053494C454E54004E4F8C
:1065C000524D414C002553204D4F44453A205065D3
:1065D0007263656E7420646F6E653A202568686426
:1065E0003B207072696E742074696D652072656DF0
:1065F00061696E696E6720696E206D696E733A20FD
:1066000025643B204368616E676520696E206D6973
:106610006E733A2025640A005072696E7465725375
:10662000746174653A2025640A00456E64206669C9
:106630006C65206C69737400426567696E206669D9
:106640006C65206C69737400556E6B6E6F776E208D
:10665000256320636F64653A2025730A000A504958
:106660004E44412074656D70657261747572653A4F
:1066700020252E3166205A20736869667420286DA3
:106680006D293A20252E3366000A537465703A202E
:1066900025642F360A000A537465703A2025642F4A
:1066A000362028736B6970706564290A50494E441E
:1066B000412074656D70657261747572653A20254C
:1066C00064205A20736869667420286D6D293A30F9
:1066D0000A000A5A45524F3A20252E33660A0073A3
:1066E000746172742074656D706572617475726521
:1066F0003A20252E31660A0025642020252E326698
:1067000000255320583A20252E356620593A202559
:106710002E3566205A3A20252E35660A00536C65C0
:1067200065702E2E2E0045303A25642052504D0AB9
:1067300050524E303A25642052504D0A00473930AD
:10674000004D31303700537570657250494E4441E9
:106750000048426564206F6E206C6F616400466C77
:10676000617368416972004572723A484F54454EF0
:10677000442046414E204552524F52002F2F616314
:1067800074696F6E3A726573756D6564002F2F6161
:106790006374696F6E3A726573756D65002F2F6152
:1067A0006374696F6E3A7265616479002F2F61635B
:1067B00074696F6E3A6E6F745F7265616479002FF1
:1067C0002F616374696F6E3A63616E63656C004D2F
:1067D0003834004F4B004C4344207374617475731C
:1067E000206368616E67656400534420636172646E
:1067F0002072656C6561736564002F2F6163746935
:106800006F6E3A737461727400473931004D3730DE
:1068100032004732382057004D3530300042616435
:1068200020696E7465727275707400576174636864
:10683000646F672074696D656F757400537461745B
:106840006963206D656D6F7279206861730A626596
:10685000656E206F7665727772697474656E004636
:1068600049524D57415245204352415348210A4312
:106870007261736820726561736F6E3A0A0020203E
:10688000506C616E6E6572427566666572427974AF
:1068900065733A20002046726565204D656D6F7204
:1068A000793A2000207C20417574686F723A20008C
:1068B000204C61737420557064617465643A2000E3
:1068C00020536F667477617265205265736574003A
:1068D000205761746368646F672052657365740044
:1068E0002042726F776E206F7574205265736574E5
:1068F000002045787465726E616C20526573657412
:1069000000506F7765725570006572726F722077F4
:10691000726974696E6720746F2066696C650044E3
:106920006F6E6520736176696E672066696C652E8F
:10693000006F6B0046696C616D656E74004D65613A
:10694000737572656420736B6577733A20256620D2
:1069500025660A0046697474696E67206661696C11
:106960006564203D3E2063616C6962726174696F89
:106970006E206661696C65642E0A0043616C696211
:10698000726174696F6E20737563636573732E0A29
:1069900000416C6C20342063616C696272617469BF
:1069A0006F6E20706F696E747320666F756E642EE3
:1069B0000A00312F3400312F3400312F3900457255
:1069C000723A5052494E542046414E204552524F41
:1069D000520025632533642F256481005A25362E05
:1069E00032662563005A2020202D2D2D200086257B
:1069F00033642525002D2D2D2525002533642525DF
:106A000000205344002020200020484F0020465200
:106A10004D2000872D2D3A2D2D2020008725337500
:106A20006820256325630087253032753A2530328A
:106A30007525632563002F2F616374696F6E3A704B
:106A40006175736564002F2F616374696F6E3A70AE
:106A5000617573650044756D7020746F2073657285
:106A600069616C0068656C702E7072757361336457
:106A70002E636F6D00666F72756D2E707275736127
:106A800033642E636F6D00707275736133642E63AF
:106A90006F6D004D3730310025533A0A2531382EBD
:106AA00032666D200A25533A0A2531306C64642021
:106AB000253032646820253032646D0025533A0A4F
:106AC0002531382E32666D200A25533A0A25313099
:106AD0006C646820253032646D2025303264730088
:106AE00025362E32666D6D0025530A25530A25532F
:106AF0003A0A25533A0025332E32668100252D317E
:106B0000342E3134533A0A25530A252D31342E318F
:106B100034533A25332E3266810A252D31342E31F5
:106B200034533A25332E3266810020203000202055
:106B3000310046494E44410050494E444100576996
:106B40007A61726420656E642073746174653A20A2
:106B500025640A0053706F6F6C4A6F696E00466956
:106B6000726D7761726500507275736120693320B0
:106B70004D4B322E3553204F4B2E004D36303000CA
:106B800053442063617264206F6B006F70656E52B6
:106B90006F6F74206661696C656400766F6C756DEB
:106BA000652E696E6974206661696C656400534482
:106BB00020696E6974206661696C006F70656E2073
:106BC0006661696C65642C2046696C653A200043F7
:106BD000616E6E6F7420656E746572207375626489
:106BE00069723A20004D3234004D32332025730053
:106BF0005072696E7465722073746F707065642072
:106C000064756520746F206572726F72732E2053E5
:106C100075706572766973696F6E207265717569DA
:106C20007265642E0047312045252D2E336620469F
:106C300032373030004D383300312F390088002092
:106C4000746F6F206C6F6E672065787472757369EE
:106C50006F6E2070726576656E7465640020636F78
:106C60006C6420657874727573696F6E20707265DC
:106C700076656E746564004D6F76652061626F7233
:106C800074656400084AD73B3BCE016E84BCBFFDEF
:106C9000C12F3D6C74319ABD56833DDA3D00C77FEC
:106CA00011BED9E4BB4C3E916BAAAABE0000008085
:106CB0003F05A84CCDB2D44EB93836A9020C50B914
:106CC000918688083CA6AAAA2ABE000000803F0739
:106CD000634236B79BD8A71A39685618AEBAAB5577
:106CE0008C1D3CB7CC5763BD6DEDFD753EF617723C
:106CF00031BF000000803F08000000BE922449120E
:106D00003EABAAAA2ABECDCCCC4C3E00000080BE31
:106D1000ABAAAAAA3E00000000BF000000803F000E
:106D200000000000084178D3BB4387D1133D190E02
:106D30003CC3BD4282AD2B3E68EC8276BED98FE16A
:106D4000A93E4C80EFFFBE01C4FF7F3F0000000062
:106D500000000D941B050C94AEC00C94B2B30C94BF
:106D6000CBFC0D940C320C94EAB00C94C1B00D9491
:106D70006C070C94C7BB0C9425B50C9478EF0D945C
:106D800007070D94C2070C9404F70D94FC120D94A0
:106D9000F9110D94CA2F0D942F320C94B3B00D94A9
:106DA00073090C94CABA0C9420FD0C94D0BB0C94BB
:106DB00018C10C9421E30C94C4FE0C940CB50D94F2
:106DC0008B3A0C94AFFE0C946DFE0D9410300C9425
:106DD0008B6D0C9494B60C94C5B00C943CC60C947A
:106DE0006DBC0D947D110C942DE30D94402F0C94EB
:106DF00038FF0C94F1FF0C9420B50C94A6C00D94B0
:106E00001F320C94EBFC0C9495BC0C9466EC0D9426
:106E1000940C0C94B7FC0C9452B70C941BF70C9484
:106E20007EFE0D940E050D942A020D94041E0C9402
:106E300090BB0C94FFFC0D9426120C94D1C00C94C2
:106E4000B3C00D9427320C94F5FC0D94BF070C943D
:106E500011B30C94846B0D94E63A0C94D4BA0C9450
:106E60005EB40C9407B50C94D2B00C9474B60D9427
:106E700084640C9453B50C947CB40C9409FD0D946B
:106E80007D000C94F3B00D94FE6A0C94B5E90D945A
:106E90003B310D94FC640C9415F00C946DEB0D9447
:106EA00031300D946A310D946A110C9440C10C94E8
:106EB000A8FE0C9442E30C9491B10C9431FD0D9416
:106EC000602F0C94CABB0C9479BC0C94F5C00D9443
:106ED00017320D940F320C94DFFC0C94D5FC0C94FB
:106EE0007D6D0D94A4010C940EE80D94FE060C9497
:106EF000C7C00C9406F70C94CDBB0D947E020C9485
:106F000023F80D946C2F0D943F320D94E26A0D948A
:106F1000CD0A0D946B960C948CEF0C9400B10D94EB
:106F20003D030C9436C10C9448E90C941DB30D94A8
:106F300064940D944F320D94D2310C9465BC0C9432
:106F400030E30D9437320D9408100D940A120C940E
:106F5000EBC00D94DF640C940FFE0C9426FE0C9491
:106F6000A16D0D9496220C94B9E90C94F8B00C9490
:106F700003FE0D94670F0D94EA010D94241D0D94EA
:106F800016050C94A1EA0C941AC60D94F5060C94FF
:106F90000FEB0C94CD6D0C942CB30C9497B10C9416
:106FA00084BC0D94A6310C94D9C00D94E5020D94C7
:106FB00003650C9455BC0C9438B30D94360E0C94A8
:106FC00002FF0C94A5F70D9460050D94FC2F0C9412
:106FD000B6FE0D94016B0C9416B50C94CCB50D94C3
:106FE000B02F0D9457320C94D6BB0C94DFBB0C948D
:106FF0000EC10C945FFD0D9467320C94BDC00D94CE
:10700000136B0C940BEB0C9436E30D940E6B0C94F9
:1070100043B30C94C8B00C942CC10C946BFE0D942B
:10702000C6110C94CEB00D9406320C94FFBA0C9499
:10703000DF6D0D94FF640D94F32F0C9422C10D9419
:1070400060310C94F4B00C945FB00C9400E30C9499
:1070500033E30C9490E60C940BF80D94CF400D9410
:10706000D8310C941BFE0C94BDFE0C94AA6D0C94AC
:10707000FFC30C94FFC00C94E6B00C9469B50D945A
:10708000E52F0D946D310C944D5E0C944B700D9466
:10709000D5310C9493BC0C94E8E20C94EEB00C94B3
:1070A00011B50C94FCB00D94762F0C945DBC0C942F
:1070B000306F0C9473FC0D9447320C94D3BB0D9439
:1070C000DB2F0C9448FE0C94726D0D949C6A0C940A
:1070D00002B50C94DCB00D9463310C9464FE0C94F6
:1070E0004AEA0D94056B0C94E0B00D949D640C94E9
:1070F000DCE20C94E5B50D947F040C94B9B00D94CA
:107100005F320D94E12F0C9444BA0C94BDB00C94F2
:10711000C1FC0D9409320D94510D0C94AEB80C9431
:10712000E1C00C9408E80C94586D0C941BB50D94B8
:1071300023310D943A010C94D8B00C9498BC6E6134
:107140006E00696E660000407A10F35A00A0724E1D
:1071500018090010A5D4E80000E87648170000E4FC
:107160000B54020000CA9A3B000000E1F505000044
:1071700080969800000040420F000000A0860100A9
:107180000000102700000000E80300000000640079
:10719000000000000A0000000000010000000000E4
:1071A0002C76D888DC674F0823DFC1DFAE59E1B108
:1071B000B796E5E3E453C63AE651997696E8E6C217
:1071C0008426EB898C9B62ED407C6FFCEFBC9C9F1E
:1071D00040F2BAA56FA5F490055A2AF75C936B6C40
:1071E000F9676DC11BFCE0E40D47FEF520E6B50034
:1071F000D0ED902E0300943577050080841E0800A2
:1072000000204E0A000000C80C333333330F986E51
:1072100012831141EF8D2114893BE65516CFFEE60E
:10722000DB18D1844B381BF77C1D901DA4BBE424D4
:10723000203284725E228100C9F124ECA1E53D2751
:107240002200002045535000204E535000204F464E
:107250004600204F4E005056303100205B4D505DAF
:107260002000256920686F757273202569206D697B
:107270006E757465730052582074696D656F75740E
:10728000004D333130004D313132004D313130005D
:1072900046756C6C205258204275666665720053C4
:1072A000657474696E67732053746F7265640053FC
:1072B000746F7265642073657474696E677320728D
:1072C00065747269657665640048617264636F64B1
:1072D00065642044656661756C74205365747469D7
:1072E0006E6773204C6F6164656400563200000065
:1072F00000C8420000C8420000C843000005430027
:1073000000484300004843000040410000F042E8CC
:10731000030000E8030000C800000088130000001C
:10732000409C4400409C44000000000000000020FD
:107330004E00000000204100002041CDCCCC3E009A
:10734000009040000000000000000000000000CDA0
:10735000CCCC3E3D0A8141FF08433EB099AB438F00
:1073600042FC42E65A343F4C62B045000000000047
:107370004040000034420000000000000000000017
:107380000041000000E03F00002C4300002C4300BF
:107390000040410000F042C0030000C0030000C8EC
:1073A000000000881300001010101000409C4400E2
:1073B00000803F0000003F191400000020307800DA
:1073C000203078006572726F723A200044323320A8
:1073D0002D20656D657267656E63792073657269CE
:1073E000616C2064756D7000437573746F6D004E31
:1073F000796C6F6E504100536174696E20200054A7
:10740000657874757200536D6F6F746800312E303B
:1074100000312E3500554E4B4E4F574E004C4131EA
:1074200030433A204C696E65617220416476616E2A
:107430006365206D6F64653A20004C413130433AFA
:107440002041646A757374656420452D4A65726BCA
:107450003A200020AA51A63E0FA8AF004800699626
:107460000000DF6025555887680427F2E0005E348D
:1074700003CC1960F33C0EF88F00DB0802949200F5
:107480003E1C079A8700E524008528527E06001BD3
:10749000E4007E781270787061F812788F884178F5
:1074A0004270787061782570787061F850788F88B4
:1074B000D1F02527078761F025278F88412C0D27DC
:1074C000AA50D1BC0707871161BE788F8811417817
:1074D0005270787061F852788F88412012788870E5
:1074E0006320527888706348527888874303111765
:1074F000997064181278F870654412F8F8F045181D
:107500004278F87065182578F87065185278F87028
:1075100065185078F870650C078F872365A20F8F68
:107520008F114500120622706900120722274900B8
:107530002506227069002507222749001206222706
:107540006C026236A2706C40456C44704C0362223F
:1075500022706C43888888F04C7812BC88806E78E2
:1075600052BC88806E38127888706F78127888875D
:107570004F38427888706F38257888706F3A007974
:10758000AC786F3D079AAC786F7850788887EF3980
:10759000497888706F0852BC8880729852F88F982A
:1075A0005220127870F07348127863875320527813
:1075B00070F0734852786387531007870F24731253
:1075C000786387245360699A988BE22304E44430FB
:1075D00074104E444324747C12888960753C508832
:1075E0008870557825288960757949088960753CC7
:1075F00012887070790C12885222594412F124F0CA
:107600007A4452F124F07A8C52F0368F5A4420F1A9
:1076100024F07A00401454CDCCCC3D0AD7233C173B
:10762000B7D13877CC2B329595E6241FB14F0A009D
:107630000020410000C84200401C4620BCBE4CCA8D
:107640001B0E5AAEC59D744E414E494E4600007AFF
:10765000430000524300005243000000000000803D
:10766000C09A99193E00000000000080C09A991944
:107670003E20503A002042403A0020403A00202F5D
:10768000002054303A00202F0020423A00202F00E2
:10769000543A0025534578636573736976652062B3
:1076A0006564206C6576656C696E6720636F7272C5
:1076B000656374696F6E3A202569206D6963726F26
:1076C0006E730A00426564206C6576656C696E674E
:1076D000206661696C65642E20546F6F206D756340
:1076E0006820766172696174696F6E2066726F6D71
:1076F00020656570726F6D206D657368004265640A
:10770000206C6576656C696E67206661696C65647E
:107710002E2053656E736F7220747269676765728D
:10772000656420746F6F20736F6F6E002020004DB2
:107730006561737572656420706F696E74733A0069
:107740005A20736561726368206865696768743A76
:1077500020352E3066004E756D20582C593A203752
:107760002C37004D65736820626564206C65766512
:107770006C696E67206E6F74206163746976652E24
:107780000020453A00205A3A0020593A0020453A54
:1077900000205A3A0020593A00583A00202D3E2045
:1077A0000053706F6F6C4A6F696E3A20002C200096
:1077B000496E61637469766974792053687574647D
:1077C0006F776E004B494C4C45442E005072696EE9
:1077D0007465722068616C7465642E206B696C6CD2
:1077E00028292063616C6C656421005A206C6976DD
:1077F000652061646A757374206F7574206F6620EC
:1078000072616E67652E2053657474696E672074AB
:107810006F20302E20436C69636B20746F20636F80
:107820006E74696E75652E005A206C6976652061EC
:10783000646A757374206F7574206F662072616E50
:1078400067652E2053657474696E6720746F2030ED
:107850000020453A3020423A00543A00627573796C
:107860003A2070617573656420666F7220696E706E
:10787000757400627573793A207061757365642060
:10788000666F72207573657200627573793A207045
:10789000726F63657373696E670073657269616C9B
:1078A0002064756D702000496E76616C69642054A7
:1078B00020636F64652E004475706C696361746544
:1078C00020542D636F64652069676E6F7265642E46
:1078D00000416476616E6365204B3D004B206F75FF
:1078E00074206F6620616C6C6F7765642072616EC6
:1078F000676521004D4B322E3553004D4B322E35EE
:10790000534D4D553253001C4FFC002533642F2539
:1079100033640025336400200A200A200A20002551
:1079200053537461746973746963733A0A255320FD
:10793000204D37382053256C752054256C750A006E
:1079400025534172632053657474696E67733A20DE
:10795000503A4D6178206C656E677468286D6D29AA
:1079600020533A4D696E206C656E67746820286DEF
:107970006D29204E3A436F7272656374696F6E733E
:1079800020523A4D696E207365676D656E74732081
:10799000463A5365676D656E74732F7365632E0A7F
:1079A000255320204D3231342050252E326620536D
:1079B000252E3266204E25642052256420462564FB
:1079C0000A00255346696C616D656E742073657499
:1079D00074696E67733A2044697361626C65640A06
:1079E00000255346696C616D656E7420736574740F
:1079F000696E67733A0A25532020204D32303020BB
:107A000044252E32660A00255352657472616374F0
:107A10003A20533D4C656E67746820286D6D2920AF
:107A2000463A537065656420286D6D2F6D29205A84
:107A30003A205A4C69667420286D6D290A25532016
:107A400020204D3230372053252E32662046252EF9
:107A50003266205A252E32660A25535265636F76A8
:107A600065723A20533D4578747261206C656E678B
:107A7000746820286D6D2920463A5370656564202E
:107A8000286D6D2F6D290A25532020204D32303866
:107A90002053252E32662046252E32660A25534174
:107AA00075746F2D526574726163743A20533D3062
:107AB00020746F2064697361626C652C20312074BE
:107AC0006F20696E74657270726574206578747267
:107AD0007564652D6F6E6C79206D6F7665732061AE
:107AE00073207265747261637473206F72207265A3
:107AF000636F7665726965730A25532020204D32C5
:107B00003039205325640A002553504944206865C4
:107B100061746265642073657474696E67733A0A90
:107B200025532020204D3330342050252E3266201E
:107B300049252E32662044252E32660A00255350F0
:107B400049442073657474696E67733A0A2553203B
:107B500020204D3330312050252E32662049252EED
:107B600032662044252E32660A0025535374657010
:107B7000732070657220756E69743A0A255320204F
:107B80004D39322058252E32662059252E32662056
:107B90005A252E32662045252E32660A25534D6120
:107BA00078696D756D2066656564726174657320B2
:107BB000286D6D2F73293A0A255320204D3230331A
:107BC0002058252E32662059252E3266205A252E21
:107BD00032662045252E32660A25534D6178696D3F
:107BE000756D20616363656C65726174696F6E2089
:107BF000286D6D2F7332293A0A255320204D3230DB
:107C0000312058256C752059256C75205A256C75C6
:107C10002045256C750A2553416363656C65726167
:107C200074696F6E3A20503D7072696E742C2052E8
:107C30003D726574726163742C20543D7472617678
:107C4000656C0A255320204D3230342050252E32C9
:107C5000662052252E32662054252E32660A255380
:107C6000416476616E636564207661726961626CFD
:107C700065733A20533D4D696E2066656564726197
:107C8000746520286D6D2F73292C20543D4D696E2D
:107C90002074726176656C206665656472617465D6
:107CA00020286D6D2F73292C20423D6D696E696D02
:107CB000756D207365676D656E742074696D6520E0
:107CC000287573292C20583D6D6178696D756D207C
:107CD0005859206A65726B20286D6D2F73292C20EE
:107CE000205A3D6D6178696D756D205A206A657204
:107CF0006B20286D6D2F73292C2020453D6D6178F8
:107D0000696D756D2045206A65726B20286D6D2F39
:107D100073290A255320204D3230352053252E3229
:107D2000662054252E32662042256C752058252E5B
:107D300032662059252E3266205A252E326620457D
:107D4000252E32660A2553486F6D65206F6666736F
:107D5000657420286D6D293A0A255320204D323054
:107D6000362058252E32662059252E3266205A2577
:107D70002E32660A004361703A25533A25630A00A1
:107D800050525553415F4D4D553200455854454E64
:107D90004445445F4D3230004155544F5245504F99
:107DA00052545F504F534954494F4E004155544F20
:107DB0005245504F52545F46414E53004155544F27
:107DC0005245504F52545F54454D50000044656C2D
:107DD0006574696F6E206661696C65642C20466904
:107DE0006C653A200046696C652064656C65746555
:107DF000643A004E6F74205344207072696E746947
:107E00006E67005072696E7420736176656400530A
:107E100044207072696E742070617573656400250A
:107E200033642F25336400667600746878005052FE
:107E30004E0022283229006E6F2076616C69642022
:107E4000636F6D6D616E64007A65726F72697A65D9
:107E50006400666163746F727920726573746F7207
:107E6000656400696E6465782C2074656D702C20E3
:107E700075737465702C20756D0050494E44412017
:107E800063616C207374617475733A2000503A001A
:107E90005761697420666F722050494E44412074C6
:107EA00061726765742074656D7065726174757256
:107EB000653A00204100205000204200204C002064
:107EC0005200205A00204E4F5420494E49544941F7
:107ED0004C495A45440053686565742000205A2077
:107EE00056414C5545204F5554204F462052414E47
:107EF000474500496E76616C6964207368656574F6
:107F00002049442E20416C6C6F7765643A20302EF6
:107F10002E004155544F004C414E472053454C20B4
:107F2000464F524345440020643A0020693A0020FD
:107F3000703A0020643A0020693A0020703A002527
:107F40006925250A00256925250A002228312900EE
:107F50002F2F00002045585452554445525F434F3F
:107F6000554E543A3100204D414348494E455F54E7
:107F70005950453A00312E3000206261736564200B
:107F80006F6E204D61726C696E204649524D5741AB
:107F900052455F55524C3A68747470733A2F2F678C
:107FA00069746875622E636F6D2F707275736133BB
:107FB000642F50727573612D4669726D77617265B9
:107FC0002050524F544F434F4C5F56455253494FE8
:107FD0004E3A00373733313032346564005F003851
:107FE000323739002B004649524D574152455F4EBA
:107FF000414D453A50727573612D4669726D7761D6
:10800000726520004D3131332053006F6B20006EBC
:108010002F61003F546F736869626120466C617321
:1080200068416972204765744950206661696C65D2
:10803000640A00000125301D0CFF24311C0BFF23B6
:108040002F1B0A17FF0406222B1A03363535382555
:1080500069206D696E2C2025692073656300496E67
:1080600076616C6964204D20636F64653A202573E6
:108070000A0050494E44412070726F62652063616E
:108080006C6962726174696F6E20737461727400DE
:108090004E6F2050494E444120746865726D69737B
:1080A000746F7200736574006E6F7A7A6C65004D40
:1080B000424C004652004C7A004C616E6700315FC2
:1080C00037356D6D5F4D4B3235532D52414D426FFB
:1080D0003133612D453344763666756C6C005265DC
:1080E0007600332E31342E312D383237390046693F
:1080F0007200534E20696E76616C696400534E00C5
:108100005245534554004D4D555245530075766CBC
:108110006F0046414E0046414E50494E5453540064
:108120005052555341004D3130345330004731588F
:1081300031305931383046343030300047315A31DF
:10814000304631333030004D313430533000473118
:10815000452D302E3037354632313030004D3230FB
:108160003453313030300047315A354637323030B1
:10817000004731452D312E35463231303000473100
:108180005A302E32004731583230322E354538467B
:1081900031343030004731592D32463130303000E3
:1081A000473158323430453235463232303000476C
:1081B000315A302E33463130303000473158353562
:1081C000453846323030300047315835453239462F
:1081D0003138303000473158353545323946313045
:1081E000373300473932453000473238004D31309F
:1081F00039004D313930001000C90210012C014006
:1082000001220170011801B0010E01F001040150BA
:1082100002FA00B002F0003003E600D003DC009068
:1082200004D2007005C800A006BE000008B400B06B
:1082300009AA00D00BA000600E960060118C00000F
:1082400015820020197800C01D6E00A0226400B0C5
:10825000275A00902C500000314600E0343C0010BA
:10826000383200903A2800603C1E00A03D14008087
:108270003E0A00203F00004578706572696D656EAA
:1082800074616C00302E383000302E363000302EC5
:10829000343000302E32350044697361626C6520E1
:1082A0006661726D206D6F64650052657365742040
:1082B0004D4D55004D4D55004D3434004739390072
:1082C00044697361626C65206661726D206D6F64D4
:1082D000653F00473238205859004D20383400851A
:1082E0002E2E002533642F30002533642F30006C90
:1082F00063645F73656C66636865636B5F6178690F
:10830000732025642C2025640A00486F74656E6410
:1083100000426564005A00590058002D2D2D2D2D66
:108320002D2D2D2D2D2D2D2D2D2D2D2D2D2D2D00AA
:10833000537570657250494E44413A003D6741673C
:108340004E8147813C812D810D682681CF67473161
:1083500059252E346645252E34660047315A252E80
:1083600032660047315835305931353500E3813DAB
:1083700067356C718167815D81473158252E346680
:1083800045252E3466004731463130383000D581DE
:10839000C881BB81AF81E381A081958185817E8188
:1083A0005425640047315A302E34004731592D335B
:1083B0004631303030004167F281ED81E981E3815F
:1083C0004D3834205859004D31303920533238302F
:1083D0000047312058313235205A32303020463172
:1083E00030303000496E76616C6964205049442019
:1083F00063616C2E20726573756C74732E204E6FE2
:10840000742073746F72656420746F2045455052F8
:108410004F4D2E004D3330312050252E32662049ED
:10842000252E32662044252E3266004D333033200F
:1084300045302053253375005243004445560042D1
:1084400045544100414C50484100000021002400A7
:1084500027002A002D003000330001010000040134
:1084600007010A0100002200250028002B002E0031
:108470003100340002010000050108010B01000079
:1084800020002300260029002C002F0032000001CC
:108490000000030106010901050505050705080897
:1084A0000808020202020A0A08080404040401017E
:1084B0000101010101010303030303030303040793
:1084C00007070C0C0C0C0C0C0C0C0202020206062A
:1084D0000606060606060B0B0B0B0B0B0B0B070712
:1084E0000A0A0A0A0A0A0505050404040808010222
:1084F00010202008081020401020408002010201B6
:10850000080402010102040810204080804020106D
:1085100008040201800402018040201008040201C6
:10852000080402010102040810204080010204082E
:108530001020408010080408801020400440801063
:108540002040048000000A0B02090C0D0E080703EE
:108550000401000000000000000000000000000016
:10856000000000000000000000000000000000000B
:1085700012111000000000000000000000000000C8
:1085800000000000000000000000000000000000EB
:1085900000000000000000000000332E31342E31B6
:1085A000000A204F726967696E616C2050727573A2
:1085B000612069330A202020507275736120526552
:1085C0007365617263680A2532302E32305300536E
:1085D000706F6F6C4A6F696E20697320006164630D
:1085E0005F696E697400200A200A200A2000416C2D
:1085F0006C20446174610053657276696365207014
:10860000726570005368697070696E67207072657A
:10861000700053746174697374696373004C616EA4
:1086200067756167650045524153494E4720616C4B
:108630006C206461746100466163746F72792052CA
:108640004553455400505255534133444657000357
:10865000000E000100400003000200000004007052
:1086600072757361336400323032352D30342D32FF
:10867000322032323A30333A35330020332E31341F
:108680002E312D383237395F373733313032346558
:1086900064007374617274004D323900252D392ED7
:1086A00039535B0033332942000058419A998D4178
:1086B00033335340200A200A20004D4D55323A00F2
:1086C0004D6561737572652063656E7465722020F7
:1086D0000078797A63616C5F6D6561737572655F4F
:1086E000656E7465720A0078797A63616C5F737085
:1086F0006972616C382063783D25642063793D257B
:1087000064207A303D256420647A3D2564207261BE
:10871000646975733D25642061643D25640A0078B1
:10872000797A63616C5F7365617263685A206E6FFA
:10873000207369676E616C0A20783D256C6420792E
:108740003D256C64207A3D256C640A00204F4E2D37
:108750005349474E414C20617420783D256420796F
:108760003D2564207A3D25642061643D25640A002E
:1087700078797A63616C5F7365617263685A207897
:108780003D256C6420793D256C64207A3D256C6420
:108790000A002530327800205B25662025665D20A2
:1087A0006D6D207061747465726E2063656E7465A2
:1087B000720A00205B25662025665D5B25665D20CC
:1087C0006D6D20646976657267656E63650A000089
:1087D00000F000F801FC03FE07FE07FE07FE07FCA1
:1087E00003F801F000000000000000F000F801FCB8
:1087F00003FC03FC03FC03F801F000000000007818
:10880000797A63616C5F6D6561737572655F6C65C4
:108810006176650A00203C20005741524E494E4780
:108820003A2046726F6E7420706F696E74206E6F9E
:108830007420726561636861626C652E20592063E3
:108840006F6F7264696E6174653A000000004041A8
:108850000000804000005C430000804000005C435A
:1088600000004443000040410000444325642F348D
:1088700000497465726174696F6E3A200043616CDF
:108880006962726174696F6E206661696C656421EA
:1088900020436865636B2074686520617865732088
:1088A000616E642072756E20616761696E2E004D85
:1088B000494E54454D5020424544206669786564D0
:1088C000004D494E54454D5020484F54454E44208C
:1088D00066697865640024F4D43050C38E20C2A247
:1088E0004017828B7011127A910D816CD90AA861A0
:1088F000E108C7586607615143061E4B5D05C14537
:10890000A7041A411104093D980371393103403617
:10891000DB0265339102D4305402802E1D02632C99
:10892000EE01752AC501B028A001102781018F250D
:1089300064012B244B01E0223401AC211F018D2066
:108940000D01801FFC00841EED00971DDF00B81C88
:10895000D200E61BC600201BBC00641AB200B2198C
:10896000A8000A19A0006A189900D11791004017B1
:108970008B00B516840031167E00B31579003A15C8
:108980007300C7146F0058146A00EE136600881352
:10899000630025135E00C7125B006C1257001512AE
:1089A0005400C111510070114F0021114B00D6101D
:1089B00049008D1047004610440002104200C00FCD
:1089C0004000800F3E00420F3C00060F3B00CB0EE4
:1089D0003800930E37005C0E3500270E3400F30D7F
:1089E0003200C10D3100900D3000600D2E00320DAF
:1089F0002D00050D2C00D90C2B00AE0C2900850C88
:108A000029005C0C2700350C27000E0C2600E80B13
:108A10002400C40B2400A00B23007D0B23005A0B61
:108A20002100390B2100180B2000F80A1F00D90A79
:108A30001E00BB0A1E009D0A1D00800A1D00630A5D
:108A40001C00470A1B002C0A1B00110A1A00F70918
:108A50001A00DD091900C4091900AB0919009209AF
:108A600017007B091800630917004C091600360926
:108A70001600200916000A091500F5081500E0087F
:108A80001400CC081400B8081400A40814009008BE
:108A900013007D0812006B081300580812004608E6
:108AA00012003408110023081100120811000108F7
:108AB0001100F0071000E0071000D0071000C007F9
:108AC0001000B0070F00A107100091070E008307E8
:108AD0000F0074070F0065070E0057070E004907C7
:108AE0000E003B070D002E070E0020070D00130798
:108AF0000D0006070D00F9060C00ED060D00E0065E
:108B00000C00D4060C00C8060C00BC060C00B00615
:108B10000C00A4060B0099060C008D060B008206C3
:108B20000B0077060B006C060B0061060A00570667
:108B30000B004C060A0042060A0038060A002E0600
:108B40000A0024060A001A060A0010060900070691
:108B50000A00FD050900F4050900EB050900E2051E
:108B60000900D9050900D0050900C7050900BE059F
:108B70000900B5050800AD050800A50509009C051C
:108B80000800940508008C050800840508007C0591
:108B90000800740508006C050700650508005D0500
:108BA0000700560508004E05070047050700400569
:108BB000080038050700310507002A0507002305CE
:108BC00007001C050600160507000F05070008052D
:108BD000060002050700FB040600F5040700EE048A
:108BE0000600E8040600E2040700DB040600D504E2
:108BF0000600CF040600C9040600C3040600BD0435
:108C00000600B7040600B1040500AC040600A60483
:108C10000600A00405009B040600950405009004CE
:108C200006008A04050085040500800406007A0415
:108C3000050075040500700405006B04050066045A
:108C40000500610405005C0405005704050052049A
:108C500005004D04050048040500430405003E04DA
:108C600004003A04050035040500300404002C0417
:108C7000050027040400230405001E0404001A0450
:108C8000040016040500110404000D040400090486
:108C900005000404040000040400FC030400F803BD
:108CA0000400F4030400F0030400EC030400E803F0
:108CB0000400E4030400E0030400DC030400D80320
:108CC0000400D4030400D0030400CC030400C80350
:108CD0000300C503030024F404D9201BC40C5C0E5C
:108CE0009804C4095F0265077101F405F900FB04EB
:108CF000B30048048700C10369005803550003030B
:108D00004500BE023A008402310053022A002902C3
:108D1000250004022000E4011C00C8011900AF0175
:108D20001700980114008401130071011000610103
:108D3000100051010E0043010D0036010B002B0104
:108D40000B0020010B00150109000C0109000301B3
:108D50000800FB000800F3000800EB000700E40037
:108D60000600DE000600D8000600D2000600CC0097
:108D70000500C7000500C2000500BD000400B900E1
:108D80000400B5000400B1000400AD000400A90017
:108D90000400A5000300A20003009F0004009B0044
:108DA0000300980003009500020093000300900068
:108DB00003008D0002008B00030088000200860083
:108DC000020084000300810002007F0002007D0099
:108DD00002007B00020079000200770001007600AB
:108DE00002007400020072000100710002006F00B6
:108DF00002006D0001006C0002006A0001006900C1
:108E000002006700010066000100650001006400C7
:108E100002006200010061000100600001005F00CB
:108E200002005D0001005C0001005B0001005A00CF
:108E300001005900010058000100570001005600D0
:108E400001005500010054000100530000005300D0
:108E500001005200010051000100500001004F00CC
:108E600001004E0000004E0001004D0001004C00CA
:108E700001004B0000004B0001004A0001004900C6
:108E800001004800000048000100470001004600C2
:108E900000004600010045000000450001004400BC
:108EA00001004300000043000100420000004200B6
:108EB00001004100000041000100400001003F00AE
:108EC00000003F0001003E0000003E0001003D00A8
:108ED00000003D0001003C0000003C0000003C00A0
:108EE00001003B0000003B0001003A0000003A0096
:108EF000010039000000390001003800000038008E
:108F00000000380001003700000037000100360083
:108F1000000036000000360001003500000035007A
:108F2000000035000100340000003400000034006F
:108F30000100330000003300000033000100320064
:108F4000000032000000320001003100000031005A
:108F5000000031000100300000003000000030004F
:108F600001002F0000002F0000002F0000002F0044
:108F700001002E0000002E0000002E0001002D0038
:108F800000002D0000002D0000002D0001002C002D
:108F900000002C0000002C0000002C0001002B0021
:108FA00000002B0000002B0000002B0001002A0015
:108FB00000002A0000002A0000002A000100290009
:108FC00000002900000029000000290000002900FD
:108FD00001002800000028000000280000002800F0
:108FE00000002800010027000000270000002700E3
:108FF00000002700000027000100260000002600D6
:1090000000002600000026000000260001002500C8
:1090100000002500000025000000250000002500BC
:1090200000002500010024000000240000002400AE
:1090300000002400000024000100230000002300A1
:109040000000230000002300000023000000230094
:109050000000230001002200000022000000220086
:109060000000220000002200000022000100210078
:10907000000021000000210000002100000021006C
:10908000000021000000210001002000000020005D
:109090000000200000002000000020000000200050
:1090A000000020000000200001001F0000001F0041
:1090B00000001F0000001F0000001F0000001F0034
:1090C00000001F0001001E0000001E0000001E0026
:1090D00000001E00000045303A20005A3A20005996
:1090E0003A2000583A20004D53312C4D5332205035
:1090F000696E7300504944204175746F74756E65D4
:109100002066696E697368656421205075742074E7
:109110006865206C617374204B702C204B69206152
:109120006E64204B6420636F6E7374616E74732081
:1091300066726F6D2061626F766520696E746F2054
:10914000436F6E66696775726174696F6E2E680031
:10915000504944204175746F74756E65206661696D
:109160006C6564212074696D656F75740020403AE8
:1091700000543A00423A00504944204175746F74DB
:10918000756E65206661696C6564212054656D703B
:109190006572617475726520746F6F2068696768A5
:1091A00000204B643A2000204B693A2000204B708D
:1091B0003A200020436C6173736963205049442056
:1091C000002054753A2000204B753A2000206D6134
:1091D000783A2000206D696E3A200020643A200021
:1091E00020626961733A2000504944204175746FD0
:1091F00074756E6520737461727400504944204127
:1092000075746F74756E65206661696C65642E2077
:10921000426164206578747275646572206E756D44
:109220006265722E00486F74656E642066616E2000
:109230007370656564206973206C6F776572207444
:1092400068616E206578706563746564005072694A
:109250006E742066616E207370656564206973208A
:109260006C6F776572207468616E206578706563D5
:10927000746564004D494E54454D502042454400AC
:109280004D494E54454D50004D415854454D5000A8
:109290004D415854454D50204245440070012C0129
:1092A00090012701B0012201C0011D01F001180148
:1092B0001002130130020E01600209019002040144
:1092C000C002FF000003FA004003F5008003F00035
:1092D000D003EB002004E6007004E100E004DC00B1
:1092E0004005D700C005D2004006CD00D006C8001A
:1092F0008007C3003008BE00F008B900C009B40000
:10930000B00AAF00B00BAA00D00CA500000EA00060
:10931000500F9B00C01096005012910000148C005A
:10932000C0158700B0178200B0197D00D01B7800EF
:10933000001E730040206E0090226900F02464003B
:1093400040275F0090295A00E02B5500102E500056
:1093500020304B0010324600E033410090353C0095
:109360001037370070383200A0392D00B03A28008D
:10937000A03B2300603C1E00103D1900903D1400EE
:10938000103E0F00703E0A00C03E0500003F000086
:1093900020484F54454E4420544845524D414C209E
:1093A00052554E4157415900204845415442454489
:1093B00020544845524D414C2052554E4157415939
:1093C00000544845524D414C2052554E4157415949
:1093D0000042454420544845524D414C2052554E80
:1093E000415741590020544845524D414C20525557
:1093F0004E41574159202850524548454154204834
:109400004F54454E44290020544845524D414C206C
:1094100052554E41574159202850524548454154D4
:109420002048454154424544290050524548454151
:1094300054204552524F5200424544205052454814
:10944000454154204552524F52002074726967675B
:109450006572656421004865617465727320737775
:10946000697463686564206F66662E20003A200088
:109470004572723A200000FF0102010002FFFFFE68
:109480000001FE01FF00506C656173652072657319
:1094900074617274005553415254322072782046E0
:1094A000756C6C212121003A2000252D31322E319E
:1094B0003253252D642F36002533642F252D336438
:1094C00000203A200025335300252D377300252D29
:1094D00031352E313553252D35640A252D31352E64
:1094E000313553252D35640A0025530A20252D31A9
:1094F000362E313653252D33640A20252D31362E54
:10950000313653252D33640025530A20252D31365D
:109510002E313653252D33640A20252D31362E3138
:109520003653252D33640A20252D31362E313653FE
:10953000252D33640025530A20252D31362E313652
:1095400053252D33640A25530A20252D31362E311B
:109550003653252D33640A0020257325336481207A
:109560000A0025752E25752E25752E2575002000DF
:109570002000466C61736841697220495020416443
:1095800064723A004D4D5520202020202020204E8E
:109590002F410025642E25642E2564002046573A6D
:1095A00000323032352D30342D323200453344769E
:1095B0003666756C6C0052414D426F31336100313B
:1095C0005F37356D6D5F4D4B323553002048617309
:1095D000683A373733313032346564002052657071
:1095E0006F3A707275736133640020332E31342EFC
:1095F000312D38323739004669726D776172653ABC
:10960000003E00464C4558202D20203234302F3566
:109610003000464C4558202D202032343000505028
:109620002020202D20203235342F31303000505072
:109630002020202D20203235340048495053202D41
:1096400020203232302F3130300048495053202D05
:1096500020203232300041425320202D202032354C
:10966000352F3130300041425320202D202032351B
:10967000350050412020202D20203237352F393021
:109680000050412020202D202032373500505642F6
:1096900020202D20203231352F37350050564220E2
:1096A000202D20203231350050432020202D202035
:1096B0003237352F3130350050432020202D2020E7
:1096C0003237350041534120202D20203236302FB3
:1096D0003130350041534120202D202032363000DA
:1096E00050455420202D20203233302F3835005063
:1096F000455420202D202032333000504C41202072
:109700002D20203231352F363000504C4120202D75
:109710002020323135006E6F7A7A6C65202D202042
:109720003235302F30006661726D2020202D2020D0
:109730003235302F383000252D31322E313253253D
:109740002B382E31660045787472756465723A0064
:1097500025632531372E32666D6D00583A00593A2F
:10976000005A3A002563252D31332E313353252BF2
:10977000352E3366002533750050494E4441206331
:10978000616C6962726174696F6E206661696C6593
:10979000642E20436F6E74696E75652077697468F6
:1097A000207072657373696E6720746865206B6ED4
:1097B0006F622E0050494E44412063616C696272B1
:1097C0006174696F6E20646F6E652E20436F6E74D6
:1097D000696E756520776974682070726573736946
:1097E0006E6720746865206B6E6F622E005A3000C1
:1097F0005A31005930005931005830005831004575
:109800006E642073746F70732064696167004738F9
:1098100030004D3435004D3435205A00473736007E
:109820004D3730312050300057697A6172642073AF
:10983000746174653A2025640A0078797A63616CF2
:109840005F73706972616C322063783D25642063B8
:10985000793D2564207A303D256420647A3D256475
:10986000207261646975733D25642061643D2564DF
:109870000A000A00436F756E74646F776E3A202594
:1098800064200025640A005363616E20636F756E67
:1098900074646F776E3A20005061747465726E2044
:1098A00063656E746572205B25662025665D2C20DD
:1098B0006D6174636820256625250A00205B256696
:1098C0002C2025665D5B25665D2066696E616C20D7
:1098D000636972636C650A000000A0400000A0404C
:1098E0000000004000007A43000056439AD95143DB
:1098F000FFFFFFE02D903E8988B24111369C3E77F4
:1099000077C14129CBB03EEFEEDA41BA49CC3EEF08
:10991000EEFC4161C3F33EEFEE16429CA2133FCD35
:10992000CC36428AB0113FABAA56428863DD3DABCC
:10993000AA5642B8AF433F555572421826533F339B
:10994000B38242302A593FEF6E8642000070C10058
:1099500000C8420000C4C10000A0410000E0C000F7
:10996000002041000060C00000C0400000A0412273
:1099700022F2400000A0C19A99A14000000CC255FB
:10998000550542436F6F6C696E672074696D65722F
:109990002073746F7070656400486561746572202F
:1099A000636F6F6C646F776E00436F6F6C696E6787
:1099B0002054696D656F7574207374617274656489
:1099C00000536176696E6720616E64207061726B0E
:1099D000696E670048656174657220636F6F6C64BF
:1099E0006F776E2070656E64696E6700526573757F
:1099F0006D696E672058595A0057726974696E67AD
:109A000020746F2066696C653A200046696C652099
:109A1000616C7265616479206F70656E6564006F5A
:109A2000575E574A5735571F570C57F656E256D1CF
:109A300056BB564A575E57A7569856845673565E7D
:109A400056025A4856365623561256FD55EA55D6F2
:109A500055C155B855A65591554D36303020415514
:109A6000544F0046494E44412066696C616D656EF5
:109A7000742072756E6F75742100436F6D6D756E15
:109A800069636174696F6E2074696D656F757400C8
:109A900050726F746F636F6C204572726F72000347
:109AA000000356657273696F6E206D69736D617422
:109AB000636800436F6D6D616E64204572726F72F2
:109AC00000436F6D6D616E642072656A65637465D5
:109AD00064004D4D5520427574746F6E207075731F
:109AE000686564005265747279427574746F6E5063
:109AF00072657373656400CC59B759A0598B597658
:109B000059625952593B5924590D59F958E558CFC2
:109B100058CF58CF58BA58BA58BA58A758A758A7C4
:109B2000589458945894587D587D587D5868586872
:109B300058685852585258525842582D5817580180
:109B400058F257E557CE57BB57A9579657845774C5
:109B500057427574746F6E00436865636B55736527
:109B600072496E7075742D62746E4C4D52200052A5
:109B7000657365745265747279417474656D70743F
:109B8000730046493A202046533A202020203E20A8
:109B900020822020208100486F74656E64207465E7
:109BA0006D70657261747572652072656163686558
:109BB0006400526573756D696E672054656D700041
:109BC000436F6F6C646F776E20666C616720636CA7
:109BD00065617265640020573A0020453A00543AA6
:109BE000004E6F2030784646207265636569766561
:109BF000640053656E64696E67203078464600469F
:109C0000696C652073656C656374656400205369D5
:109C10007A653A200046696C65206F70656E6564F0
:109C20003A20004E6F772066726573682066696C13
:109C3000653A20004E6F7720646F696E6720666911
:109C40006C653A20002220706F73002220706172D0
:109C5000656E743A2200535542524F5554494E4551
:109C60002043414C4C207461726765743A22007441
:109C70007279696E6720746F2063616C6C207375F4
:109C8000622D67636F64652066696C657320776910
:109C9000746820746F6F206D616E79206C657665D5
:109CA0006C732E002022257322002025236C78005F
:109CB0004449525F45584954004449525F454E5407
:109CC00045523A20257320222573220A00617574BB
:109CD0006F25692E6700041A44656372656D656EB1
:109CE000745265747279417474656D707473000890
:109CF0001B1C0B14525354436F6D6D54696D656F8B
:109D00007574002C206C6173742062797465733AE9
:109D1000200022206661696C65643A20427566669F
:109D200065722066756C6C21002200456E71756548
:109D3000696E6720746F207468652066726F6E7438
:109D40003A2022004572726F723A004D4D553274BE
:109D50006F6F6C3D004D4D55323A004D4D55323AC6
:109D6000006563686F3A003E53302A63362E004D1B
:109D70004D552069732000252E31305320002534A5
:109D80006400457872656D65207370616E206F6642
:109D900020746865205A2076616C756573210025F2
:109DA000642F39004D4D55323A00253364001801B7
:109DB0000419020A92611C61A2603560EC5F5A5F6F
:109DC000E25E7A5E2B5E0B5EBF5D0B5EA85DA85DFA
:109DD000A85DA85DA85DA85DA85DA85DA85DA85D5B
:109DE000A85DA85DA85DA85DA85DA85DA85DA85D4B
:109DF000A85DA85DA85DA85D715D305DE65C735CE3
:109E00003E5CF45BAA5B4C5B135BD15AB45A010114
:109E100001010101010271017101323232030303B8
:109E20000303030303030303030303030303030302
:109E30009393243803930301025603650066006779
:109E400000680069006A006B006C00730074007D9C
:109E5000007E00C900D300DD00CA00D400DE002D62
:109E600001370141012E01380142012F013901431F
:109E70000130013A01440131013B014501320191B8
:109E8000019201F501F601F701F801F901FA01FB70
:109E900001FC0184031F62886214620B6204628AFF
:109EA0004AFF3CFD61F361252E3230530A70727512
:109EB00073612E696F2F3034256875007B5B4552C6
:109EC000523A00332E31342E31005D5B4657523A00
:109ED000005D5B54494D3A005D5B464E4D3A005D76
:109EE0005B46454D3A005D5B5043443A005B544647
:109EF000553A005B50524E3A005B50464E3A305D48
:109F0000005B4449413A005D5B4154423A005D5B6D
:109F10004154303A005D5B5354423A005B53543035
:109F20003A007B5B50524E3A355D007B5B50524E9F
:109F30003A305D007B5B50524E3A395D007B5B509E
:109F4000524E3A385D007B5B5245533A305D5B467A
:109F5000494C3A007B5B5245533A315D5B46494C74
:109F60003A0000002110422063308440A550C660B2
:109F7000E770088129914AA16BB18CC1ADD1CEE1C6
:109F8000EFF13112100273325222B5529442F7723D
:109F9000D662399318837BB35AA3BDD39CC3FFF316
:109FA000DEE36224433420040114E664C774A4444D
:109FB00085546AA54BB528850995EEE5CFF5ACC566
:109FC0008DD55336722611163006D776F66695561D
:109FD000B4465BB77AA719973887DFF7FEE79DD7B6
:109FE000BCC7C448E5588668A778400861180228AD
:109FF0002338CCC9EDD98EE9AFF9488969990AA906
:10A000002BB9F55AD44AB77A966A711A500A333A7C
:10A01000122AFDDBDCCBBFFB9EEB799B588B3BBB55
:10A020001AABA66C877CE44CC55C222C033C600C0C
:10A03000411CAEED8FFDECCDCDDD2AAD0BBD688DA5
:10A04000499D977EB66ED55EF44E133E322E511E5C
:10A05000700E9FFFBEEFDDDFFCCF1BBF3AAF599FF5
:10A06000788F8891A981CAB1EBA10CD12DC14EF195
:10A070006FE18010A100C230E320045025404670FB
:10A080006760B9839893FBA3DAB33DC31CD37FE326
:10A090005EF3B1029012F322D2323542145277624B
:10A0A0005672EAB5CBA5A89589856EF54FE52CD5F6
:10A0B0000DC5E234C324A01481046674476424549B
:10A0C0000544DBA7FAB79987B8975FE77EF71DC706
:10A0D0003CD7D326F2369106B016576676761546EB
:10A0E00034564CD96DC90EF92FE9C899E9898AB956
:10A0F000ABA94458654806782768C018E10882383B
:10A10000A3287DCB5CDB3FEB1EFBF98BD89BBBAB65
:10A110009ABB754A545A376A167AF10AD01AB32A8A
:10A12000923A2EFD0FED6CDD4DCDAABD8BADE89DB5
:10A13000C98D267C076C645C454CA23C832CE01CDA
:10A14000C10C1FEF3EFF5DCF7CDF9BAFBABFD98F45
:10A15000F89F176E367E554E745E932EB23ED10E2A
:10A16000F01E7C3C3E3F2F2A225C00002D384D5EC5
:10A1700011241FBECFEFD1E2DEBFCDBF00E00CBF88
:10A1800013E0A0E0B2E0EEECFEE403E00BBF02C09F
:10A1900007900D92A430B107D9F727E1A4E0B3E00E
:10A1A00001C01D92A430B207E1F710E5C7EBD0E57E
:10A1B00000E006C021970109802FFE010F94ABA19A
:10A1C000C63BD10780E00807A9F70E949CD80D94F0
:10A1D00055A70C94B8742F923F924F925F926F9252
:10A1E0007F928F929F92AF92BF92CF92DF92EF9227
:10A1F000FF920F931F93CF93DF93CDB7DEB72F97C7
:10A200000FB6F894DEBF0FBECDBF6C011B015A0123
:10A21000FC011782168283819E012F5F3F4F490107
:10A2200081FDD2C08FEF9FEFEEC2F12C512C00E0E8
:10A23000003238F48B3209F190F48032F9F0833235
:10A2400009F107FD34C020ED280F2A3020F506FF64
:10A250001BC0FAE0FF9E200D1124F22E05C08D32A6
:10A2600079F0803371F70160F10193FD859193FFDF
:10A2700081911F018111DCCF1AC002600460F4CF0C
:10A280000860F2CF0061F0CF3AE0539E200D112418
:10A29000522E0062E9CF8E3221F406FDB1C2006475
:10A2A000E3CF8C3611F40068DFCF8836E9F29BEB00
:10A2B000980F933008F05FC00061805E06FD02C019
:10A2C00046E0F42E102F1F73853609F05BC0106432
:10A2D00017FF61C08F2D9BE39F1508F48BE3442487
:10A2E0004394480E27E03501F4E06F0E711CF50130
:10A2F0006081718182819381042DA4010F94549D0A
:10A300005C01F981FC87F0FF03C00DE2F3FF07C099
:10A310000BE211FD04C0012F047012FD00E22C8538
:10A320002C70E22E09F46BC00111D8C2F3E0E12CCD
:10A33000F515A0F483E0E52CE81A13FD08C0B6017A
:10A3400080E290E00F94039FEA94E110F8CF00239D
:10A3500029F0B601802F90E00F94039F3C852EE3F7
:10A36000A22E21E7B22E33FD04C092E4A92E91E77C
:10A37000B92E107122C09BE9980F933008F047C1A5
:10A380000F7E9CCF863611F41068A2CFFF2009F40F
:10A390009FCFFA949DCFE7E02F2DEF1518F427E01B
:10A3A00037E0F32E412C9FCF11118052B60190E07F
:10A3B0000F94039F8FEFA81AB80AF50184918111B9
:10A3C000F3CFE11084C25301F6019381F10193FDB3
:10A3D000859193FF81911F01882309F411C2853271
:10A3E00041F493FD859193FF81911F01853209F01E
:10A3F0001CCFB60190E00F94039F3501E4CF17FF07
:10A400006FC04A0CFC85F4FF04C08A81813309F4D3
:10A410004A9414140CF086C028E0241510F488E047
:10A42000482E85E090E017FF06C0C501B7FE02C0C8
:10A4300090E080E0019601110196FF2031F02F2D70
:10A4400030E02F5F3F4F820F931F5816190619F007
:10A4500014F0E52CE81A812F897011F4E11067C01F
:10A46000002329F0B601802F90E00F94039F13FD85
:10A4700002C0E11063C017FF7CC08501B7FE02C0B7
:10A4800010E000E0C501841991092C016F2D70E0E6
:10A49000EE27FF27E61BF70BFF87EE870F3F10071E
:10A4A00029F4B6018EE290E00F94039FA016B10646
:10A4B0000CF44BC0401651060CF047C0F501E01BF0
:10A4C000F10BE80DF91D8181015011092E853F85A1
:10A4D00002171307E4F1B60190E00F94039FDECF5B
:10A4E00016FD9FCFEF2DF0E0EA15FB0534F03CEFB1
:10A4F000A3163FEFB3060CF010683296E80DF91D75
:10A5000001C0FA94FF2019F082918033D1F317FF34
:10A5100088CF442443944F0CFA141B0431F02CF0E0
:10A52000FA187FCF442443947CCFF12C7ACFB60124
:10A5300080E290E00F94039FEA9490CFB60180E30D
:10A5400090E00F94039FEA9494CF80E3BDCFA016D0
:10A55000B10641F49A81963350F4953319F43C8551
:10A5600034FF05C0B60190E00F94039F2ACF81E32A
:10A57000F9CF8A81813319F09C859F7E9C87B60133
:10A5800090E00F94039FFF20A9F0B6018EE290E0C7
:10A590000F94039FF394F394E2E001E00E0FE80DB3
:10A5A000F92DF11D8081B60190E00F94039FE02FFB
:10A5B0000F11F3CF85E690E014FF02C085E490E030
:10A5C000B6010F94039FB7FC06C0A114B104C1F4F7
:10A5D000EC85E4FF15C0B194A194B1088DE2B601F9
:10A5E00090E00F94039F80E32AE0A216B10454F494
:10A5F000B60190E00F94039FB601C501C096B4CF99
:10A600008BE2EDCF8F5FFAE0AF1AB108EDCF833662
:10A61000C9F0833771F1833509F05BC03501F2E091
:10A620006F0E711CF501A080B1806F2D70E006FDEA
:10A6300002C06FEF7FEFC5010F94979E9D878C87B7
:10A6400000680DC0350132E0630E711CF501808198
:10A65000898321E030E03D872C8754010F7703FD8B
:10A6600006C02C853D855216130609F0A8F4E52C8A
:10A670002BC0350132E0630E711CF501A080B18062
:10A680006F2D70E006FD02C06FEF7FEFC5010F94E4
:10A69000BC9E9D878C87E2CFB60180E290E00F944C
:10A6A000039F5A94DECFF50107FD859107FF819145
:10A6B0005F01B60190E00F94039FE110EA948C854E
:10A6C0009D8501979D878C87EC85FD85EF2B59F73C
:10A6D00078CE843619F0893609F074C0350107FF49
:10A6E00066C0F4E06F0E711CF5016081718182819A
:10A6F0009381102F1F7697FF08C0909580957095D5
:10A7000061957F4F8F4F9F4F10682AE030E0A40182
:10A710000F942AA0A82EA818BA2C012F16FF0AC041
:10A720000E7FAF1438F414FF04C012FD02C0012FD5
:10A730000E7EBF2C04FFA3C0FE01EA0DF11D808137
:10A74000803309F095C0097EF02FF870EF2E03FDDD
:10A75000A5C000FF9FC0FA2CB51410F4F50CFB182F
:10A7600004FFA2C0B60180E390E00F94039F02FFB4
:10A7700009C088E790E001FF02C088E590E0B601DB
:10A780000F94039FAF1408F49BC0AA940A2D10E005
:10A790000F5F1F4F080D191DF80182918F01B6013F
:10A7A00090E00F94039F80169106B1F70ACEF2E075
:10A7B0006F0E711CF50160817181072E000C880BF2
:10A7C000990B97CF102F8537A9F41F7E2AE030E030
:10A7D000350117FF44C0F4E06F0E711CF501608174
:10A7E000718182819381A4010F942AA0A82EA818B8
:10A7F0001F7792CF197F8F3679F1F0F4883539F1D0
:10A80000F601868197812F960FB6F894DEBF0FBEB2
:10A81000CDBFDF91CF911F910F91FF90EF90DF900F
:10A82000CF90BF90AF909F908F907F906F905F90F0
:10A830004F903F902F900895803739F0883701F777
:10A8400014FD146020E130E0C3CF1061F9CF04FDA6
:10A85000166020E132E0BCCF28E030E0B9CFF2E072
:10A860006F0E711CF5016081718190E080E0BBCFBB
:10A8700002FD02C0B39468CFB394B39465CF802F28
:10A88000867809F461CFF6CFB60180E290E00F94AC
:10A89000039FB394B514C0F3E12C62CFE52CEB1801
:10A8A000B51408F45DCFF8CF802F867809F46ACF0D
:10A8B0008BE201FF80E207FD8DE2B60190E060CF00
:10A8C000B60180E390E00F94039FFA945BCFB6014A
:10A8D00080E290E00F94039FEA9473CD24E0E12C92
:10A8E000251508F036CD84E026CD20E030E040E8A4
:10A8F0005FEB60917E0270917F0280918002909167
:10A9000081020F94B8A2882321F1E091CB11F0913C
:10A91000CC11E252F04F80818B7F8230D1F480E104
:10A92000EEE7F2E0A5EFB1E101900D928A95E1F733
:10A9300080E090E0A0E8BFEB80937E0290937F02DE
:10A94000A0938002B09381028091E0119091E11177
:10A95000089581E090E0089580E1E3E9F6E0A5EF55
:10A96000B1E101900D928A95E1F70895E6E1F6E7ED
:10A97000833021F0E82FF0E0ED5EF94884910895EE
:10A980008091AF059091B0052091B1053091B2054D
:10A99000821B930B8F7799270895982F9F7083FFC1
:10A9A0000DC080917B00886080937B0080917C004B
:10A9B000887F9770892B80937C00089580917B001D
:10A9C000877FF2CF8091B1059091B2059093B00549
:10A9D0008093AF0581E399E69F938F938091D11186
:10A9E0009091D211A091D311B091D4110196A11DD3
:10A9F000B11DBF93AF939F938F938BE394E69F9387
:10AA00008F9382E494E69F938F930F945D9F8DB70D
:10AA10009EB70A960FB6F8949EBF0FBE8DBF0895DD
:10AA20000F931F93CF93DF93EC01C60FD71F8C17A3
:10AA30009D0779F08C010F5F1F4F0F949BA08F3FF4
:10AA400031F081E0DF91CF911F910F910895C801FE
:10AA5000EECF80E0F7CF682F880F770B8091CB1176
:10AA60009091CC118F51904F0F94F2A69C0190932E
:10AA7000F6168093F51681E0232B09F480E0089503
:10AA80008091F5169091F6164AE050E070E060E093
:10AA900001960F94269C862F08958091F51690912B
:10AAA000F6164AE050E070E060E001960F94269CB4
:10AAB000CB0108950F931F93CF93DF938C01862FC3
:10AAC000EA010E942B55882319F10E944D559C01E3
:10AAD00097FF03C0319521953109253631059CF04A
:10AAE0009F938F9384E49DE99F938F9383E996E7E7
:10AAF0009F938F930F945D9F0F900F900F900F90E7
:10AB00000F900F9080E0DF91CF911F910F910895EA
:10AB1000F80180818823B1F3CE01DF91CF911F919D
:10AB20000F910D949BA08091F5169091F6164AE036
:10AB300050E070E060E001960D94269C60E086E6AF
:10AB40009FE00F94BFA060E088E69FE00F94BFA055
:10AB500060E085E69FE00F94BFA060E084E69FE0A0
:10AB60000F94BFA060E082ED9EE00F94BFA060E074
:10AB70008FEC9EE00D94BFA080369105F8F44091D3
:10AB8000CB115091CC112091DC0F3091DD0F421789
:10AB9000530739F46091CF117091D0111616170632
:10ABA0006CF0B901680F791FFB01E359FF4F2417BF
:10ABB000350730F481E04E175F0708F480E0089510
:10ABC000EE3EF140F8F06C5F7F4F6E3E714018F43E
:10ABD00049365105B8F483599F4F4817590770F308
:10ABE0004DEE51E0421B530B70E060E0C901825210
:10ABF000904F0F94CDA68FB7F8941092DD0F10925E
:10AC0000DC0F8FBF81E008952F923F924F925F92A9
:10AC10006F927F928F929F92AF92BF92CF92DF926C
:10AC2000EF92FF920F931F93CF93DF93CDB7DEB7D1
:10AC3000CC58D2400FB6F894DEBF0FBECDBFCB5874
:10AC4000DD4F688379838A839B83C557D240FE0199
:10AC5000E754FE4F88E2DF011D928A95E9F7E85B31
:10AC6000F1401F0180E991E0DF01FC011D92319765
:10AC7000E9F7C75ADD4F19821882C955D2409E01A3
:10AC80002F513E4FC159DD4F39832883CF56D240D3
:10AC90008E01075A1D4FCE018F5C9D4FC359DD4F6A
:10ACA00099838883CD56D2403C01490140EBA42EC4
:10ACB0004FE0B42E53E2C52ED12CF12CE12CB6017D
:10ACC0000D2C000C880B990B0F94299BD4016D93CC
:10ACD0007D938D939D934D01F801619171918F0149
:10ACE000072E000C880B990B0F94299BD3016D93B1
:10ACF0007D938D939D933D01BFEFEB1AFB0AE6E038
:10AD0000EE16F10409F038C3CB58DD4F28813981A4
:10AD10004A815B81C557D240C159DD4FA881B981B5
:10AD2000CF56D2406D917D918D919C910F944CA402
:10AD3000412C512C320118160CF402C3C359DD4FBB
:10AD400008811981CD56D2400C5E1F4FC159DD4F8D
:10AD5000E880F980CF56D240B4E1EB0EF11C6E01D1
:10AD6000EFEDCE1AEDEFDE0A9E012B553E4FCF5888
:10AD7000DD4F39832883C157D240D8014D905D9073
:10AD80006D907C90F7016081718182819381D70100
:10AD90005E914E913E912E917D010F94C2A14B0187
:10ADA0005C01F80152914291329122918F01C301CD
:10ADB000B2010F94C2A1A50194010F94C2A2D601C1
:10ADC0009E938E937E936E936D01CF58DD4FE881F5
:10ADD000F981C157D240B292A29292928292CF58F8
:10ADE000DD4FF983E883C157D240C359DD4F288135
:10ADF0003981CD56D2400217130709F0BECF4E015C
:10AE00003FE6831A3EEF930A5E0183EFA81A8DEFA7
:10AE1000B80A61018101EE24E394F12CD4014D9034
:10AE20005D906D907D904D012D913D914D915C9186
:10AE3000C301B2010F94C3A19B01AC010F94C3A144
:10AE4000F80164A775A786A797A7F1E0EF16F104AC
:10AE500061F0D80198964D925D926D927C929B978D
:10AE6000F8014482558266827782FFEFEF1AFF0A6B
:10AE7000F501208131814281538184E0A80EB11C0B
:10AE800064817581868197810F94C2A120E030E0B2
:10AE900040EC50E40F94689BD601DC966D937D9353
:10AEA0008D939C93DF97045D1F4FB8E2CB0ED11CAE
:10AEB000E5E0EE16F10409F0B1CF7E01FDE2EF0E00
:10AEC000F11C28E2A22EB12C00EB1FEF24E0220E91
:10AED000311CD7012D913D914D915C91139798961E
:10AEE0006D917D918D919C919B970F94C2A22B01A6
:10AEF0003C016101C01AD10A88248394912CF60187
:10AF0000E00FF11FEA0DFB1D208131814281538149
:10AF1000C301B2010F94689B9B01AC01F6016081F3
:10AF20007181828193810F94C2A1D6016D937D932B
:10AF30008D939D936D01BFEF8B1A9B0AE6E08E16F1
:10AF40009104E9F63CE2E30EF11C0852110988E293
:10AF5000A80EB11C08339FEF190709F0BACF1E01E4
:10AF6000F5EB2F0E311C6E0121EBC20ED11C7E01C0
:10AF700037E3E31A3EEFF30A04E010E04801B12C96
:10AF8000A12C412C512C3201F601EA0DFB1DD701F9
:10AF9000AA0DBB1D2D913D914D915C9160817181F8
:10AFA000828193810F94689B9B01AC01C301B20124
:10AFB0000F94C3A12B013C018FEF881A980A94E0EB
:10AFC000A90EB11CA5E08A169104F1F6A301920125
:10AFD000F10160817181828193810F94C2A1D601B8
:10AFE0002D913D914D915C910F94C2A2F701608328
:10AFF00071838283938301501109F8E22F1A31087B
:10B000002CE2C21AD10834E0E31AF1080115110547
:10B0100009F0B4CFCB50DE4F88819981AA81BB81E2
:10B02000C55FD140CF57DD4F88839983AA83BB8307
:10B03000C158D2401E0197E4291A9EEF390A10E048
:10B0400000E0C159DD4FA881B981CF56D240CD90E3
:10B05000DD90ED90FD90C159DD4FB983A883CF56A7
:10B06000D240CB58DD4F288139814A815B81C55759
:10B07000D240C701B6010F94B8A21816B4F0CB584D
:10B08000DD4F288139814A815B81C557D240C15942
:10B09000DD4FE881F981CF56D24060817181828194
:10B0A00093810F944CA487FF18C00430110509F058
:10B0B00030C1CB58DD4F288139814A815B81C5572A
:10B0C000D240CF57DD4F688179818A819B81C158F9
:10B0D000D2400F94B8A287FF1CC1D10114968D9065
:10B0E0009D90AD90BC9017978D919D910D90BC91C6
:10B0F000A02DCF58DD4F88839983AA83BB83C15786
:10B10000D240F801EE0FFF1FEE0FFF1F21E931E0E3
:10B110002C0F3D1FE20FF31F40805180628073802F
:10B12000C359DD4FA881B981CD56D2408D919D91F3
:10B130000D90BC91A02DC358DD4F88839983AA83BD
:10B14000BB83CD57D240A7019601CB58DD4F688114
:10B1500079818A819B81C557D2400F94C2A16B012E
:10B160007C0120E030E040E450E40F9433A5CB575D
:10B17000DD4F688379838A839B83C558D240C35847
:10B18000DD4F288139814A815B81CD57D240C35937
:10B19000DD4FE881F981CD56D24064817581868189
:10B1A00097810F94C2A1A30192010F94C2A2C75824
:10B1B000DD4F688379838A839B83C957D240A3017B
:10B1C0009201C301B2010F94C3A1CF58DD4F288172
:10B1D00039814A815B81C157D2400F94689BC75720
:10B1E000DD4F688379838A839B83C958D240A3014A
:10B1F0009201C501B4010F94689B9B01AC01C75734
:10B20000DD4F688179818A819B81C958D2400F9432
:10B21000C3A120E030E040EC50E40F94C2A29B01B7
:10B22000AC01C758DD4F688179818A819B81C957FC
:10B23000D2400F94C2A1A70196010F94689BC758F2
:10B24000DD4F688379838A839B83C957D240CF5867
:10B25000DD4F288139814A815B81C157D240C501C8
:10B26000B4010F94C2A14B015C0120E030E040EC3E
:10B2700050E4C301B2010F94689B9B01AC01C5016E
:10B28000B4010F94C2A2CB57DD4F288139814A8186
:10B290005B81C558D2400F94689B4B015C0120E054
:10B2A00030E040E05FE3CF58DD4F688179818A81EB
:10B2B0009B81C157D2400F94689B2B013C01A70191
:10B2C0009601C701B6010F94689B9B01AC01C301B5
:10B2D000B2010F94689B9B01AC01C501B4010F94AE
:10B2E000C3A19B01AC01C758DD4F688179818A8178
:10B2F0009B81C957D2400F94C3A1C358DD4F288109
:10B3000039814A815B81CD57D2400F94C3A12B0173
:10B310003C010F5F1F4FF4E02F0E311CC359DD4F6E
:10B3200028813981CD56D2402C5F3F4FC359DD4F24
:10B3300039832883CD56D2400530110509F081CEDE
:10B34000C301B201C457DD4F0FB6F894DEBF0FBE84
:10B35000CDBFDF91CF911F910F91FF90EF90DF90C4
:10B36000CF90BF90AF909F908F907F906F905F90A5
:10B370004F903F902F900895C5010F94A9A0D80138
:10B380008D939C93B5E0CB0ED11CE2E0AE0EB11CC8
:10B3900096CC0F931F93CF9320919412213079F57F
:10B3A0008C0180E50E942B55882349F10E9440556D
:10B3B000C82F853020F5013C82E0180749F0023C97
:10B3C000124069F08C2FCF911F910F910D946A6BF1
:10B3D00060E08C2FCF911F910F910D94AD6B8EEC8F
:10B3E0009EE00F949BA0882351F00F947354882300
:10B3F00031F08C2FCF911F910F910D942A6CCF912A
:10B400001F910F9108958F929F92AF92BF92CF920A
:10B41000DF92EF92FF920F931F93CF93DF930091F0
:10B42000F5161091F6160F5F1F4F68018FEFC81ABF
:10B43000D80AD801DC918D2F90E00F942C9E7C01CE
:10B44000892B01F5DD3201F56801B2E0CB0ED11C8C
:10B45000F801D181C1E086010150110943E050E0BB
:10B460006AE476E7C8010F94629E892BC1F460E01C
:10B4700070E080E89FEFC111DBC060E070E080E821
:10B480009FE7D6C08601D1CFDB3239F46801F2E004
:10B49000CF0ED11CD8011196DC91C0E0DCCF43E087
:10B4A00050E067E476E7C8010F94629E892B09F4A7
:10B4B000CCC0F60110E000E020E030E0A9016F010F
:10B4C000D053DA3060F5BC2E6894B1F88C2F8870B8
:10B4D000C2FF09C0811102C00F5F1F4F3196D60114
:10B4E000DC91CB2DECCF882311F001501109A5E0A0
:10B4F000B0E00F9430A19B01AC01220F331F441F19
:10B50000551F2D0F311D411D511D2839B9E93B072C
:10B510004B07B9E15B0710F3C660BC2EDFCFDE3FFF
:10B5200031F4C3FD33C0BC2E6894B3F8D7CFD53304
:10B5300069F580818D3231F4C061BF016E5F7F4F4C
:10B54000818105C0BF018B32C9F36F5F7F4F80538C
:10B550008A30E0F4FB01B0E8EB16BCE0FB065CF4DB
:10B56000B701660F771F660F771FE60EF71EEE0C0A
:10B57000FF1CE80EF11C819180538A3060F3C4FFF8
:10B5800003C0F194E194F1080E0D1F1DCA01B90129
:10B590000F94279BC370C33009F490584B015C0192
:10B5A00020E030E0A9010F94B8A2882309F43EC03E
:10B5B000C3E4D6E717FF05C0119501951109CBE249
:10B5C000D6E76E01E8E1CE1AD10880E2E82EF12C30
:10B5D0000DC0FE0125913591459154910E191F0919
:10B5E000C501B4010F94689B4B015C01D501C401F6
:10B5F0000E151F0574F72497F594E794CC16DD0615
:10B60000A9F78A2F880F8B2F881F8F3F49F020E0E2
:10B6100030E0A901C501B4010F94B8A2811106C0A0
:10B6200082E290E09093F9168093F816C501B40178
:10B63000DF91CF911F910F91FF90EF90DF90CF900E
:10B64000BF90AF909F908F90089560E070E080EC85
:10B650009FE7EECF2F923F924F925F926F927F9231
:10B660008F929F92AF92BF92CF92DF92EF92FF9212
:10B670000F931F93CF93DF93CDB7DEB7A1970FB68C
:10B68000F894DEBF0FBECDBF84EC92E09D8F8C8F0F
:10B6900085EF282E81E1382E03E916E091E09A8F9C
:10B6A000198EEC8DFD8D8191FD8FEC8F0E942B55B5
:10B6B000E82E882309F454C1F090EB11FA8DFF2293
:10B6C0000E94035A2B013C01F801408251826282A0
:10B6D0007382F98DF33009F045C0DD24D394F11065
:10B6E00001C0D12C8090100290901102A090120203
:10B6F000B090130220E030E040E85FE3C501B40100
:10B700000F94B8A2882359F1F11015C020910112AD
:10B71000309102124091031250910412C301B20100
:10B720000F94C2A160939F067093A0068093A10618
:10B730009093A206DE2CA501940160919F06709162
:10B74000A0068091A1069091A2060F94689B609339
:10B750009F067093A0068093A1069093A206D11035
:10B7600003C05FC0FF2089F0F10120813181428157
:10B770005381F80160817181828193810F94C3A10B
:10B78000F8016083718382839383F98DF230D9F558
:10B7900080918903823009F0EEC08CE0E0EAF2E0AB
:10B7A000DE011D9601900D928A95E1F78CE0ECEA9E
:10B7B000F2E0DE01119601900D928A95E1F7C090BA
:10B7C0009B06D0909C06E0909D06F0909E0620E09F
:10B7D00030E0A901C701B6010F94B8A287FF52C09B
:10B7E000CE0101967C01D12CF7016191719181917B
:10B7F00091917F010F9434A38D2D0F941B22D3942C
:10B80000F3E0DF12F1CFF98DFF5FF98F8A8D880F9A
:10B810008A8F94E0290E311C0C5F1F4FF43009F021
:10B8200040CF86E40E942B55882399F00E94035A4A
:10B830006B017C0120E030E0A9010F944CA41816A4
:10B8400044F4C0927A02D0927B02E0927C02F092A1
:10B850007D02A1960FB6F894DEBF0FBECDBFDF917B
:10B86000CF911F910F91FF90EF90DF90CF90BF90FD
:10B87000AF909F908F907F906F905F904F903F9090
:10B880002F90089520E030E048E453E4C701B6016A
:10B890000F944CA41816A4F4CE010D967C01D12C63
:10B8A000F70161917191819191917F010F9434A37E
:10B8B0008D2D0F941B22D394F3E0DF12F1CFA3CF91
:10B8C000CE01019699A388A3FE013D96FF8FEE8FCE
:10B8D0001B8EE8A1F9A1C190D190E190F190F9A35C
:10B8E000E8A3EE8DFF8D6191719181919191FF8F10
:10B8F000EE8FA70196010F94C2A120E030E048E44A
:10B9000053E40F94C2A24B015C0120919B0630913D
:10B910009C0640919D0650919E060F94689B2B01BA
:10B920003C0120E030E0A901C501B4010F94689BFF
:10B930009B01AC01C701B6010F94C2A19B01AC01F0
:10B94000C301B2010F94C3A10F9434A38B8D0F9444
:10B950001B22FB8DFF5FFB8FF33009F0BACF53CF73
:10B96000F10180819181A281B381F801808391836B
:10B97000A283B38348CFEA8DEE0FEA8FF4E02F0E57
:10B98000311C0C5F1F4F83E0898F8BCE60910017B5
:10B990007091011790E08A3020F0895A9F4F0D94E2
:10B9A000039FC096FCCF84FF18C05A9A85FF17C02A
:10B9B000A49A2FB786FF15C0F89490910201906861
:10B9C000909302012FBF87FF11C0A39A5B9A85E075
:10B9D0008A95F1F700005B9808955A98E7CFA498EC
:10B9E000E8CFF894909102019F77EACFA398EECF29
:10B9F0000F931F93CF93DF93C82FD62F8A0160FF39
:10BA000015C05D9A8AE18A95F1F700C08C2F0E94DB
:10BA1000D35CD1FD04C08C2F82950E94D35CC801F9
:10BA2000DF91CF911F910F910C94DBBF5D98EACF0E
:10BA3000CF92DF92EF92FF92CF93DF93EC016A01F6
:10BA40007B010F94A3A06F3F7F4F8F4F9F4F59F4FF
:10BA5000B701A601CE01DF91CF91FF90EF90DF906B
:10BA6000CF900D94F1A0DF91CF91FF90EF90DF90F8
:10BA7000CF9008957F928F929F92AF92BF92CF9274
:10BA8000DF92EF92FF920F931F93CF93DF93CDB787
:10BA9000DEB760970FB6F894DEBF0FBECDBF5C0176
:10BAA0006B01742E81E0809378021F930F931F9295
:10BAB0002F938DE793E69F938F930F945D9F81E47F
:10BAC0000E942B550F900F900F900F900F900F909A
:10BAD000882389F08091F5169091F616FC0121815A
:10BAE000283709F056C040E150E070E060E002966F
:10BAF0000F94269C5B0183E40E942B55882309F454
:10BB00004DC00E9493554B017501CA14DB0408F423
:10BB10007601C4018E0D9F1DC816D90618F08E152A
:10BB20009F0518F446018E189F0888E50E942B5542
:10BB3000882309F471C02091F5163091F6162F5F15
:10BB40003F4FCE0101965C01DC01D12CC12CF901E3
:10BB500080812F5F3F4F8823B9F190E1C916D1044E
:10BB600099F18032A1F38A3079F190ED980F9A30F3
:10BB7000C8F48295807F9F012E5F3F4F918140EDF9
:10BB8000490F4A30B8F4842B8D93EFEFCE1ADE0ABA
:10BB9000DECF0E94035A0F9434A3ACCF88248A943A
:10BBA000982CB2CF9FE9980F963058F48295807FF9
:10BBB0008057E1CF4FE9490F463018F49755892B4C
:10BBC000E3CFD194C194D108912C812CC814D9040D
:10BBD00091F0F50161915F01C4018E0D9F1DF1E0AF
:10BBE0007F1631F0FC016083FFEF8F1A9F0AEECFC2
:10BBF0000F94E3A0F9CFFF92EF921F930F939F92C0
:10BC00008F9283E593E69F938F930F945D9F0FB67A
:10BC1000F894DEBF0FBECDBF472DB401C7016096BB
:10BC20000FB6F894DEBF0FBECDBFDF91CF911F914D
:10BC30000F91FF90EF90DF90CF90BF90AF909F90CB
:10BC40008F907F900D94A45380E1E5EFF1E1A0E99E
:10BC5000B2E001900D928A95E1F780918E02909169
:10BC60008F029093F4118093F3118091F1119091D0
:10BC7000F2119093F0118093EF118091ED11809368
:10BC8000EC118091EB1183FB882780F98093EA11F6
:10BC90008091E9118093E8110895CF93DF938AEFA3
:10BCA00095E10E94317088E394E1892B51F0CAE05C
:10BCB000D5E1A397CE010E94317084E1C833D80743
:10BCC000C1F785E194E10E94317080EF93E1DF914B
:10BCD000CF910C943170CF93DF93C5EFD1E120E089
:10BCE00030E048EC51E46C857D858E859F850F940E
:10BCF000C3A16C877D878E879F8763E373E383E5AA
:10BD000090E4DF91CF910D942F8560E085EA9FE06C
:10BD10000F94BFA060E08FE79CE00F94BFA080E08D
:10BD200090E0A0E8BFEB80937E0290937F02A09307
:10BD30008002B093810282E0809379021092E71131
:10BD400008958091EF119091F0112091F1113091AF
:10BD5000F2112817390771F09093F2118093F111C5
:10BD600081E0809399030F94FC0F0F94574F82E06A
:10BD70008093990308958091E711882341F0809181
:10BD80008E0290918F029093F4118093F311089595
:10BD9000CF92DF92EF92FF92C090CA04D090CB0472
:10BDA000E090CC04F090CD048091C904882309F47C
:10BDB0004EC020E030E0A901C701B6010F944CA4A9
:10BDC00018160CF044C02BED3FE049E450E4C701E5
:10BDD000B6010F94689BA70196010F94689B20E021
:10BDE00030E040E85EE30F94689B9B01AC0160E0AB
:10BDF00070E080E89FE30F94C2A26B017C01609128
:10BE0000590270915A0264367105A1F0072E000C98
:10BE1000880B990B0F94299B2AE037ED43E25CE3F2
:10BE20000F94689B9B01AC01C701B6010F94689BFE
:10BE30006B017C01C0921002D0921102E0921202BA
:10BE4000F0921302FF90EF90DF90CF900895C12CF5
:10BE5000D12C80E8E82E8FE3F82ED1CF8F929F92DD
:10BE6000AF92BF92CF92DF92EF92FF9281EF9FE06D
:10BE70000F9476496B017C018DEE9FE00F9476491B
:10BE80004B015C010F94F21C2CE330E040E050E0E9
:10BE90000F940EA1BA01A901480D591D6A1D7B1D01
:10BEA0008DEE9FE00F94D1A060918406709185067D
:10BEB000809186069091870628EE33E040E050E0BE
:10BEC0000F940EA1BA01A9014C0D5D1D6E1D7F1DC1
:10BED00081EF9FE00F94D1A00F94C72010928406A9
:10BEE0001092850610928606109287068091941211
:10BEF000813081F4609198127091991290E080E005
:10BF00000F945E49109299121092981210929B12FF
:10BF100010929A12FF90EF90DF90CF90BF90AF9069
:10BF20009F908F9008958091E9111F928F93809137
:10BF300040031F928F93E5E8F3E0428153812CE3A5
:10BF4000249FC001259F900D11249F938F934081C2
:10BF50005181249FC001259F900D11249F938F93A1
:10BF600084E194E69F938F930F945D9F8DB79EB766
:10BF70000A960FB6F8949EBF0FBE8DBF08958AE44F
:10BF800093E00D94291220E030E040E752E40F9452
:10BF9000C2A208951092770240913B0350913C0356
:10BFA00060913D0370913E0340937A0250937B026F
:10BFB00060937C0270937D0290938F0280938E0237
:10BFC0008AE493E00D9429121F93CF93DF93182FE7
:10BFD00080917A0290917B02A0917C02B0917D02C7
:10BFE00080933B0390933C03A0933D03B0933E03A7
:10BFF000C0918E02D0918F0284E690E090938F02E0
:10C0000080938E028AE493E00F94291210937702B2
:10C01000CE01DF91CF911F910895CF92DF92EF92E1
:10C02000FF920F931F93CF93DF9390E0EC01CC0F1F
:10C03000DD1FCC0FDD1FFE01EB59F948259135912D
:10C0400045915491FE01E657FB4FC080D180E280BC
:10C05000F3808E010B501E4EC701B6010F94C3A191
:10C06000F8016083718382839383FE01E75AF94864
:10C0700025913591459154918E010C5D1D4FC7015D
:10C08000B6010F94C3A1F801608371838283938307
:10C09000FE01E35BF9482591359145915491C85EC5
:10C0A000DD4FC701B6010F94C3A1688379838A83EA
:10C0B0009B83DF91CF911F910F91FF90EF90DF90C5
:10C0C000CF90089540E050E0BA018DEE9FE00F94CC
:10C0D000D1A040E050E0BA0181EF9FE00F94D1A0E1
:10C0E0000E949E5570E060E085E09FE00F94DDA027
:10C0F00070E060E083E09FE00F94DDA070E060E01E
:10C1000081E09FE00F94DDA070E060E08FEF9EE0A3
:10C110000F94DDA070E060E083ED9EE00F94DDA061
:10C1200070E060E080ED9EE00F94DDA040E050E024
:10C13000BA0188EA9CE00D94D1A0F89488E19FE0D0
:10C140000FB6F894A895809360000FBE909360009E
:10C15000FFCF85EA9FE00F949BA091E0811101C081
:10C1600090E0892F089580919B03811106C081E0A2
:10C1700090915903923009F080E0089580916A13FC
:10C1800081110AC08091D511811106C081E0909182
:10C190005903913009F080E00895CF93DF93C09167
:10C1A0000512C1111FC08091061281111CC00E948E
:10C1B000B360811118C0D091C80DD43061F4809162
:10C1C000F1119091F211892B91F48091ED119091E0
:10C1D000EE11892B61F40E94BE60C82F811103C04B
:10C1E000C1E0D111C0E08C2FDF91CF910895C1E063
:10C1F000FACF0E94CD60882389F020E030E040E053
:10C2000050E46091FD117091FE118091FF119091A9
:10C2100000120F94B8A2881F8827881F08950E94D3
:10C22000BE60811118C00E94B360811114C080915A
:10C23000E711811110C08091C80D81110BC0809150
:10C240009512811107C080910512811104C080915F
:10C250000612089581E0089580E1E5EFF1E1A3E998
:10C26000B6E001900D928A95E1F708954F925F92A2
:10C270006F927F928F929F92AF92BF92CF92DF92F6
:10C28000EF92FF920F931F93CF93DF9300D000D0D4
:10C290001F921F92CDB7DEB72091E711222309F438
:10C2A00073C120919C03223009F46EC120919C033C
:10C2B000213011F410929C032B013C011092E911E2
:10C2C0001091EC1160918A0370918B0380918C0323
:10C2D00090918D030F943BA3611731F0812F90E073
:10C2E0009093EE118093ED110E94A15E8091E81170
:10C2F0008093E9119091EB118091EA118195892742
:10C30000887089278093EB11A301920160919C02B0
:10C3100070919D0280919E0290919F020F94C2A104
:10C320006D837E838F839887CE0105960F948775E2
:10C330001092400220E030E040E85FEB6091900214
:10C340007091910280919202909193020F94B8A201
:10C35000811120C08091F5119091F611A091F711F3
:10C36000B091F8118093900290939102A093920261
:10C37000B09393028091F9119091FA11A091FB1161
:10C38000B091FC118093940290939502A093960231
:10C39000B0939702A301920160919C0270919D025B
:10C3A00080919E0290919F020F94C2A169837A832B
:10C3B0008B839C83E090FD11F090FE110091FF11A2
:10C3C00010910012209194023091950240919602B2
:10C3D0005091970260919002709191028091920227
:10C3E000909193021F921F921F921F92E2E68E2E4F
:10C3F000E7E29E2EE6E7AE2EE2E4BE2EFE01319687
:10C400006F010F94E175A301920160919C027091FC
:10C410009D0280919E0290919F020F94C2A1698318
:10C420007A838B839C83E0909802F090990200912C
:10C430009A0210919B0220919402309195024091B2
:10C4400096025091970260919002709191028091B2
:10C450009202909193021F921F921F921F920F942B
:10C46000E175E0909802F090990200919A02109183
:10C470009B02209194023091950240919602509136
:10C480009702609190027091910280919202909136
:10C4900093021F921F921F921F92812C912CF8EEF3
:10C4A000AF2EF2E4BF2EACE9CA2EA2E0DA2E0F9432
:10C4B000E1750F94CE2211E0109340026091E211D9
:10C4C0007091E31190E080E00F94279B60937A02D3
:10C4D00070937B0280937C0290937D028091F31194
:10C4E0009091F41190938F0280938E0280E1E0E9A5
:10C4F000F2E0A5EFB1E101900D928A95E1F70E947B
:10C500002C61809179020FB6F894DEBF0FBECDBFCB
:10C51000811151C06091D8117091D9118091DA11B7
:10C520009091DB1160937E1670937F168093801636
:10C53000909381160F94B5448091D8119091D911A0
:10C54000A091DA11B091DB118093DC119093DD1191
:10C55000A093DE11B093DF1110936A1360E085EAB7
:10C560009FE00F94BFA060E08FE79CE00F94BFA016
:10C5700087E69BE60E9499E682E08093790210921A
:10C58000E71181E08093AC0D28960FB6F894DEBFDA
:10C590000FBECDBFDF91CF911F910F91FF90EF9014
:10C5A000DF90CF90BF90AF909F908F907F906F90D3
:10C5B0005F904F900895813089F68091D8119091C5
:10C5C000D911A091DA11B091DB118093D111909320
:10C5D000D211A093D311B093D4111092DB0F10920B
:10C5E000DA0F0E94E254BACF3F924F925F926F925D
:10C5F0007F928F929F92AF92BF92CF92DF92EF92F3
:10C60000FF920F931F93CF93DF933090DC1633206C
:10C6100009F480C08B01EC0131FE54C08880998000
:10C62000AA80BB80FB01C080D180E280F380209192
:10C63000B1163091B2164091B3165091B416C5019F
:10C64000B4010F94689B2B013C012091B5163091E9
:10C65000B6164091B7165091B816C701B6010F949F
:10C66000689B9B01AC01C301B2010F94C3A12B01D4
:10C670003C012091A9163091AA164091AB16509119
:10C68000AC16C501B4010F94689B4B015C0120916D
:10C69000AD163091AE164091AF165091B016C7014D
:10C6A000B6010F94689B9B01AC01C501B4010F94C6
:10C6B000C3A1688379838A839B83F8014082518276
:10C6C0006282738230FE26C02091D4163091D51636
:10C6D0004091D6165091D716688179818A819B81C5
:10C6E0000F94C3A1688379838A839B832091D81692
:10C6F0003091D9164091DA165091DB16F80160811D
:10C700007181828193810F94C3A1F8016083718349
:10C7100082839383DF91CF911F910F91FF90EF90D0
:10C72000DF90CF90BF90AF909F908F907F906F9051
:10C730005F904F903F9008952F923F924F925F925B
:10C740006F927F928F929F92AF92BF92CF92DF9221
:10C75000EF92FF920F931F93CF93DF9300D000D0FF
:10C760001F921F92CDB7DEB78C011B01FC018081A7
:10C770009181A281B38189839A83AB83BC83FB01BE
:10C7800080819181A281B3818D839E83AF83B8879D
:10C79000BE016B5F7F4FCE0101960E94F462C9809B
:10C7A000DA80EB80FC8020E030E0A901C701B6010F
:10C7B0000F94B8A287FF35C019821A821B821C828F
:10C7C000FF24F3948D809E80AF80B88420E030E019
:10C7D00040E850ECC501B4010F94B8A287FF35C002
:10C7E00080E090E0A0E8B0EC8D839E83AF83B887B3
:10C7F000CD80DE80EF80F88489809A80AB80BC8019
:10C800007090DC1671104CC0F80180829182A28277
:10C81000B382F101C082D182E282F382FF24F394D9
:10C8200025C020E030E04AE753E4C701B6010F9489
:10C830004CA4F12C181634F680E090E0AAE7B3E49B
:10C8400089839A83AB83BC83BBCF20E030E042E591
:10C8500053E4C501B4010F944CA418162CF480E0E5
:10C8600090E0A2E5B3E4C0CFF110C2CF8F2D28969F
:10C870000FB6F894DEBF0FBECDBFDF91CF911F91F1
:10C880000F91FF90EF90DF90CF90BF90AF909F906F
:10C890008F907F906F905F904F903F902F90089572
:10C8A00070FE1CC02091D4163091D5164091D6163A
:10C8B0005091D716C501B4010F94C2A14B015C0180
:10C8C0002091D8163091D9164091DA165091DB1686
:10C8D000C701B6010F94C2A16B017C0171FE9ECF0E
:10C8E0002091C4163091C5164091C6165091C716B6
:10C8F000C501B4010F94689B2B013C012091C8161F
:10C900003091C9164091CA165091CB16C701B60195
:10C910000F94689B9B01AC01C301B2010F94C3A1AA
:10C92000F80160837183828393832091CC163091C8
:10C93000CD164091CE165091CF16C501B4010F947B
:10C94000689B4B015C012091D0163091D11640912B
:10C95000D2165091D316C701B6010F94689B9B0164
:10C96000AC01C501B4010F94C3A1F10160837183CF
:10C970008283938353CFCF92DF92EF92FF92CF9334
:10C98000DF93EC01BC016C5F7F4F0E949C63C09001
:10C990002C02D0902D02E0902E02F0902F02A701E1
:10C9A0009601688579858A859B850F94B8A287FF53
:10C9B00004C0C886D986EA86FB86C0902002D09043
:10C9C0002102E0902202F0902302A70196016885DF
:10C9D00079858A859B850F944CA4181624F4C88603
:10C9E000D986EA86FB86DF91CF91FF90EF90DF90AA
:10C9F000CF9008952F923F924F925F926F927F92C5
:10CA00008F929F92AF92BF92CF92DF92EF92FF925E
:10CA10000F931F93CF93DF93CDB7DEB7A2970FB6D7
:10CA2000F894DEBF0FBECDBF1C0183E996E00E94E3
:10CA3000BB648AE493E00F9429124090F511509062
:10CA4000F6116090F7117090F811C0909306D09095
:10CA50009406E0909506F0909606A7019601C30112
:10CA6000B2010F94B8A281113FC020919706309176
:10CA700098064091990650919A066091F91170912B
:10CA8000FA118091FB119091FC110F94B8A28111C1
:10CA90002BC020E030E040E752E460917A027091D0
:10CAA0007B0280917C0290917D020F94C2A20F9430
:10CAB000FC840E94AC54A2960FB6F894DEBF0FBE61
:10CAC000CDBFDF91CF911F910F91FF90EF90DF903D
:10CAD000CF90BF90AF909F908F907F906F905F901E
:10CAE0004F903F902F90089560918E0270918F0229
:10CAF000072E000C880B990B0F94299B20917A022A
:10CB000030917B0240917C0250917D020F94689B92
:10CB10002EE333EC4EE259E30F94689B6F837887E2
:10CB200089879A8780919C12882309F40FC1A301F9
:10CB30009201C701B6010F94C2A12B013C012091C3
:10CB4000F9113091FA114091FB115091FC11609153
:10CB50009706709198068091990690919A060F9485
:10CB6000C2A16B877C878D879E87C301B2019F77A7
:10CB70002B853C854D855E855F770F94C3A16B0146
:10CB80007C0120E030E0A9010F944CA418160CF0B1
:10CB9000DDC020E030E040EF51E4C701B6010F9462
:10CBA000C2A20F94A1A20F943BA37E836D83623037
:10CBB000710508F4CBC02114310409F4C7C02091D9
:10CBC000FD113091FE114091FF11509100126091C2
:10CBD0009B0670919C0680919D0690919E060F94F5
:10CBE000C2A16F87788B898B9A8B2091011230912B
:10CBF0000212409103125091041260919F067091AD
:10CC0000A0068091A1069091A2060F94C2A16B8B01
:10CC10007C8B8D8B9E8BAD81BE81CD01B0E0A0E081
:10CC20008F8F98A3A9A3BAA32D813E812216330624
:10CC300008F08CC0B10190E080E00F94279B6B015D
:10CC40007C016F8D78A189A19AA10F94279B9B01EC
:10CC5000AC01C701B6010F94C2A26B017C01AC010B
:10CC60009B016B897C898D899E890F94689B9B01B0
:10CC7000AC016091011270910212809103129091A7
:10CC800004120F94C3A169837A838B839C83A701C9
:10CC900096016F85788989899A890F94689B20917C
:10CCA000FD113091FE114091FF11509100120F942F
:10CCB000C3A16F8B788F898F9A8FA70196016B859F
:10CCC0007C858D859E850F94689B2091F91130910C
:10CCD000FA114091FB115091FC110F94C3A16B8F7D
:10CCE0007C8F8D8F9E8FA7019601C301B2010F9497
:10CCF000689B2091F5113091F6114091F7115091F8
:10CD0000F8110F94C3A13F922F92A5EFB1E1BF9309
:10CD1000AF938F809884A984BA84DE0111966D0147
:10CD2000EF88F88C098D1A8D2B8D3C8D4D8D5E8D85
:10CD30000F94E1750F900F900F900F908091AC0DB4
:10CD40008111B7CEBFEF2B1A3B0A6ECFE0909B0646
:10CD5000F0909C0600919D0610919E0620919706EA
:10CD6000309198064091990650919A0660919306E9
:10CD70007091940680919506909196061F921F924D
:10CD8000E5EFF1E1FF93EF938F809884A984BA8453
:10CD9000EFE9CE2EE6E0DE2E0F94E1750F900F90B6
:10CDA0000F900F9086CECF92DF92EF92FF92CF93AB
:10CDB000C090FD11D090FE11E090FF11F090001294
:10CDC000A70196010F94C3A16093FD117093FE110A
:10CDD0008093FF119093001283B19091A506911159
:10CDE00002C084FF26C085EF91E10E94BB64609180
:10CDF0004E0470914F0480915004909151040F940F
:10CE00002F850F94CE22A70196016091FD1170919C
:10CE1000FE118091FF11909100120F94C2A16B013D
:10CE20007C01C701B601CF91FF90EF90DF90CF90CA
:10CE3000089515980F94CE2281E00F94062DC82FE7
:10CE400065E575E585E591E40F942F850F94CE2275
:10CE500082E00F94BA22A70196010F94C2A16B0140
:10CE60007C018C2F0F94062DDCCF8F929F92AF9276
:10CE7000BF92CF92DF92EF92FF924B015C01C09084
:10CE8000FD11D090FE11E090FF11F0900012AC0166
:10CE90009B01C701B6010F944CA487FF11C0A501E7
:10CEA0009401C701B6010F94C2A19F77FF90EF9044
:10CEB000DF90CF90BF90AF909F908F900C94D366EF
:10CEC000FF90EF90DF90CF90BF90AF909F908F90AA
:10CED00008952F923F924F925F926F927F928F921E
:10CEE0009F92AF92BF92CF92DF92EF92FF920F93F9
:10CEF0001F93CF93DF9300D01F921F92CDB7DEB761
:10CF0000D82E2A013B01322EE982FA820B831C8340
:10CF10000F94CE2281E080930512FC2CE32CD310D9
:10CF200010C0ED2CDC100DC060E070E080EA90E4F1
:10CF30000E943567FF24F394EE24E3942224239483
:10CF400001C02D2C0F941B9080919C128D83109208
:10CF50009C1282E00F94BA226093FD117093FE112F
:10CF60008093FF1190930012F1100F94CA8B81E00F
:10CF70000E94E45F8C010E942C6110927A02109250
:10CF80007B0210927C0210927D02222019F080E038
:10CF90000F947B54EE2019F081E00F947B54DD2038
:10CFA000E9F04114510461047104C1F0C301B201FC
:10CFB0000F94299B9B01AC0160918A0470918B04B2
:10CFC00080918C0490918D040F94C3A16093F5110E
:10CFD0007093F6118093F7119093F811332001F1BB
:10CFE00089819A81AB81BC810097A105B105C1F00F
:10CFF000BC01CD010F94299B9B01AC0160918E0473
:10D0000070918F0480919004909191040F94C3A12A
:10D010006093F9117093FA118093FB119093FC11B6
:10D02000FF2009F499C060E070E080EA90E40E947B
:10D0300035678091A306811102C00F947B548091C3
:10D04000A406811103C081E00F947B540F9480905B
:10D05000E0E5F8E885919591A591B491ECE4F8E8C4
:10D060004591559165917491409393065093940620
:10D070006093950670939606809397069093980612
:10D08000A0939906B0939A0667E976E083E996E063
:10D090000E94F4620F94E28F20E030E040E850EC10
:10D0A00060919706709198068091990690919A06E2
:10D0B0000F94B8A287FF0CC080E090E0A0E8B0EC2D
:10D0C0008093970690939806A0939906B0939A063A
:10D0D00080E090E0A6E1B3E480937A0290937B0233
:10D0E000A0937C02B0937D02109277020F94EF839D
:10D0F00060917A0270917B0280917C0290917D0216
:10D100000F94FC840F94CE22809193069091940604
:10D11000A0919506B09196068093F5119093F61123
:10D12000A093F711B093F81180919706909198060B
:10D13000A0919906B0919A068093F9119093FA11F3
:10D14000A093FB11B093FC1181E0809377020F94C0
:10D15000222D82E00F947B54CC20E9F081149104BD
:10D16000A104B104C1F0C501B4010F94299B9B0136
:10D17000AC01609192047091930480919404909119
:10D1800095040F94C3A16093FD117093FE118093D9
:10D19000FF11909300120F94EF83C8010E94CA5FA1
:10D1A0000F94222D0F9480900F941E8ED11007C0E3
:10D1B000311005C08B8D811102C0CC2039F1F110E6
:10D1C00025C09D81992311F181E080939C120F94D9
:10D1D000BA226B017C0180E00F94BA22A70196016C
:10D1E0000F94C7609B01AC016091FD117091FE111D
:10D1F0008091FF11909100120F94C2A16093FD11D4
:10D200007093FE118093FF119093001284E10F94AC
:10D21000BE980F94CE22109205120F900F900F908F
:10D220000F900F90DF91CF911F910F91FF90EF9092
:10D23000DF90CF90BF90AF909F908F907F906F9036
:10D240005F904F903F902F900895E3E3F3E09FE7C6
:10D2500081918F3731F0DF01119787FF07C08F77FA
:10D260008C9383E0EB33F80799F708959C93F9CFFB
:10D2700090915B02981710F480935B0280915C029E
:10D28000882339F0E091D203F091D303309709F06D
:10D2900019940895CF93DF93CDB7DEB7AE014A5FFF
:10D2A0005F4FFA0161917191AF0180EC93E00F94AF
:10D2B000E29FDF91CF91089560EC73E00D94339F6E
:10D2C00060EC73E0082E000C990B0D94039FCF9334
:10D2D000C82FC15020F080E20E946069FACFCF9140
:10D2E0000895CF93C82F862F643008F083E0809391
:10D2F00032030E94B6548C0F8093310344E650E011
:10D3000060E08068CF910C94F85CCF93DF93EA01E2
:10D310000E94716960EC73E0CE01DF91CF910D94B2
:10D32000339FCF93C42F0E94716960EC73E08C2F00
:10D33000CC0F990BCF910D94039F60E080E00E9489
:10D34000716910923103089540E456E060E081E095
:10D350000E94F85C109232031092310348E050E0D2
:10D360006FE770E083E393E00D94CDA690915C02AB
:10D37000981709F180935C028823E9F01092070561
:10D38000109206051092110681EB93E00F9429127A
:10D390000F94FC0F61507109810991096093930307
:10D3A0007093940380939503909396030E94A469CD
:10D3B00082E00C9438690895CF93C82F10923203FD
:10D3C0001092310348E050E06FE770E083E393E0B0
:10D3D0000F94CDA644E951E162E080E30E94F85C3D
:10D3E00046E950E062E080E30E94F85C46E950E0E4
:10D3F00062E080E30E94F85C46E950E062E080E28F
:10D400000E94F85C8091CE0344E650E060E08062C8
:10D410000E94F85C84E08093300344E650E060E0D2
:10D420008CE00E94F85CC1110E94A46944E650E0BF
:10D4300060E086E0CF910C94F85C81E00C94DC69AC
:10D44000CF92DF92FF920F931F93CF93DF9300D081
:10D4500000D01F921F92CDB7DEB78A30D9F48091E9
:10D460003203843018F08FEF8093320360913203DF
:10D470006F5F80E00E94716928960FB6F894DEBF56
:10D480000FBECDBFDF91CF911F910F91FF90DF9025
:10D49000CF90089590E8980F44E650E061E09A3408
:10D4A00008F5482F4058550B9A0196E0929FA0012D
:10D4B000939F500D1124FA01E45AFB48F490E3E3E2
:10D4C000F3E030E020E09FEF6191782F76277F77BF
:10D4D00089F4F901ED5CFC4F8083F22E44E650E0C4
:10D4E00061E08F2D0E94F85C809131038F5F809303
:10D4F0003103C2CF6F3709F03CC0F901ED5CFC4F3E
:10D500008083922FF92EFA01E95AFB488E010F5FB2
:10D510001F4FD801959188E0182E10FE05900294B7
:10D52000802D9795881F8D931A94B9F7BF2DE8E049
:10D53000BE02C001112444E650E060E080640E9415
:10D54000F85C6E01F9E0CF0ED11C44E650E061E0DA
:10D55000D8018D918D010E94F85CC016D106A9F703
:10D560008091310344E650E060E080680E94F85CFE
:10D57000B5CF67FF922F2F5F3F4F2830310509F05D
:10D58000A3CF9F3F09F0BECFA9CF8F929F92AF92BA
:10D59000BF92EF92FF920F931F93CF93DF93CDB77C
:10D5A000DEB7A0970FB6F894DEBF0FBECDBF6115F2
:10D5B00071058105910599F480E3A0960FB6F89462
:10D5C000DEBF0FBECDBFDF91CF911F910F91FF90B6
:10D5D000EF90BF90AF909F908F900C94206A00E0E6
:10D5E000842E912CB12CA12C9E012F5F3F4F7901ED
:10D5F000A50194010F940EA1F701E00FF11D6083C6
:10D60000B901CA010F5F611571058105910581F7A7
:10D610000E0D1F2D111DE016F10659F0F801829133
:10D620008F018A3020F4805D0E94206AF4CF895CEB
:10D63000FBCFA0960FB6F894DEBF0FBECDBFDF9133
:10D64000CF911F910F91FF90EF90BF90AF909F905F
:10D650008F900895CF92DF92EF92FF926B017C0141
:10D66000F7FE0BC08DE20E94206AF094E094D09403
:10D67000C094C11CD11CE11CF11C4AE0C701B601D9
:10D68000FF90EF90DF90CF900C94C56A0F931F939B
:10D69000CF938C01C62FCC2359F0F801249122237B
:10D6A00039F00F5F1F4F84910E94206AC150F3CF61
:10D6B0008C2F0E9467698C2FCF911F910F91089535
:10D6C0000F931F93CF938C01C62FCC2349F0F80101
:10D6D00081918F01882321F00E94206AC150F5CFEB
:10D6E0008C2F0E9467698C2FCF911F910F91089505
:10D6F000CF93DF93EC018991882319F00E94206A6F
:10D70000FACFDF91CF9108950E94206A90E080E0E7
:10D71000089510926303109214060895CF93809198
:10D720006303C1E0811104C0C0E08C2FCF91089544
:10D730000E94896BFACF8EEF9FE00F949BA08E3FE3
:10D7400039F091E020912F03281390E0892F08955C
:10D7500080E0089510922F036EEF8EEF9FE00D94FE
:10D76000BFA0853728E6920709F459C0F8F48E3631
:10D7700025E6920709F459C050F4833723E692074F
:10D78000B1F185369446B1F182E993E60895823786
:10D7900026E6920791F1823728E6920709F442C003
:10D7A0008337954689F789EE93E608958C3620E70E
:10D7B000920731F170F48C362EE6920721F18F3604
:10D7C0002EE6920731F184379946F1F687ED93E61C
:10D7D00008958B3623E79207F9F0863723E79207FF
:10D7E000A9F08F36924781F685E993E6089589EF8F
:10D7F00093E6089581EF93E6089580EE93E6089509
:10D8000080ED93E6089585EC93E608958DEB93E61D
:10D81000089587EB93E608958CEA93E6089585EAE8
:10D8200093E608958CE993E6089581E094E60895DF
:10D83000E3E5F4E785919591A591B4918F3F9F4FD2
:10D84000AF4FBF4FB1F020E031E081E0F9014591E9
:10D85000559165917491453A5A45644B7B4409F062
:10D860000895F901349645915491240F351F8F5F27
:10D87000EDCF81E008950F931F93811113C0109293
:10D880002E0310922D0310922F0390912F039813C3
:10D890005CC0682F8EEF9FE00F94BFA081E01F91C6
:10D8A0000F910895813089F7E0E0F1E045915591BD
:10D8B00065917491453A5A45644B7B4431F7E4E0F5
:10D8C000F1E0A591B491E8E0F1E06591749150E048
:10D8D00040E030E020E0A417B50729F5261B370B00
:10D8E0003227232732276217730709F0CECFECE0E7
:10D8F000F1E00591159125913491E3E5F4E7459127
:10D90000559165917491041715072607370709F09B
:10D91000BCCF20E031E030932E0320932D0391E023
:10D9200090932F03B2CFFA01E050FF4FE491F0E063
:10D9300098E040FD90E002C0EE0FFF1F9A95E2F7DD
:10D940002E0F3F1F4F5F5F4FC6CF80E0A8CF2091C3
:10D950002F03211104C0FC013296CF01089540919C
:10D960002D0350912E0341155105A9F3FC0125917A
:10D9700034912F3F320779F3F9013896EE0FFF1FEC
:10D98000E40FF51F25913491FA01E20FF31F249162
:10D99000222309F3E2CFCF93DF93EC0120E030E0C4
:10D9A0004CE852E4609101127091021280910312CE
:10D9B000909104120F94C3A160930112709302120C
:10D9C000809303129093041260E070E080EA91E487
:10D9D0000F942F850E946B5E0E94A46982E09AE5F5
:10D9E0000E94A76CAC0160E080E00E94856988819C
:10D9F000882339F061E080E00E947169CE010E94C5
:10DA0000786B85E699E30E94A76CAC0162E080E048
:10DA10000E94856983E49BE20F946D0CDF91CF91A6
:10DA20000D94CE220F944A428F3F11F180E00E9464
:10DA3000B6690E94A4698EE596E50E94A76CAC01C8
:10DA400061E080E00E94856980E20E94206A0F9474
:10DA50004A42682F70E06F5F7F4F072E000C880BE3
:10DA6000990B0E942A6B0F94526B81E00C94B6695B
:10DA700008951F920F920FB60F9211240BB60F92BA
:10DA80002F938F939F93EF93FF93E0912803E830B8
:10DA9000E8F4F0E08827E05BF2498F4F0D94ABA1EA
:10DAA000586D726D7D6D8B6DA16DAA6DCD6DDF6D45
:10DAB0008091920681110AC080915B06880F809345
:10DAC0002703882319F081E080932803FF91EF91C9
:10DAD0009F918F912F910F900BBE0F900FBE0F90C3
:10DAE0001F901895809126038F5F80932603909155
:10DAF0002703981758F382E0E7CF83E08093280349
:10DB00008FE0809325038FEF86BD81E085BD84B5CE
:10DB10008F7E84BDDBCF809125038295807F8195A8
:10DB200088BD80912503882321F0815080932503AF
:10DB3000CDCF84E0809328038FEF88BD8EEF86BD24
:10DB4000C5CF85E0809328038FEF88BD86BD82E036
:10DB500085BDBCCF2FEF28BD809192068111B6CF35
:10DB6000809126038F5F8093260390912703891766
:10DB700008F4ACCF80915B0690E08F3791050CF0F4
:10DB8000A5CF86E0809328038FE08093250326BDF0
:10DB900081E085BD84B58061BCCF809125038295ED
:10DBA000807F819588BD809125038111BECF87E05C
:10DBB0008093280380E886BD8FEF88BD87CF1092C1
:10DBC000280380E886BD8FEF88BDC1CFCF93DF9358
:10DBD000EC0187E69FE00F949BA091E0811101C0CA
:10DBE00090E081E02881211101C080E089139883B1
:10DBF00087E09FE00F949BA091E0811101C090E02D
:10DC0000998385ED9EE00F949BA091E0811101C066
:10DC100090E09A8387E49DE00F949BA08F3F21F0D2
:10DC20008887DF91CF9108951886FBCFCF93C82FB7
:10DC3000682F87E69FE00F94BFA0CC2319F0CF9107
:10DC40000D94FD535198599810928416CF910895D0
:10DC5000109284030F94FC0F60938D1670938E16B0
:10DC600080938F169093901608958093240380FDDF
:10DC70001CC010924003209140038FEF820F8E3F13
:10DC8000E8F08091A000877F8093A0001092AD0003
:10DC90001092AC009FB7222361F0F89480910201AA
:10DCA0008062809302019FBF08958FEF80934003AD
:10DCB000E2CFF894809102018F7DF3CFEFB7F89413
:10DCC0008091A00088608093A00030E08091720075
:10DCD0004FEF50E081FF04C04091A8005091A9008F
:10DCE000249FC001259F900D349F900D11246FEF4C
:10DCF00070E00F9464A17093AD006093AC00EFBF2F
:10DD000008951F93CF93DF93D0912403D1FD1DC0BD
:10DD100010919A03C1E020E030E048E452E46091C1
:10DD2000C40D7091C50D8091C60D9091C70D0F94D3
:10DD30004CA418160CF0C0E0DE7FCD2B81E0111151
:10DD400001C080E0C82BC093240380912403DF919D
:10DD5000CF911F910C94356EEF92FF920F931F930A
:10DD6000CF93DF93EC018B017A010E941055811152
:10DD70000BC0A801BE01C701DF91CF911F910F9188
:10DD8000FF90EF900D94AFA0DF91CF911F910F9175
:10DD9000FF90EF9008950F931F93CF93DF938C0123
:10DDA000D62FC72F0F94A9A08F3F980739F46D2F56
:10DDB0007C2FC8010F94F9A08D2F9C2FDF91CF915C
:10DDC0001F910F9108950F931F93CF938C01C62F2E
:10DDD0000F949BA08F3F29F46C2FC8010F94E3A0F0
:10DDE0008C2FCF911F910F910895CF93DF93EC016A
:10DDF0000F94A9A0BC016F5F7F4FCE01DF91CF913F
:10DE00000D94F9A0CF93DF93EC010F949BA061E0F8
:10DE1000680FCE01DF91CF910D94E3A02BE0829F9C
:10DE2000C0011124805B924F0F94A9A021E00196BC
:10DE300009F420E0822F0895CF93DF93C82FD8E014
:10DE4000CF5FC8300CF0C0E08C2F0E940E6F8111A4
:10DE500003C0D150A9F7CFEF8C2FDF91CF91089558
:10DE600081EA9DE00F949BA00E941C6F87FD05C076
:10DE7000682F81EA9DE00D94BFA008950F931F9332
:10DE8000CF93C82F8B0166E074E7823070F06FEF9C
:10DE900073E7843050F067EF73E7843031F06FEE52
:10DEA00073E7853011F068EE73E7C8010F94529E56
:10DEB0008CEF8C0F823028F0C170CF5CF801C683E4
:10DEC0001782CF911F910F91089561E080EC9FE040
:10DED0000F94BFA060E08FEB9FE00F94BFA060E0C5
:10DEE0008EEB9FE00F94BFA060E08DEB9FE00F945E
:10DEF000BFA060E08CEB9FE00D94BFA0CF93C82F34
:10DF000082958F700E94C65C8C2F8F70CF910C947D
:10DF1000C65C4091CF115091D01190E080E0411546
:10DF20005105B1F12091CB113091CC1190E080E0FE
:10DF3000F901E252F04FA081A23021F46181728197
:10DF4000860F971F4150510919F1F901EF51F04F18
:10DF5000A1919F012E5D3F40A111FACFF901E2523C
:10DF6000F04F2D3EA1E03A0730F4A191A111E0CF8E
:10DF70002F5F3F4FF6CF2D3EE1E03E07C9F6EEEDB5
:10DF8000FFE09F012E5D3F40A191AA23D1F3D0CFA6
:10DF900008958091CF119091D011181619060CF0A8
:10DFA00043C001979093D0118093CF11892BA1F496
:10DFB0008091DA0F9091DB0F892B21F41092DD0F05
:10DFC0001092DC0F8091DC0F9091DD0F9093CC11BB
:10DFD0008093CB1181E008958091CB119091CC1169
:10DFE0000396FC01E252F04F208101962111F9CFF6
:10DFF000FC01E252F04F8D3E21E0920740F4419146
:10E000009C012F5F3F4F4111E1CFC901F4CFEEEDED
:10E01000FFE08D3E21E09207C9F6CF018E5D9F4063
:10E0200021912223D1F3D2CF80E00895FC0120E09A
:10E030003EE2DB014D91BD01403249F0283011F440
:10E0400030833196DB0111974C91408331962F5FDD
:10E050002B3079F71082089540E050E0BA010D941A
:10E06000F739FC01238121110D94516F089590918E
:10E070000405911107C09091C00095FFFCCF8093DB
:10E08000C6000895913031F49091C80095FFFCCFFF
:10E090008093CE0008950E94377090E080E008954C
:10E0A000CF93DF93EC01FE018491882321F00E943D
:10E0B00037702196F8CFDF91CF910895CF92DF92FC
:10E0C000EF92FF92C090C40DD090C50DE090C60DA8
:10E0D000F090C70D89E598E70E94507042E0C701B3
:10E0E000B6010F94089881E598E70E9450706091FE
:10E0F0008A0370918B0380918C0390918D0341E092
:10E100000F940898FF90EF90DF90CF900D94BB98FC
:10E110004F925F926F927F928F929F92AF92BF9237
:10E12000CF92DF92EF92FF920F931F93CF93DF93E3
:10E13000CC24CA94DC2C76010EEA1FE093E2892EEF
:10E14000912CA12CB12C412C512C3201D0E0C0E0FB
:10E150008FEFC81609F45DC0C8010F94A9A0EC01A7
:10E16000BC01990F880B990B0F94299B20913E04B9
:10E1700030913F0440914004509141040F94C2A259
:10E180002B013C01C701B6010F9461978DEA97E717
:10E190000E945070C501B4010F9461978DEA97E712
:10E1A0000E945070BE010D2E000C880B990B0F942D
:10E1B00061978DEA97E70E94507020E030E04AE7CF
:10E1C00054E4C301B2010F94689B0F94454285E06B
:10E1D000880E911CA11CB11C0E5F1F4F8FEFC81A37
:10E1E000D80AE80AF80A0A3B8FE0180709F0B0CF0E
:10E1F000DF91CF911F910F91FF90EF90DF90CF9023
:10E20000BF90AF909F908F907F906F905F904F9056
:10E2100008958CE89DE30E945070B8CF882371F177
:10E2200081EA97E70E9450706091231270E090E0BD
:10E2300080E00F946197809123128430D8F010927F
:10E2400023128CE997E70E9450708091231290E08E
:10E250000F946242809123122091EF113091F011BE
:10E260003093F2112093F1110E9433F70E946B5EFC
:10E270000D94CE228F5F80932312E3CF84E29EE33E
:10E280000E94A76C70E060E00E94E7BCE5CFCF93EE
:10E29000DF9389E997E70E945070C5EFD1E168816B
:10E2A00079818A819B8142E00F94089885E997E7FC
:10E2B0000E9450706C817D818E819F8142E00F941D
:10E2C000089881E997E70E945070688579858A856A
:10E2D0009B8542E00F9408988DE897E70E94507064
:10E2E0006C857D858E859F8542E00F94089889E036
:10E2F00094E60E94507080E00F94AC220F94299B0A
:10E30000C2E3D4E02C813D814E815F810F94C2A293
:10E3100042E00F94089889E897E70E94507081E0E6
:10E320000F94AC220F94299B288539854A855B85FB
:10E330000F94C2A242E00F94089885E897E70E94E4
:10E34000507082E00F94AC220F94299B2C853D8560
:10E350004E855F850F94C2A242E00F94089881E831
:10E3600097E70E94507083E00F94AC220F94299B92
:10E37000288939894A895B890F94C2A2DF91CF919C
:10E380000D94454280E996E70E9450706091C40D5B
:10E390007091C50D8091C60D9091C70D41E00F940D
:10E3A00008988DE896E70E9450706091F111709185
:10E3B000F211072E000C880B990B0F94299B41E05A
:10E3C0000F94089889E896E70E94507060918A033C
:10E3D00070918B0380918C0390918D0341E00F9499
:10E3E000089886E896E70E9450706091ED11709150
:10E3F000EE11072E000C880B990B0F94299B41E01E
:10E400000F94089881E896E70E9450706091C40DBF
:10E410007091C50D8091C60D9091C70D41E00F948C
:10E4200008988EE796E70E9450706091F111709104
:10E43000F211072E000C880B990B0F94299B41E0D9
:10E440000F9408988AE796E70E94507060916206E0
:10E4500070E090E080E00F94619785E796E70E9476
:10E46000507060915B0670E090E080E00F946197DF
:10E4700081E796E70E94507060918E0670918F063A
:10E48000809190069091910641E00F9408980D9428
:10E49000BB980E9450700D94BB988F929F92AF9240
:10E4A000BF92CF92DF92EF92FF920F94FC0F6B011D
:10E4B0007C0120913202222309F1409178024130FF
:10E4C000E9F08091140290911502A0911602B0918A
:10E4D000170246015701881A990AAA0ABB0A30E0B6
:10E4E000A8EEB3E00F943BA186169706A806B906DE
:10E4F0006CF0443031F19CF44230D4F4C0921402F8
:10E50000D0921502E0921602F0921702FF90EF905F
:10E51000DF90CF90BF90AF909F908F90089545303F
:10E5200069F781E69DE90E9450708CE598E706C086
:10E5300081E69DE90E94507089E898E70E9449723F
:10E54000DDCF81E69DE90E94507083E798E7F6CF22
:10E55000CF9381EA9DE00F949BA0CBE08C9FC001FC
:10E560001124805B924F0F94A9A08156904F803A5E
:10E570009F40C8F088E298E70E94497281EA9DE0D6
:10E580000F949BA08C9FC001112470E060E0805B21
:10E59000924F0F94F9A08BEE97E70F94A90B81E0AF
:10E5A000CF910C94B669CF910895EC01F8940F9433
:10E5B000E712179A1092A306169A1092A406149ABC
:10E5C00084E49DE90E9450708CEC97E70E944972A8
:10E5D000209779F0CE010E944972BE0185E99CE046
:10E5E0000F94F9A062E484E99CE00F94E3A00E94F8
:10E5F0009D60C4ECD7E7F1CF8AE493E00F94291231
:10E600008091CF119091D011892B79F0E091CB11AD
:10E61000F091CC11E252F04F8081813011F08630C0
:10E6200021F481E399E60C94497208958091CF1109
:10E630009091D011892B29F00E94FC720E94C96F21
:10E64000F5CF1092CC111092CB111092DD0F1092D9
:10E65000DC0F81E08093E6110895EF92FF920F9313
:10E660001F93CF93DF9380919C12882389F186E5D5
:10E6700097E70E94497280E497E70E9449728FE20F
:10E6800097E70E944972C7E0DCE1C15058F1CD9F85
:10E690007001112401E010E08CE297E70E945070B5
:10E6A000F801EE0FFF1FEE0FFF1FEE0DFF1DE756E7
:10E6B000FD4E608171818281938145E00F940898BD
:10E6C0000F5F1F4F0830110539F70F94BB98DDCF4E
:10E6D00083E697E7DF91CF911F910F91FF90EF9025
:10E6E0000C944972DF91CF911F910F91FF90EF90A1
:10E6F0000895CF92DF92EF92FF926B017C01C0925E
:10E700002903D0922A03E0922B03F0922C038091EC
:10E7100045038230B1F420E030E040E950E4C70125
:10E720000F94B8A287FF14C0809162049091630493
:10E73000A0916404B0916504803D9740A105B105A6
:10E7400020F5C701B601FF90EF90DF90CF900895BC
:10E750002AE939E949E95EE3C701B6010F94B8A295
:10E7600087FF0AC020E030E048E351E4C701B6016A
:10E770000F94689B6B017C018AE394E70E945070C0
:10E78000C701B6010F944542DCCF2AE939E949E9CE
:10E790005EE3C701B6010F94B8A287FDE3CF20E086
:10E7A00030E040E85EE3C701B6010F94689B20E0CB
:10E7B00030E048E550E40F94C3A1DCCFCF92DF9264
:10E7C000EF92FF92CF93909145039817B9F1C82F1C
:10E7D000C0902903D0902A03E0902B03F0902C03E3
:10E7E00020E030E0A901C701B6010F94B8A2882348
:10E7F00041F0C0928604D0928704E0928804F0929F
:10E8000089048DE194E70E945070C13011F1E0F06D
:10E81000C23011F1C0934503609186047091870462
:10E8200080918804909189040E9479736093860492
:10E83000709387048093880490938904CF91FF900C
:10E84000EF90DF90CF90089585E194E70E944972A0
:10E85000E1CF81E194E7FACF8DE094E7F7CF0F9411
:10E86000CE22179AE3EAF6E01082169A1182149AE1
:10E8700080E00E94DE738FEF9FEF9093750280938C
:10E8800074022FEF2093710290933E0280933D0219
:10E8900020933F02909373028093720290933C0204
:10E8A00080933B020895182FF894CDB7DEB700D0BF
:10E8B000CF90DF90EF9088E199E20FB6F894A89599
:10E8C000809360000FBE909360009FB7F894E2E0E1
:10E8D000F1E08081886080839FBF0F94E7128CEC09
:10E8E00093E70E94497284EC93E70E945070612F75
:10E8F00070E090E080E04AE00F94EB9680EC93E7C4
:10E900000E9450708E2DB60190E040E10F94EB967E
:10E910008CEB93E70E945070BE0190E080E040E1F4
:10E920000F94EB960F94BB9840E060E072E290E0A9
:10E9300080E00F94A45381E399E60E9449720E94FB
:10E940009D60C82F9FB7F8948091020184608093E6
:10E9500002019FBF6C2F83E09DE00F94BFA08091C8
:10E960007C06882319F08C2F0E9453740E949D60AE
:10E970001F920F920FB60F92112483E00E94A17490
:10E980001F920F920FB60F92112482E00E94A17481
:10E9900041ED50E06BEE72E782E394E00F94359E18
:10E9A0000F9454750F9422190E94C85E81E69DE968
:10E9B0000E94507089EC92E70C94497244E050E058
:10E9C00064E170E082E394E00F948BA043E050E0B8
:10E9D0006BEE72E782E394E00F947A9E892B09F044
:10E9E0005DC0EFEAF3E7459155916591749188ED2B
:10E9F00090E00E94185DE3EBF3E745915591659136
:10EA000074918CED90E00E94185DE7EBF3E7649160
:10EA100080EE90E00E94E36EE8EBF3E7659174917D
:10EA200081EE90E00E94CB6EEAEBF3E76591749182
:10EA300083EE90E00E94CB6EEBEAF3E745915591AF
:10EA40006591749184ED90E00E94185D47E853E76A
:10EA500060E170E080EB90E00E94AC6E47E953E724
:10EA600060E170E080EC90E00E94AC6E41ED50E01F
:10EA700064E170E082E394E00F948BA00E94C85E92
:10EA80000F9454750F94221981E69DE90E945070ED
:10EA90008FEA92E70E94497281E008950E94C8744B
:10EAA00064E070E084E190E00E94105591E08927D5
:10EAB00008956BEE72E782E394E00F94529E41ED6D
:10EAC00050E064E170E082E394E00F94AFA081E64F
:10EAD0009DE90E9450708FE992E70C9449722F9241
:10EAE0003F924F925F926F927F928F929F92AF92DE
:10EAF000BF92CF92DF92EF92FF920F931F93CF932B
:10EB0000DF93CDB7DEB7A0970FB6F894DEBF0FBE88
:10EB1000CDBF8FE590E00E94BC55882309F4A1C0C9
:10EB20000E94C0548F37910561F48091B105909196
:10EB3000B2059093B0058093AF0580E992E70E94FB
:10EB400049726E014FE1C40ED11C992493940E9426
:10EB5000C054181619060CF078C08091E71188236C
:10EB600029F00E94B360882309F46FC0809161038B
:10EB700081116BC02091B1053091B2058091AF0534
:10EB80009091B0058217930711F3F901E15DFA4FF7
:10EB900080812F5F3F4F2F7733273093B20520932B
:10EBA000B1058F3F09F079C080911B03882309F4D8
:10EBB00071C090921A0310921B031F8E18A28090AE
:10EBC0001E03882021F280911C038F8FF1E0F8153D
:10EBD00018F480911D0388A310921E031601822D44
:10EBE0008C19881508F0B3CFF10111911F0181E252
:10EBF00093E00F945E1017FDF2CF8091DA0F9091A1
:10EC0000DB0F1A3009F44BC11D3009F448C18F35B0
:10EC100091050CF049C11B3311F49092200320910F
:10EC200020032111DCCF9C012F5F3F4F3093DB0F7E
:10EC30002093DA0F2091DC0F3091DD0F2252304FFC
:10EC4000820F931FFC011383CACF8091DA0F90913A
:10EC5000DB0F181619060CF451C280916A1381114A
:10EC600067C2A0960FB6F894DEBF0FBECDBFDF918E
:10EC7000CF911F910F91FF90EF90DF90CF90BF90B9
:10EC8000AF909F908F907F906F905F904F903F904C
:10EC90002F90089590921B0390CF90911A0399237F
:10ECA00009F458C0893FE9F170F5863F09F44AC07C
:10ECB000873F09F443C08BE592E70E94507086E5D8
:10ECC00092E70E9450701091190382E592E710FDBF
:10ECD00002C08DE492E70E945070012F027088E418
:10ECE00092E711FD02C083E492E70E94507082E433
:10ECF00092E70E944972002349F185E480930B0258
:10ED000010921A035ACF8A3F41F08B3FA1F68091AF
:10ED10001903816080931903CECF809119038E7FF0
:10ED2000F9CF10921E0310921A0310921903109239
:10ED3000180310921B0310921703BDCF8091190383
:10ED40008260E8CF809119038D7FE4CF90E29093A9
:10ED50000B02D6CF90911B0330911903992331F107
:10ED6000E0911E0330FF49C020911703222309F4CC
:10ED700040C091E09E0F90931E03AE2FB0E0A45EC2
:10ED8000BC4FFFEFFC9340911803442351F0EE5F1A
:10ED9000E0931E03E92FF0E0E45EFC4F4083109205
:10EDA000180321502093170310921B03E0911E03B8
:10EDB00030FF6CC090911703992349F121E02E0F89
:10EDC00020931E03AE2FB0E0A45EBC4F8C938091C5
:10EDD0001803882351F0EE5FE0931E03E22FF0E06A
:10EDE000E45EFC4F808310921803915090931703B8
:10EDF000E4CE42E040931703D7CF91E09E0F90936B
:10EE00001E03F0E0E45EFC4F9FEF9083CDCFA82F70
:10EE1000AF7030E021E0AF3029F0B0E0A050BE4F3D
:10EE20003C9120E0482F407F403F59F4226020FF72
:10EE300013C09092170321FF0CC0E2E0E093170388
:10EE4000BCCE82958F70A82FB0E0A050BE4F9C9191
:10EE5000EECF90931803B1CE81E08E0F80931E0306
:10EE6000AE2FB0E0A45EBC4F3C933A3009F4A5CE7F
:10EE700021FF03C090921703A0CEEE5FE0931E0324
:10EE8000E82FF0E0E45EFC4F908397CE91E09E0F78
:10EE900090931E03F0E0E45EFC4F80838ECE0097DB
:10EEA00019F410922003DDCE0091DC0F1091DD0FDC
:10EEB0000F51104F800F911FFC0110821A8309839C
:10EEC000809120038111FDC0F80180818E3409F00A
:10EED00084C04AE050E0BE016F5F7F4FC8010196D9
:10EEE0000F94269C2B013C01E980FA80F701808178
:10EEF000803231F4FFEFEF1AFF0AFA82E982F4CF91
:10EF00008091D1119091D211A091D311B091D411CF
:10EF10000196A11DB11D84159505A605B70549F0FB
:10EF200044E050E06BE872E7C7010F947A9E892BAA
:10EF3000A1F46AE270E0C7010F94F2A69093F6166E
:10EF40008093F516009709F441C0F801F12C8E1753
:10EF50009F07F1F02191F226FACF84E49DE90E9407
:10EF6000507080E293E60E9450706091D1117091D0
:10EF7000D2118091D3119091D4110F9461970F9475
:10EF8000BB980E94E2541092DB0F1092DA0F69CE08
:10EF90000E944D55F816190639F084E49DE90E9447
:10EFA000507081E093E6DFCFE091F516F091F61610
:10EFB0001082E980FA8066E872E7C7010F94499EE3
:10EFC000892B39F587E695E60E94D57284E49DE9A0
:10EFD0000E94507087ED92E6C6CF89819A81FC012C
:10EFE0002081203221F401969A838983F6CF6AE248
:10EFF00070E00F94F2A6892B39F084E49DE90E9419
:10F0000050708DEA92E6AFCF44244A94542C3201DA
:10F01000D0CF44E050E061E872E7C7010F947A9ED8
:10F020005C01F7018081873481F48091CB0D8530BC
:10F0300061F085ED91E10F945E10F6E0F093CB0D59
:10F0400060E085EA9FE00F94BFA0AB2821F080919B
:10F05000CE11811198CF26E077FC21E08091DC0F62
:10F060009091DD0FFC01E252F04F208349815A81DB
:10F07000F801DA0140175107A1F501900020E9F7E6
:10F080009F01201B310B0396280F391F2D3EF1E005
:10F090003F0779F13093DD0F2093DC0F8091CF1182
:10F0A0009091D01101969093D0118093CF1177FC5D
:10F0B00008C04092D1115092D2116092D311709237
:10F0C000D4111092DB0F1092DA0F0E94C054892BDA
:10F0D00009F4C7CD8FE590E00E94BC5581117FCD2A
:10F0E000C0CD6D9161939D01241B350B6111F9CF4A
:10F0F000CACF1092DD0F1092DC0FD0CF8091CA0DD5
:10F1000060E273E0811102C060ED77E081E293E09C
:10F110000F942F10882309F4A0CD10922003109291
:10F12000DB0F1092DA0F86E792E70E94497299CDC1
:10F130008091FD15882309F494CD8091DA0F909188
:10F14000DB0F892B09F08DCD8091CF119091D011DB
:10F15000892B11F410921F0312E001E040917E16FA
:10F1600050917F166091801670918116809177166C
:10F1700090917816A0917916B0917A164817590790
:10F180006A077B0708F0C1C080911F038111BDC0D1
:10F190000F948D4940910216509103166091041608
:10F1A0007091051640937E1650937F1660938016DB
:10F1B000709381162091DA0F3091DB0F8A3061F065
:10F1C0008D3051F0833209F487C02F35310524F496
:10F1D0008F3F980709F087C02115310509F441CD0B
:10F1E0008091FD15811103C040E050E0BA0180918B
:10F1F000DC119091DD11481B590BA091DC0FB091EF
:10F20000DD0FFD01E252F04F1083418352831396CC
:10F210002252304FF901EA0FFB1F1082A252B04F69
:10F22000FD0101900020E9F73197EA1BFB0BF894F0
:10F230008091CF119091D01101969093D01180932D
:10F24000CF11EC5F8091DC0F9091DD0FE80FF92F6B
:10F25000F11DF093DD0FE093DC0F8091FD15882305
:10F2600009F43DC080917E1690917F16A091801682
:10F27000B09181168093DC119093DD11A093DE1183
:10F28000B093DF11ED3EF14021F41092DD0F1092AA
:10F29000DC0F7894109220031092DB0F1092DA0F9B
:10F2A00040917E1650917F16609180167091811664
:10F2B0008091771690917816A0917916B0917A1670
:10F2C000481759076A077B0700F58FE590E00E9411
:10F2D000BC55811143CFC5CC00931F037DCF80E087
:10F2E00090E0DC01C7CFA9014F5F5F4F5093DB0F68
:10F2F0004093DA0F4091DC0F5091DD0F4252504F96
:10F30000240F351FF901838329CF40917E16509138
:10F310007F1660918016709181168091771690917A
:10F320007816A0917916B0917A16481759076A078E
:10F330007B0708F496CC0E94896F892B09F091CC49
:10F340000F949C428AE992E60E9449720F94F21C43
:10F350006B017C010E942E5F8CE3882E912CA12CE6
:10F36000B12CC701B601A50194010F940EA1CA01E9
:10F37000B901A50194010F940EA17F936F93C7016A
:10F38000B60120E13EE040E050E00F940EA13F9333
:10F390002F9382E692E79F938F938E010F5F1F4F0B
:10F3A0001F930F930F94B29F81E69DE90E945070C6
:10F3B000C8010F94BC99C8010E94BBEF0F94FD4D8A
:10F3C000109256020FB6F894DEBF0FBECDBF8091EB
:10F3D0006B13882359F00F94D0448091CA0D882371
:10F3E00009F43FCC86E00F94BE983BCC81E00F94AB
:10F3F0003C4E80916B138111EECFEFCF0F931F9393
:10F40000CF93DF93D82F80918416813009F449C0BF
:10F41000823009F44DC00E940F618111ECC08091CF
:10F42000F1119091F211009739F42091ED11309182
:10F43000EE11232B09F4DFC04091330250913402C6
:10F4400060913502709136024115510561057105D3
:10F4500009F4D1C0892B31F48091ED119091EE1116
:10F46000892B29F080911A06882309F42CC18091F8
:10F47000CA0D882321F040EE52E369E270E08AE190
:10F4800096E00F946A10882309F4B7C00F94E7122E
:10F4900080E696E30E94A76C0F94A90B0E946DFE74
:10F4A000ACC082E0809384160E94F9C380938716D3
:10F4B0001092881680918416823009F0ACCF80912A
:10F4C000891681113DC00E94F9C3C82F809187160B
:10F4D000C81709F4A0CFC093871689E896E10F9466
:10F4E0005E10CC23B1F180918516882311F18091B3
:10F4F000620381111EC0809194128130D1F08091FD
:10F50000A80D9091A90D891B8F7099F40E94BE607F
:10F5100081110FC08091C80D843059F08FE59FE0B4
:10F520000F949BA0811105C061E083E198E30F94E3
:10F53000E89481E08093881681E080935B026BCF32
:10F5400064E670E089E896E10F942F108111BBCF3B
:10F5500062CF80918616882379F3809162038111AE
:10F56000EBCF8091A80D9091A90D891B8F7021F48C
:10F570000E94BE60882301F38091E7118111DCCFE6
:10F58000809194128130C1F28091C80D8430A1F233
:10F590008FE59FE00F949BA08111CECF88E694E683
:10F5A0009F938F938EE494E69F938F930F945D9F28
:10F5B00010928616109285160F900F900F900F9054
:10F5C0008091E711811105C060E070E0CB010F94DC
:10F5D000A94260E070E0CB010E94366185E69FE0C1
:10F5E0000E94026F81E09FE00E94F56E8BE79BE630
:10F5F0000F941644A1CF10921A068091CF119091CA
:10F60000D011039714F40E946F759091A80D80910A
:10F61000A90D981781F08091CB0D863061F468E8D0
:10F6200073E185ED91E10F942F10882321F085ED92
:10F6300091E10F945E104091460350914703609111
:10F64000480370914903411551056105710509F0A1
:10F650003FC0409137025091380260913902709159
:10F660003A024115510561057105A9F08AE493E05C
:10F670000F946A10882379F09091A80D8091A90DBC
:10F68000981309C0D11107C0179A1092A306169AB1
:10F690001092A406149AC091E9119091A90D80913D
:10F6A000A80D981701F18091A90D9EE6899FF001A0
:10F6B0001124E25FF84FC0819091A80D981799F03E
:10F6C0008F5F8F70F9CF8AE196E00F94291295CF62
:10F6D0008AE493E00F946A10882309F4BACF80EB90
:10F6E00097E70E94D572CC2309F4BEC080914103F4
:10F6F00090914203A0914303B0914403892B8A2B3C
:10F700008B2B81F40F94FC0F605E7C4F8F4F9F4FCB
:10F7100060934103709342038093430390934403A7
:10F72000CFEF0FC00F94FC0F0091410310914203E3
:10F7300020914303309144036017710782079307B8
:10F7400078F380918403882309F497C0C0936702FB
:10F7500080912D04811107C081E080932D040F94C6
:10F76000116510922D04809113068823C9F110921F
:10F7700013064FB7F89480911106282F082E000C1D
:10F78000330B37FF03C03195219531092430310502
:10F790000CF476C0982F87FF02C093E0980F9595E0
:10F7A00095952091060530910705290F311D97FD8C
:10F7B0003A953093070520930605837887FF03C0A9
:10F7C00081508C6F8F5F809311064FBF86E00F943E
:10F7D0002B2D80915B02811103C081E080935B023D
:10F7E00080911406882361F00E94896BE091D40314
:10F7F000F091D503309721F080915C028111199529
:10F800002091621330E0A8EEB3E00F943BA1AB016E
:10F81000BC0183E693E10F946A10882399F08091EC
:10F82000611380FD0E94C2718091611382FD0E946C
:10F8300047718091611381FD0E94935F83E693E19C
:10F840000F9429128091CA0D811102C00E944D723D
:10F8500040E355E760E070E08AE593E0DF91CF9107
:10F860001F910F910D946A10109241031092420360
:10F87000109243031092440364CFC093050568CFF0
:10F88000109211064FBF80E0A2CFCF93DF93EC011F
:10F890000F94133381E00E94FE7980E00E94386962
:10F8A000209799F0C233D10540F062E370E080E028
:10F8B00090E00F94030EE297EBCFBE0190E080E062
:10F8C0000F94030ED0E0C0E0E3CFDF91CF91089515
:10F8D000CF93DF93C82FDFEF0F94133381E00E94A3
:10F8E000FE79809192128F3FD9F480912712843053
:10F8F00021F480912A128111EFCF809165129091AD
:10F900006612019749F780918C1290918D1289327D
:10F91000904811F360E089E290E80F946950DCCFE1
:10F92000D0939212853039F4CF3FF9F261E08C2FF9
:10F930000F94AD6BD1CF8430C1F6DF91CF91089594
:10F94000CF93DF93EC018991882319F00E943770DF
:10F95000FACFDF91CF910895FF920F931F93CF932A
:10F96000DF93EC01F62E662309F44BC00F94599EE9
:10F970008C01C8010E94BC55882309F453C08091B2
:10F98000DC0F9091DD0FFC01E252F04F23E0208369
:10F990008F51904FBE01FF20E9F10F94529E81E6F6
:10F9A0009DE90E9450708FE892E60E94507080910D
:10F9B000DC0F9091DD0F8F51904F0E94A07C80E46E
:10F9C00092E70E9449728091DC0F9091DD0F0496BE
:10F9D000080F191F0D3E81E01807F9F01093DD0F95
:10F9E0000093DC0F8091CF119091D01101969093EC
:10F9F000D0118093CF11DF91CF911F910F91FF9084
:10FA00000895FC0101900020E9F731978F01081B50
:10FA1000190BAFCF0F9406A7C2CF1092DD0F109233
:10FA2000DC0FE0CF84E49DE90E9450708FE892E6FD
:10FA30000E945070CE01FF2059F00E94507082E168
:10FA40009DE9DF91CF911F910F91FF900C94497226
:10FA50000E94A07CF4CF0F931F93CF93DF93D62FF8
:10FA60008C01C0E0F8018591949128E68D309207D1
:10FA700021F420919412213019F461E00E94AC7CB1
:10FA8000CF5F0E5F1F4FDC13EDCFDF91CF911F9142
:10FA90000F910895CF93DF93CDB7DEB76E970FB672
:10FAA000F894DEBF0FBECDBF9E012C5D3F4FF90124
:10FAB000419151919F016EE170E0CE0101960F944A
:10FAC000F19F60E0CE0101960E94AC7C6E960FB66D
:10FAD000F894DEBF0FBECDBFDF91CF9108951F9286
:10FAE0000F920FB60F9211240BB60F922F933F93E4
:10FAF0004F935F936F937F938F939F93AF93BF9336
:10FB0000EF93FF932091780030917900E0911603F4
:10FB1000F0E0EE0FFF1FEA5FFC4F80819181820FC2
:10FB2000931F91838083809105038F5F80930503EA
:10FB30008031E9F5809116038F5F8093160388303A
:10FB400071F5809106039091070390934A06809384
:10FB5000490680910A0390910B0390934C06809381
:10FB60004B06809108039091090390934806809377
:10FB7000470681E080936306FF91EF91BF91AF91BB
:10FB80009F918F917F916F915F914F913F912F91B5
:10FB90000F900BBE0F900FBE0F901F901895809185
:10FBA00004034FE553E08F5F41F41092040380910A
:10FBB0007A00806480937A00DFCF9A01082E02C019
:10FBC000359527950A94E2F720FFEDCF8093040343
:10FBD0000E94CD5410920503EACFCF93DF93CAE77A
:10FBE000D0E088818F7B88831092050310921603E2
:10FBF0001092040380E00E94CD54E6E0F3E080E13F
:10FC0000DF011D928A95E9F7888180648883DF91FE
:10FC1000CF9108952F923F924F925F926F927F9271
:10FC20008F929F92AF92BF92CF92DF92EF92FF920C
:10FC30000F931F93CF93DF93CDB7DEB7A4970FB683
:10FC4000F894DEBF0FBECDBF0F94CE228091AC0DD5
:10FC5000811117C081E0809306128091A30688234A
:10FC600049F08091A406882329F02091A5062F83CE
:10FC7000211120C081E08093E61182E198E60F9483
:10FC80001644A4960FB6F894DEBF0FBECDBFDF9129
:10FC9000CF911F910F91FF90EF90DF90CF90BF9089
:10FCA000AF909F908F907F906F905F904F903F901C
:10FCB0002F9008958BEA9DE00F949BA0182F8EE45F
:10FCC0000E942B55082F0E9440558E83002329F057
:10FCD000873009F4C9C0833029F0133009F0C3C05C
:10FCE00063E06E8380E090E0A0E8BFE38A839B83BB
:10FCF000AC83BD838AEA9DE00F949BA0888F83E448
:10FD00000E942B55182F0E944055112329F088235B
:10FD100019F08B3008F4888F88E50E942B558823D2
:10FD200009F4ABC00E94035A20E030E048E052E4FE
:10FD30000F94C2A120E030E048EB51E40F94C2A13F
:10FD40006A877B878C879D8789E50E942B5588234E
:10FD500009F49CC00E94035A20E030E048E052E4DD
:10FD60000F94C2A120E030E040EA50E40F94C2A119
:10FD70006C8B7D8B8E8B9F8B87E50E942B55882308
:10FD800009F489C00E94035A2A853B854C855D850C
:10FD90000F94C3A120E030E048E852E40F94C3A1DF
:10FDA000698F7A8F8B8F9C8F88E40E942B558823D4
:10FDB00009F47AC00E94035A2C893D894E895F89D3
:10FDC0000F94C3A120E030E048E852E40F94C3A1AF
:10FDD0006D8F7E8F8F8F98A30F94B05680912C02D9
:10FDE00090912D02A0912E02B0912F0280939D122E
:10FDF00090939E12A0939F12B093A0120F94CA8B5F
:10FE000005EC1FE0C8010F94A9A0019609F051C0AC
:10FE10000E5F1F4F053D8FE01807A1F7212CACE9BD
:10FE2000B2E1BAA3A9A3B987A887512C412C312CE0
:10FE3000042D842D63E00F944AA1988B6884798403
:10FE400010E0F889F11137C0812F63E00F944AA1C7
:10FE5000911131C021103FC17E81733009F470C00F
:10FE60008F818E8737C01E836AE979E989E19FE334
:10FE70006A837B838C839D833DCF80E090E0A0E804
:10FE8000BFEF8A879B87AC87BD875ECF60E070E05D
:10FE900080E89FEF6DCF80E090E0A0E8BFE7898F1A
:10FEA0009A8FAB8FBC8F80CF60E070E080E89FE7D7
:10FEB0008FCF2F80B4CF60E070E080EC9FE7D3015C
:10FEC00011966D937D938D939C931497BE81B3305F
:10FED000C1F11E86812F0F94248C4B015C01802F71
:10FEE0000F94248C6B017C01A50194016A857B85AC
:10FEF0008C859D850F944CA418160CF41CC1298D7B
:10FF00003A8D4B8D5C8DC501B4010F944CA418162D
:10FF10000CF411C1A70196016C897D898E899F8996
:10FF20000F944CA418160CF406C12D8D3E8D4F8DE8
:10FF300058A1C701B6010F944CA418160CF4FBC0CD
:10FF400033941F5F24E0620E711C173009F079CFE3
:10FF50006FEF461A560A888599854C969987888747
:10FF600097E04916510409F063CF0E9436F1A09141
:10FF7000C706AF83B091AC03B88781E08093C70612
:10FF80008AE0830D8093AC0381E00E94386980E0B1
:10FF900090E0A0EAB0E48093FD119093FE11A0934D
:10FFA000FF11B093001265E575E585E591E40F94C6
:10FFB0002F8580E00E94E45F9CA38BA3312C832DCE
:10FFC00067E00F944AA1F82E092F682F70E07F8711
:10FFD0006E8780FF03C076E0791B072F802F63E0D8
:10FFE0000F944AA1911105C08F2D0F944AA111E0E1
:10FFF000911110E0802F0F94248C688B798B8A8B61
:020000021000EC
:100000009B8B8F2D0F94248C4B015C018E81833050
:1000100009F099C01111C8C027E0AE85BF852A9F9D
:10002000F0012B9FF00D1124E00FF11DEE0FFF1FCB
:10003000EE0FFF1FE456FD4E60E070E080EC9FE79E
:1000400061837283838394833394E1E33E12B7CF59
:1000500080E090E0A0EAB0E48093FD119093FE115F
:10006000A093FF11B093001265E575E585E591E475
:100070000F942F850F94CE22B1E33B1609F43CC2B6
:1000800080913F0391E0980F90933F03882309F4F8
:10009000D3C160E080E00E94CCEF84E396E30E944D
:1000A000A76C0F94A90B80E00F946B3081E08093D4
:1000B000780287E69BE60E9499E62F812093C70687
:1000C00068856093AC0382E00E9438690F94CE2269
:1000D00010920612D6CD011103C0112309F4BCCE33
:1000E000812F63E00F9456A1840D952D911D880FEB
:1000F000991F8D53904F0F94A9A0BC01990F880BA5
:10010000990B0F94299B2AE037ED43E25CE30F94AF
:10011000689B9B01AC0160919D1270919E12809131
:100120009F129091A0120F94C3A1F3016183728377
:100130008383948391CEFE85FF2309F402CF22208E
:1001400009F4FECEFECE288939894A895B896A8501
:100150007B858C859D850F944CA4181604F1288905
:1001600039894A895B89698D7A8D8B8D9C8D0F9435
:10017000B8A287FD14C0A50194016C897D898E8980
:100180009F890F944CA4181654F0A50194016D8D0D
:100190007E8D8F8D98A10F94B8A287FF05C0112383
:1001A00009F452CF211050CF10E0A7E08E859F8533
:1001B000A89FF001A99FF00D1124E00FF11FEE0F91
:1001C000FF1FEE0FFF1FE456FD4E418052806380FB
:1001D0007480C12CD12CE0EAEE2EE0E4FE2E222029
:1001E00051F023E333E343EB5EE3C301B2010F9429
:1001F000C3A16B017C01A70196016091FD11709173
:10020000FE118091FF11909100120F94B8A287FF08
:1002100010C0C092FD11D092FE11E092FF11F09239
:10022000001265E575E585E591E40F942F850F943F
:10023000CE22688979898A899B896093F5117093A8
:10024000F6118093F7119093F8118092F911909222
:10025000FA11A092FB11B092FC1169EF71E185EFE8
:1002600091E10E949C6360E070E086E193E40F946A
:100270002F850F94CE228091AC0D882339F07F8199
:100280007093C70688858093AC03FBCC812C912C9E
:1002900070E2A72E71ECB72E222051F02A813B810B
:1002A0004C815D81C301B2010F94C2A14B015C017D
:1002B000488DC501B4010F94BA5681110BC087E275
:1002C00092E60E94A76C9F938F930F945D9F0F906F
:1002D0000F90BECE2091FD113091FE114091FF1183
:1002E00050910012C701B6010F94C2A120E030E086
:1002F000A9010F94B8A287FF36C060E070E080EAE1
:1003000090E46093FD117093FE118093FF11909320
:10031000001265E575E585E591E40F942F850F944E
:10032000CE22488DC501B4010F94BA56882339F204
:100330002091FD113091FE114091FF11509100125A
:1003400060E070E080EA90E40F94C2A12DEC3CECF8
:100350004CEC5DE30F94B8A287FF05C08DEF96E7E4
:100360000F94849F75CEC090FD11D090FE11E09047
:10037000FF11F09000122220A1F0A7019601C30105
:10038000B2010F94C2A19B01AC015F776A817B81AE
:100390008C819D810F94B8A287FF03C084EC96E7FF
:1003A000DFCF8FEA9FE00F949BA0882309F440C021
:1003B00086EA9FE00F949BA08823D1F160918E067E
:1003C00070918F0680919006909191060E9404563C
:1003D00020913E0430913F044091400450914104EB
:1003E0000F94C2A29B01AC01E7E0AE85BF85EA9FF6
:1003F000C001EB9F900D1124080F191F000F111F52
:10040000000F111F04561D4EC701B6010F94C2A163
:10041000D80111966D937D938D939C931497809141
:10042000AC0381508093AC0381E00E9438690CCE0C
:1004300020E030E0A901D8CF85E00F942B2DC12C0E
:10044000D12C90EAE92E90E4F92E80E096E30E9408
:10045000A76C0F94220B90E080E00F94593581E057
:100460000F94B53580E00F94062D182F60E070E0F2
:1004700080E89FEB0E94D36681E00F94062DC09226
:10048000FD11D092FE11E092FF11F092001265E58D
:1004900075E585E591E40F942F850F94CE22812F89
:1004A0000F94062D82E00F94BA2220E030E040EA5B
:1004B00050E40F944CA4181644F2EF81E093C70661
:1004C000F885F093AC0381E00E94B669DD24D394F3
:1004D000DF92812C912C5401CC24C394E12CF12C7B
:1004E000870121E040E050E0BA0181E00E946967A5
:1004F000D092E6110F90C5CB10923F038BA19CA127
:100500000E94CA5F10922A051092290580E10E947C
:1005100052D8882391F00E94A87281EA9DE00F943E
:100520009BA02BE0829FC0011124805B924F0F940F
:10053000A9A090932A0580932905609129057091BF
:100540002A05072E000C880B990B0F94299B9058B5
:1005500020913E0430913F04409140045091410469
:100560000F94C2A20F94908B80EC9FE00F949BA0FD
:1005700091E0813009F090E099834FEB5FE06CE40B
:10058000CE0101960E945A55F82E4EEB5FE062E5CF
:10059000CE0101960E945A55082F4DEB5FE066E4AC
:1005A000CE0101960E945A55182F4CEB5FE062E491
:1005B000CE0101960E945A55212F110F330B082EA0
:1005C000000C990B5C01A21AB30A8F2DFF0C990B3A
:1005D000280F391F46E0429F6001439FD00C112431
:1005E000F12CE12C002E000C110B081B190BB7018C
:1005F00063567D4E3B01460177E07A83D3012D900F
:100600003D904D905D903D01FD013497FB87EA8759
:10061000B401092C000C880B990B0F94299B2FE334
:1006200033EC4EE259E30F94689BA20191010F94C1
:10063000C3A1AA85BB856D937D938D939C931397DE
:10064000BA81B150BA83800E911EB111D7CFCA0CB6
:10065000DB1CECE1EE0EF11CF4ECEF16F10439F6C4
:100660000E9436F18DE40E942B55882309F484C042
:100670000E9440552E81273009F094C0882309F448
:1006800091C0BB24B394AA24AA94AB0C09A11AA1CB
:10069000612C8EEF882E8B0C6A2D862D0F945B8B30
:1006A00099249394960C81116EC06B2D862D0F9416
:1006B0005B8BC12CD12C7601712C882381F020E03A
:1006C00030E0A901D8015D966D917D918D919C914D
:1006D00090970F94C3A16B017C0177247394682DCC
:1006E000862D0F945B8B882369F0F8017B9720811E
:1006F000318142815381C701B6010F94C3A16B01BF
:100700007C0173946A2D892D0F945B8B882361F093
:10071000F8012581368147815085C701B6010F94C4
:10072000C3A16B017C0173946A2D8FEF860D0F942A
:100730005B8B882331F1F80133972081318142812D
:100740005381C701B6010F94C3A16B017C0173945F
:10075000672D70E090E080E00F94299B9B01AC0135
:10076000C701B6010F94C2A2D80111966D937D9373
:100770008D939C93149707C08CEA9DE00F949BA0E7
:1007800079CF7110E5CF692C0C5F1F4FB7E09B123A
:1007900083CFB394E9A1FAA17C96FAA3E9A3F8E088
:1007A000BF1271CF81E080939C128FE40E942B5581
:1007B000811103C00F94E58B79CC0E9440558111C3
:1007C000F9CF0E94BF5F72CC2F923F924F925F92FF
:1007D0006F927F928F929F92AF92BF92CF92DF9251
:1007E000EF92FF920F931F93CF93DF93CDB7DEB7B6
:1007F000C356D1090FB6F894DEBF0FBECDBF82E05D
:10080000809378020091CB111091CC110F51104FB1
:1008100045E050E060E271E8C8010F947A9E892BB0
:1008200009F09BC18091CA0D882309F44DC08EE266
:100830009EE70F941075882379F08091F7161F9228
:100840008F9382EF94E69F938F930F945D9F0F9009
:100850000F900F900F9008C08AE29EE70F941075DA
:10086000882341F01092D60381E0809378020E94A1
:10087000FC723AC287E29EE70F941075882321F13B
:100880008091F5169091F61661E003960F94C54C91
:100890000F948D498C018091021690910316A091BE
:1008A0000416B091051680937E1690937F16A09340
:1008B0008016B0938116802F0E9437700A30110580
:1008C00039F70F949C42D0CF86E191E80F941075D0
:1008D0008111CACF82E191E80F941075882321F12C
:1008E00040918703509188032CE3249FC001259FEA
:1008F000900D11249F938F9340918503509186030F
:10090000249FC001259F900D11249F938F9386E211
:1009100097E69F938F930F945D9F0F900F900F908A
:100920000F900F900F90A0CF8DE091E80F9410756D
:10093000882311F18CE89FE00F949BA0811110C0D7
:1009400061E085EE9BE60E94AC7C60E085EA9FE07A
:100950000F94BFA060E08FE79CE00F94BFA084CF0E
:10096000813009F081CF0F94E22085ED91E10F9461
:100970005E100F94081078CF86E091E80F94107500
:10098000882321F080E00F941C636ECF80E091E813
:100990000F94107581110E949D608DEF90E80F9467
:1009A00010758823A9F044E150E065E17DE0CE01B7
:1009B00001960F948BA08C89882329F082EF90E810
:1009C0000F94849F51CFCE0101960F942AA74CCF4C
:1009D0008EEE90E80F941075882329F082EE90E84F
:1009E0000E94497241CF8EED90E80F9410758823D4
:1009F00019F08EEB90E8F4CF89EB90E80F94107526
:100A0000882319F00E94AA6B2FCF86EB90E80F94F1
:100A10001075882379F081EA9DE00F949BA02BE06C
:100A2000829FC001112470E060E0805B924F0F94C0
:100A3000DDA01ACF83EB90E80F941075882351F056
:100A40000E94A46940E070E060E084E690E00F94CA
:100A50006F32D8CF8FEA90E80F9410758823E1F0B9
:100A600086E50E942B55882309F4FECE0E944D5541
:100A700011E0892B09F410E00F94CE2280919C1292
:100A800090E01817190609F4EFCE10939C128DEF21
:100A900091E10F94BA75E8CE88EA90E80F9410754A
:100AA000882309F4E1CE84E40E942B558823A1F029
:100AB0000E94035A20E030E04AE754E40F94689B18
:100AC00020E030E040E05FE30F94C3A10F943BA32C
:100AD000CB010E9458F0C8CE84EA90E80F941075BC
:100AE000882349F18091CA0D882329F18091F51658
:100AF0009091F61602969093F6168093F5160E9442
:100B0000035A6B017C016FEF87EA9DE00F94BFA051
:100B100020E030E04AE754E4C701B6010F94689B37
:100B200020E030E040E05FE30F94C3A10F943BA3CB
:100B300085EA9DE07CCF85EA9DE00F94A9A0BC01E9
:100B400090E080E00F94279B20E030E04AE754E4F7
:100B50000F94C2A20F94454287CED8018C9187345E
:100B600011F00C94D8901093F6160093F5160E948D
:100B70004D5590935803809357038B34910509F496
:100B800045C60CF04BC18430910509F4AAC50CF0A0
:100B9000C5C097FDCFC002970CF0A2C10E9475544A
:100BA0008C010E942A5B6091840670918506809179
:100BB0008606909187060F94279B6B017C014090DD
:100BC00001125090021260900312709004128090F3
:100BD0009F069090A006A090A106B090A206A50145
:100BE0009401C301B2010F94C2A120E030E048ECAF
:100BF00052E40F94689B9B01AC01C701B6010F94AE
:100C00004CA41816D4F4A3019201C501B4010F94A9
:100C1000C2A120E030E048EC52E40F94689BA701A9
:100C200096010F94C3A10F943BA360938406709325
:100C3000850680938606909387068091B404882366
:100C400009F446C188E50E942B55811141C189E50F
:100C50000E942B5581113CC18AE50E942B558111C0
:100C600037C185E40E942B55882309F431C12091B6
:100C700001123091021240910312509104126091BE
:100C80009F067091A0068091A1069091A2060F94F4
:100C9000C2A16B017C012DEC3CEC4CEC5DEB0F94A4
:100CA000B8A287FF07C18091030581110C941BB086
:100CB0000F94CE2280919F069091A006A091A1064C
:100CC000B091A2068093011290930212A093031296
:100CD000B093041281E092E10F948775909103051F
:100CE00081E089270E9450BECD59DF4F0FB6F8949E
:100CF000DEBF0FBECDBFDF91CF911F910F91FF904F
:100D0000EF90DF90CF90BF90AF909F908F907F90AB
:100D10006F905F904F903F902F900895853191058F
:100D200009F4D9C0FCF48A30910509F423C50B9766
:100D300009F424C58091CB119091CC118F51904F23
:100D40009F938F931F9287E48F9388E496E69F93F7
:100D50008F930F945D9F0F900F900F900F900F90B7
:100D60000F90B9C08C31910509F40AC54E9711F75F
:100D70000F94CE2281E0809305120E94E45F8C01E3
:100D800080E090E0A8E4B4E480937A0290937B0240
:100D9000A0937C02B0937D0243E060E070E080E2CB
:100DA00091EC0F94BA567090FD116090FE11509026
:100DB000FF1140900012B090F911A090FA1190909C
:100DC000FB118090FC11F090F511E090F611D0909D
:100DD000F711C090F8118DE695E50E94A76C4F922F
:100DE0005F926F927F928F929F92AF92BF92CF92BB
:100DF000DF92EF92FF929F938F9381E097E69F930C
:100E00008F930F945D9FC8010E94CA5F10920512D4
:100E10000FB6F894DEBF0FBECDBF5DC0883591051B
:100E200009F459C0F4F48135910511F40C941E9025
:100E30005CF48C34910509F40CC58035910509F0FA
:100E400079CF0E940A7E47C08635910511F40C9433
:100E500022908735910509F06DCF80E10E9483C60D
:100E60003AC08C35910511F40C942E9074F48A35A7
:100E7000910511F40C9427908B35910509F05ACF08
:100E80008091EB1187600C942A908236910511F4C1
:100E90000C94C5908336910509F04CCF1092CA0D81
:100EA00060E084EC9FE00F94BFA082E00E9438696C
:100EB0000C94D4902DEC3CEC4CEC5DE3C701B601F6
:100EC0000F944CA4181624F4809103058111F0CEE0
:100ED000C8010E94FA641092580310925703C4CCC0
:100EE0000E9475542E969FAF8EAF2E970E942A5B5C
:100EF00089E40E942B55882309F4A0C30E94035A59
:100F000060934F0370935003809351039093520367
:100F10008AE40E942B55C12CD12C7601882321F024
:100F20000E94035A6B017C01C0925303D092540378
:100F3000E0925503F0925603E0915703F091580365
:100F4000A496FFAFEEAFA49780904F03909050030C
:100F5000A0905103B0905203A7019601C501B401BE
:100F60000F945FA424966CAF7DAF8EAF9FAF249794
:100F700060918E0270918F02072E000C880B990BE6
:100F80000F94299B20917A0230917B0240917C0240
:100F900050917D020F94689B2EE333EC4EE259E3AF
:100FA0000F94689B68AF79AF8AAF9BAF80E1E5EFA4
:100FB000F1E1DE01119601900D928A95E1F7A5010C
:100FC0009401505828A739A74AA75BA7D701C601A3
:100FD000B0588CA79DA7AEA7BFA729813A814B81A6
:100FE0005C8128962CAF3DAF4EAF5FAF2897C5010F
:100FF000B4010F94C3A162966CAF7DAF8EAF9FAF6B
:1010000062978D819E81AF81B8852C968CAF9DAF04
:10101000AEAFBFAF2C979C01AD01C701B6010F94D5
:10102000C3A166966CAF7DAF8EAF9FAF66972985E3
:101030003A854B855C8560919B0670919C068091FA
:101040009D0690919E060F94C2A16A966CAF7DAFEB
:101050008EAF9FAF6A97209193063091940640918E
:101060009506509196066E962CAF3DAF4EAF5FAF92
:101070006E9762962CAD3DAD4EAD5FAD62976E96AC
:101080006CAD7DAD8EAD9FAD6E970F94C2A16B011F
:101090007C018091970690919806A0919906B09155
:1010A0009A06A2968CAF9DAFAEAFBFAFA2976696E1
:1010B0002CAD3DAD4EAD5FAD6697BC01CD010F943B
:1010C000C2A14B015C013090F6042090F70490918E
:1010D000F8049CABA091F904ACAFB091FE04B8AB9E
:1010E000A701960168A579A58AA59BA50F94689B81
:1010F0002B013C01A50194016CA57DA58EA59FA5A2
:101100000F94689B9B01AC01C301B2010F94C3A172
:101110002B013C01A501940168A579A58AA59BA591
:101120000F94689B4B015C01A70196016CA57DA5FE
:101130008EA59FA50F94689B9B01AC01C501B401CE
:101140000F94C2A1A30192010F9442A26B017C01F2
:1011500020E030E0A9010F94B8A287FF0AC02BED70
:101160003FE049EC50E4C701B6010F94C3A16B0105
:101170007C016091FF04709100056115710509F40F
:1011800061C290E080E00F94279B9B01AC016BED66
:101190007FE089EC90E40F94C2A224962CAD3DAD83
:1011A0004EAD5FAD24970F94689B5B018C016091FD
:1011B00001057091020561157105E1F090E080E094
:1011C0000F94279B20E030E040E752E40F94689BA7
:1011D0009B01AC0168AD79AD8AAD9BAD0F94C2A205
:1011E0003B014C019501A8010F94B8A287FF02C0F2
:1011F000530184014090FA045090FB046090FC0479
:101200007090FD049501A801B201C3010F944CA494
:10121000181684F09501A801632D722D8CA99CAD40
:101220000F94B8A22501380187FF04C0432C522C2B
:101230006CA87CACA496EEADFFADA497329751F4A8
:101240002BED3FE049EC50E4C701B6010F94C2A179
:101250006B017C016E962CAD3DAD4EAD5FAD6E97D2
:1012600028966CAD7DAD8EAD9FAD28970F94B8A23A
:10127000811123C0A2962CAD3DAD4EAD5FADA297BE
:101280002C966CAD7DAD8EAD9FAD2C970F94B8A212
:10129000811113C020E030E0A901C701B6010F940D
:1012A000B8A281110AC02BED3FE049EC50E4C70120
:1012B000B6010F94C3A16B017C01A701960124968E
:1012C0006CAD7DAD8EAD9FAD24970F94689B6A96F3
:1012D0002CAD3DAD4EAD5FAD6A970F945FA44B0151
:1012E0005C012FE632E143E85AE30F94B8A287FD90
:1012F0009EC19201A301C501B4010F94C2A20F9433
:10130000A1A20F943BA37DAB6CAB6230710508F4D6
:101310005EC12E964EAD5FAD2E97452B09F457C199
:1013200090E080E00F94279B4B015C01AC019B0196
:10133000C701B6010F94C2A22B013C01A501940183
:101340006A966CAD7DAD8EAD9FAD6A970F94C2A2CB
:1013500028966CAF7DAF8EAF9FAF28972D853E85C9
:101360004F85588960919F067091A0068091A106D3
:101370009091A2060F94C2A1A50194010F94C2A25C
:101380002C966CAF7DAF8EAF9FAF2C97A3019201CF
:10139000C301B2010F94689B6B017C01AC019B01FE
:1013A000C301B2010F94689B20E030E040EC50E4B0
:1013B0000F94C2A29B01AC01C301B2010F94C2A160
:1013C0006CAF7DAF8EAF9FAF20E030E040E05FE3D9
:1013D000C701B6010F94689B9B01AC0160E070E00F
:1013E00080E89FE30F94C2A124966CAF7DAF8EAFCF
:1013F0009FAF249722242394312CD8A8DA9458A99B
:10140000511125C1B10190E080E00F94279BA30109
:1014100092010F94689B6B017C010F94BDA26CA795
:101420007DA78EA79FA7C701B6010F9483A54B0187
:101430005C01C0904F03D0905003E0905103F090B6
:101440005203F7FAF094F7F8F094809153039091D7
:101450005403A0915503B091560388AB99ABAAAB46
:10146000BBABA70196016CA57DA58EA59FA50F948A
:10147000689B68A779A78AA79BA728A939A94AA921
:101480005BA9C501B4010F94689B9B01AC0168A5E1
:1014900079A58AA59BA50F94C3A168A779A78AA758
:1014A0009BA7A7019601C501B4010F94689B6B012E
:1014B0007C0128A939A94AA95BA96CA57DA58EA59F
:1014C0009FA50F94689B9B01AC01C701B6010F94C7
:1014D000C2A16CA77DA78EA79FA79091FE0498AB91
:1014E00028A539A54AA55BA562966CAD7DAD8EADEC
:1014F0009FAD62970F94C3A169837A838B839C838A
:101500002CA53DA54EA55FA566966CAD7DAD8EADB7
:101510009FAD66970F94C3A16D837E838F83988759
:1015200028962CAD3DAD4EAD5FAD289769857A8587
:101530008B859C850F94C3A169877A878B879C874D
:101540002C962CAD3DAD4EAD5FAD2C976D857E8557
:101550008F8598890F94C3A16D877E878F87988B1D
:10156000CE0101960E94BB642E96AEADBFAD2E9704
:101570002A163B06F8F0E984FA840B851C852D8138
:101580003E814F81588569817A818B819C813F9210
:101590002F92E5EFF1E1FF93EF9388AC99ACAAAC01
:1015A000BBACFE013D966F010F94E1750F900F905B
:1015B0000F900F908091AC0D811139C0FFEF2F1A61
:1015C0003F0A2CA93DA92215330509F016CF83E95E
:1015D00096E00E94BB64E0909B06F0909C06009110
:1015E0009D0610919E062091970630919806409195
:1015F000990650919A066091930670919406809195
:101600009506909196061F921F92E5EFF1E1FF93E8
:10161000EF9388AC99ACAAACBBACEFE9CE2EE6E078
:10162000DE2E0F94E1750F900F900F900F900E9497
:10163000AC548AE493E00F9429124DCC60E070E042
:10164000CB015ECCA32CB22C0CA91CADB0CD28A52F
:1016500039A54AA55BA56CAD7DAD8EAD9FAD0F9450
:10166000689B4B015C012CA53DA54EA55FA524966A
:101670006CAD7DAD8EAD9FAD24970F94689B9B01A3
:10168000AC01C501B4010F94C3A17B018C0128A555
:1016900039A54AA55BA524966CAD7DAD8EAD9FADF9
:1016A00024970F94689B4B015C012CA53DA54EA58A
:1016B0005FA56CAD7DAD8EAD9FAD0F94689B9B011A
:1016C000AC01C501B4010F94C2A168A779A78AA78C
:1016D0009BA7D8AAC701D8018CA79DA7AEA7BFA773
:1016E000FFCE80E50E942B55C12CD12C760188239A
:1016F00031F00E94035A0F943BA36B017C0183E5F8
:101700000E942B55882361F00E94035A20E030E0AC
:101710004AE754E40F94689B0F943BA36B017C0150
:10172000C114D104E104F10441F08091C70687306F
:1017300021F08DE197E60E9499E60F94CE220F9456
:10174000FC0FC60ED71EE81EF91E8AE493E00F9424
:1017500029120F94FC0F6C157D058E059F0508F06E
:10176000BACB0F94133380E00E94FE7980E00E9490
:101770003869EFCF81E00E9450BEADCB80E0FBCF57
:1017800088E50E942B55382E412C512C320188239C
:1017900021F00E9493552B013C0189E50E942B55B5
:1017A000282E882371F10E9493556CA77DA78EA7E0
:1017B0009FA78AE50E942B55D82E812C912C54018D
:1017C000882321F00E9493554B015C0187E50E941C
:1017D0002B5588A78F93CD2CECA4FDA40EA51FA597
:1017E000222DB301A201832D0E9469670F90311051
:1017F00072CB211070CB38A531116DCBD1106BCBD2
:1018000020CB1CA61DA61EA61FA6D3CF08E210E063
:1018100098EFE92E96E6F92E602F70E090E080E0D8
:101820000F94279B0E9404569F938F937F936F93EF
:101830001F930F93FF92EF920F945D9F0F5F1F4FC7
:101840000FB6F894DEBF0FBECDBF0F36110521F7DE
:1018500042CB0F943A15811105C080E990E80E94AF
:10186000497239CB82E00E9452D8811107C08AEDBB
:1018700099E30E94A76C0F94A90B2DCB8091A3062E
:10188000882341F08091A406882321F0D090A506FA
:10189000D11008C081E08093E61182E198E60F94B0
:1018A000164419CB81E999E30E94A76C0F94A90B08
:1018B00089ED90E50E94A76C41E060E00F948A2ECC
:1018C00081116EC080E090E0A0EAB0E48093FD1149
:1018D0009093FE11A093FF11B093001260E070E0AE
:1018E00088E492E40F942F8580E090E0A8E4B2E4CD
:1018F0008093FD119093FE11A093FF11B0930012FD
:1019000080E090E0A4E3B3E48093F9119093FA119E
:10191000A093FB11B093FC1160E070E088E492E4C6
:101920000F942F850F94CE228FEA90E50E94A76C2A
:101930000F94A90BE0E5F8E885919591A591B491F4
:101940008093F9119093FA11A093FB11B093FC11BD
:10195000ECE4F8E885919591A591B4918093F51107
:101960009093F611A093F711B093F81160E070E036
:1019700088E492E40F942F850F94CE2281E08F9318
:10198000812C912C5401CC24C394E12CF12C87019F
:1019900020E040E050E0BA0180E00E9469670F90CB
:1019A00020E030E04CE052E460918E0670918F06AA
:1019B00080919006909191060F944CA418160CF00B
:1019C00076C08091CA0D811172C080E090E0A8ECD1
:1019D000B2E48093FD119093FE11A093FF11B09398
:1019E000001260E070E088E492E40F942F850F9479
:1019F000E71219821A821B821C821D82CE01019677
:101A00000F94291283E2F82E0FE11EE720E030E068
:101A10004CE052E460918E0670918F0680919006A2
:101A2000909191060F944CA41816C4F583E499E3A1
:101A30000E94A76C0F94220B42E864E080E00E94B1
:101A400091691F92FF9260918E0670918F0680912E
:101A50009006909191060F9434A37F936F931F93F8
:101A60000F930E944A6981E80E94606988EE93E0C2
:101A70000E94457C0E945E7040E053E567E070E0A4
:101A8000CE0101960F946A100F900F900F900F9057
:101A90000F900F90882309F4B9CFD12C81E00E94D8
:101AA000B669D11004C080E00F943A0C14CA0F94A8
:101AB000CE2281E0809305120E94B66982E790E809
:101AC0000E94497280908E0690908F06A09090069A
:101AD000B090910620E030E040EA50E4C501B40146
:101AE0000F94C2A20F9434A325E0269FA001279F44
:101AF000500D1124BA01550F880B990B0F94299B97
:101B00001B017C0120E030E04CE052E40F94B8A2CD
:101B100087FF06C0212C312C1CE0E12E02E4F02EC0
:101B2000222D332D4E2D5F2DC501B4010F944CA4F1
:101B3000181664F420E030E040EA50E4622D732D82
:101B40008E2D9F2D0F94C3A11B017C01FF92EF925C
:101B50003F922F928FED96E69F938F930F945D9F08
:101B600020E030E040EF51E4622D732D8E2D9F2D4B
:101B70000F94C2A120E030E04CE852E40F94C3A1DE
:101B80000F9434A37093EE116093ED1184E0809371
:101B9000C70681E08093AC0385EE9AE30E94A76CB0
:101BA0000E9499E680E090E0A0EAB0E48093FD1105
:101BB0009093FE11A093FF11B093001260E070E0CB
:101BC00088E492E40F942F8580E090E0A0EAB1E4ED
:101BD0008093F5119093F611A093F711B093F8113B
:101BE00080E090E0A0E7B2E48093F9119093FA11BD
:101BF000A093FB11B093FC1160E070E088E492E4E4
:101C00000F942F858AE999E9A9E1BEE38093FD113C
:101C10009093FE11A093FF11B093001260E070E06A
:101C200088E492E40F942F850F94CE220F900F90AA
:101C30000F900F900F900F9020918E0630918F068D
:101C40004091900650919106622D732D8E2D9F2DFF
:101C50000F944CA418163CF488EE93E00E94457C47
:101C60000E945E70E9CF60E086EA9FE00F94BFA01B
:101C700080E090E0A0EAB0E48093FD119093FE1123
:101C8000A093FF11B093001260E070E088E492E44A
:101C90000F942F85ECE4F8E885919591A591B49186
:101CA0008093F5119093F611A093F711B093F8116A
:101CB000E0E5F8E885919591A591B4918093F911AB
:101CC0009093FA11A093FB11B093FC1160E070E0C7
:101CD00088E492E40F942F850F94CE2243E060E0D5
:101CE00070E080E89FEB0F94BA56811105C00F9405
:101CF0003A0C10920512EFC89091FD1198A7A0918F
:101D0000FE11ACA7B091FF11B8ABE0910012E8AFA3
:101D1000EF93BF93AF939F9382ED96E69F938F933C
:101D20000F945D9F0F900F900F900F900F900F905A
:101D3000AEEA8A2EAFE09A2EB3E2CB2ED12C0FEF73
:101D40001FEFB6010D2C000C880B990B0F94299BEB
:101D50002B013C01DF92CF92C80102969F938F9393
:101D600026E936E63F932F930F945D9F58015FEF6E
:101D7000A51AB50A0F900F900F900F900F900F902B
:101D800011F40C9429B070E060E0C4010F94DDA060
:101D9000A3019201622D732D8E2D9F2D0F94B8A259
:101DA000181644F485E0A816B10411F00C9435B06F
:101DB00005E010E0580197E2A91A98EFB90AAA0CB9
:101DC000BB1C85E0809F1001819F300C11240D5FAA
:101DD0001F4FEAE94E2EE9E95E2EE9E16E2EEEE3B1
:101DE0007E2EFDE58F2EF6E69F2EC8010297059701
:101DF0000CF0D4C0B101635D7F4F072E000C880B3F
:101E0000990B0F94299B6B017C011F930F93A9E8F9
:101E1000B6E6BF93AF930F945D9F0093AC0320E0B1
:101E200030E040EF51E4C701B6010F94C2A120E0B9
:101E300030E040E251E40F94689B20E030E040EA5B
:101E400050E40F94C2A220E030E048E452E40F9442
:101E5000C3A10F9434A37093EE116093ED1180E051
:101E600090E0A0EAB0E48093FD119093FE11A0935E
:101E7000FF11B093001260E070E088E492E40F94E8
:101E80002F8520E030E040EA51E42093F5113093B3
:101E9000F6114093F7115093F81180E090E0A0E71D
:101EA000B2E48093F9119093FA11A093FB11B093CF
:101EB000FC1160E070E088E492E40F942F8540927A
:101EC000FD115092FE116092FF117092001260E0BD
:101ED00070E088E492E40F942F850F94CE220F9047
:101EE0000F900F900F9020918E0630918F064091A9
:101EF000900650919106C701B6010F944CA4181694
:101F00003CF488EE93E00E94457C0E945E70EBCF2B
:101F100080E090E0A0EAB0E48093FD119093FE1180
:101F2000A093FF11B093001260E070E088E492E4A7
:101F30000F942F85ECE4F8E885919591A591B491E3
:101F40008093F5119093F611A093F711B093F811C7
:101F5000E0E5F8E885919591A591B4918093F91108
:101F60009093FA11A093FB11B093FC1160E070E024
:101F700088E492E40F942F850F94CE2243E060E032
:101F800070E080E89FEB0F94BA5695E0290E311C63
:101F90000F5F1F4F811104C00F943A0C81E0A7CE50
:101FA00078A56CA598A988AD272F362F492F582FD3
:101FB0006091FD117091FE118091FF1190910012BE
:101FC0000F94C2A1F62EE72ED82EC92E20913E04E2
:101FD00030913F044091400450914104D701F601F3
:101FE0006B2F7A2F8F2F9E2F0F94689B0F9434A303
:101FF0006CAB7DAB8EAB9FABCF92DF92EF92FF923B
:10200000809191068F93809190068F9380918F0697
:102010008F9380918E068F939F928F920F945D9FE6
:102020006CA97DA9C5010F94DDA0A2E0AA0EB11C88
:102030000FB6F894DEBF0FBECDBFD7CE0E942D7372
:102040000C946B8780E10E942EC60C946B87809164
:10205000EB11887F8093EB110C946B8754ECC52EA9
:1020600052E0D52E8E010C5D1F4F5801EE24E394F3
:10207000F12CD6018D916D010E942B55F5018193B4
:102080005F01882391F00E94035AF701EE0FFF1FB2
:10209000EE0FFF1F349721E030E02C0F3D1FE20FC1
